:020000040800F2
:1000000000060020E1010008CD0D0008D10D000818
:10001000290E0008D10D0008FD0D0008E3010008BD
:10002000E3010008E3010008E30100083D210008A6
:10003000E3010008E3010008E3010008E301000810
:10004000E3010008E3010008E3010008E301000800
:10005000E3010008E30100081D32000849320008EE
:1000600075320008A1320008CD320008E301000813
:10007000E3010008E3010008E3010008E3010008D0
:10008000E3010008E3010008E3010008E3010008C0
:10009000E3010008E3010008E3010008F932000869
:1000A000E3010008E3010008E3010008E3010008A0
:1000B00091300008E3010008E3010008E3010008B3
:1000C000E3010008E3010008E3010008E301000880
:1000D000E3010008E3010008E3010008E301000870
:1000E00061330008E3010008E3010008E3010008B0
:1000F000E3010008E3010008E3010008E301000850
:10010000E3010008E3010008E3010008E30100083F
:10011000E3010008E3010008E3010008E30100082F
:10012000E3010008E3010008E3010008E30100081F
:10013000E3010008E3010008E3010008E30100080F
:10014000E3010008E3010008E3010008812800083A
:10015000E3010008E3010008E3010008E3010008EF
:10016000E3010008E3010008E3010008E3010008DF
:10017000E3010008E3010008E3010008E3010008CF
:10018000E3010008E3010008E3010008E3010008BF
:10019000E3010008E3010008E3010008E3010008AF
:1001A000E3010008E3010008E3010008E30100089F
:1001B000E3010008E3010008E3010008E30100088F
:1001C000E3010008E3010008E3010008E30100087F
:1001D000E3010008E3010008E3010008E30100086F
:1001E00002E000F000F8FEE772B6394880F30888B4
:1001F000384880F3098838484EF60851CEF200019D
:10020000086040F20000CCF200004EF63471CEF2ED
:1002100000010860BFF34F8FBFF36F8F40F2000003
:10022000C0F2F0004EF68851CEF200010860BFF334
:100230004F8FBFF36F8F4FF00000E1EE100A4EF6C4
:100240003C71CEF200010860062080F31488BFF3F1
:100250006F8F01F0D1FF02F077FE4FF055301F494C
:100260001B4A91423CBF41F8040BFAE71C49194A6A
:1002700091423CBF41F8040BFAE71A491A4A1B4B5A
:100280009A423EBF51F8040B42F8040BF8E70020F5
:100290001749184A91423CBF41F8040BFAE701F0B4
:1002A000AFFF02F0ADFE144C144DAC4203DA54F82B
:1002B000041B8847F9E700F041F8114C114DAC429E
:1002C00003DA54F8041B8847F9E701F097BF0000F0
:1002D000000600200022002000000008000000208E
:1002E0000006002090370008002200203C22002059
:1002F00040220020A42D0020E0010008E0010008B9
:10030000E0010008E00100082DE9F04F2DED108A12
:10031000C1F80CD0C3689D46BDEC108ABDE8F08FD3
:10032000002383F311882846A047002001F004FB36
:10033000FEE701F085FA00DFFEE7000038B501F0C6
:10034000CFFE044601F0F4FE0546D8B90F4B9C429F
:100350001AD001339C4218BF054641F2883404BFCD
:1003600001250024002001F0C5FE0DB100F058F871
:1003700000F000FD00F09EFB204600F0AFF800F01A
:100380004FF8F9E70024EDE70446EBE7010007B07A
:1003900008B500F061FBA0F120035842584108BDA8
:1003A00007B5054B02211B88ADF8043001A800F009
:1003B00071FB03B05DF804FB5C34000810B520232A
:1003C00083F311881248C3680BB101F051FB00237D
:1003D000104A0F484FF47A7101F0F8FA002383F3C2
:1003E00011880D4C236813B12368013B23606368B7
:1003F00013B16368013B6360084B1B7833B96368D2
:1004000023B9022000F02CFC3223636010BD00BF32
:1004100040220020BD0300085C230020542200205D
:1004200010B5254B254953F8042F013200D110BDDA
:100430008B42F8D1224C234B22689A423AD9224B64
:100440009B6803F1006303F540439A4232D20020D7
:1004500000F04AFB1D4B0220187000F0FFFB1C4B04
:100460001A6C00221A64196E1A66196E596C5A6455
:10047000596E5A665A6E5A6942F080025A615A6938
:1004800022F080025A615A691A6942F000521A61D8
:100490001A6922F000521A611B6972B60D4A0E4B9E
:1004A00013601B682268202181F311889D4683F325
:1004B0000888104710BD00BFFCBF00081CC0000822
:1004C00004C00008FFBF00080022002054220020C2
:1004D0000038024008ED00E000C000082DE9F04FB0
:1004E00099B0B94D00902022FF2110A8AC6800F00F
:1004F000E3FBB64A01951378A3B9B5480121C3605F
:100500001170202383F31188C3680BB101F0B0FA96
:100510000023B04AAE484FF47A7101F057FA002335
:1005200083F31188009BAC4A03B11360AB4B009D71
:10053000029300261E705660B2463746B14601202F
:1005400000F08CFB002D00F02582A34B1B68002BD4
:1005500040F0208219B0BDE8F08F0220FFF718FFAD
:10056000002840F01082009B002E08BF1D469C4BC7
:1005700002211B88ADF82C300BA800F08BFADEE7C7
:100580004FF47A7000F068FAB0F10008EBDB02205B
:10059000FFF7FEFE0028E6D008F1FF38B8F1040F9F
:1005A00000F2F381DFE808F0031E2124270018A8D9
:1005B000052340F8343D042100F06CFA012303FACE
:1005C00008F848EA0A0A5FFA8AFA4FF0000900F0D0
:1005D000C7FB27B10AF00B030B2B08BF0025FFF761
:1005E000DFFEACE704217848E6E704217D48E3E735
:1005F00004217D48E0E74FF01C09484600F076FAF8
:1006000009F104090B9004210BA800F043FAB9F199
:100610002C0FF2D1D2E7002FA5D00AF00B030B2B41
:10062000A1D10220FFF7B4FE804600289BD0012014
:100630006A4E00F059FA0220307000F00FFB0027DC
:100640005FFA87FB584600F05FFA054688B15846C6
:1006500000F06AFA01370028F2D146460025634BC4
:1006600002211B88ADF82C300BA800F013FA474686
:1006700065E701230220337000F0EEFA2C46019B5F
:100680009B689C4206D2204600F030FA0130E4D14B
:100690000434F4E7029B00241C704F4B46465C6018
:1006A0004746254693E7002F3FF45DAF0AF00B0362
:1006B0000B2B7FF458AF029B0220187000F0CEFA8B
:1006C000322000F0C9F9B0F1000BFFF64CAF1BF07F
:1006D00003087FF448AF019B996804EB0B028A4240
:1006E0003FF641AFBBF5807F3FF63DAF404A0392F6
:1006F000D8450FDA4FF47A7000F0AEF904900499FF
:100700000029FFF630AF039A049908F8021008F1A7
:100710000108ECE7C820FFF73BFE804600283FF4C5
:1007200022AF1F2C11D8C4F120075F4528BF5F46B8
:1007300010AB24F003003A462D49184400F092FA19
:100740003A46FF212A4800F0B7FA4FEAAB03DAB283
:1007500027490393204600F0B7FA074600283FF4E4
:100760007EAF039B04EB830431E70220FFF710FE0A
:1007700000283FF4F8AE00F0FDF900283FF4F3AE96
:100780004FF000084346019A9268904532D2B8F182
:100790001F0F12D8109A01320FD028F0030218A9A7
:1007A0000A4452F8202C0B92184604220BA900F0A0
:1007B0004FFB08F104080346E5E74046039300F0C9
:1007C00095F9039B0B90EFE70022002058230020AF
:1007D00040220020BD0300085C230020542200209A
:1007E0005E34000804220020082200206034000843
:1007F0005822002018A8042140F84C3D00F04AF986
:10080000E5E618A8002340F8343D642100F038F9EB
:1008100000287FF4A8AE0220FFF7BAFD00283FF4BD
:10082000A2AE0B9800F092F918AB43F8480D0421E2
:100830001846E3E718A8002340F8343D642100F08F
:100840001FF900287FF48FAE0220FFF7A1FD0028DA
:100850003FF489AE0B9800F087F918AB43F8440DCC
:10086000E5E70220FFF794FD00283FF47CAE00F09E
:1008700091F918AB43F8400DD9E70220FFF788FD46
:1008800000283FF470AE0BA9142000F089F98046CF
:1008900018A8042140F83C8D00F0FCF841460BA854
:1008A000ACE7322000F0D8F8B0F10008FFF65BAEFC
:1008B00018F0030F7FF457AE019A926808EB090312
:1008C00093423FF650AE0220FFF762FD00283FF44E
:1008D0004AAE28F00308C844C1453FF478AE484604
:1008E00000F004F904210A900AA800F0D3F809F1F5
:1008F0000409F1E74FF47A70FFF74AFD00283FF44E
:1009000032AE00F037F9002842D0109B01330BD0F3
:10091000082210A9002000F0D7F9002838D02022A2
:10092000FF2110A800F0C8F9FFF73AFD364801F0A2
:1009300009F80FE6002F3FF416AE0AF00B030B2B5D
:100940007FF411AE18A8002340F8343D642100F074
:1009500097F8804600287FF406AE0220FFF718FDC6
:1009600000283FF400AE0390FFF71AFD41F28830F3
:1009700000F0E8FF0B9800F027FA00F0F1F9039B74
:1009800045461F46DBE5074621E64FF00009EAE54C
:10099000B84664E6002000F05FF80490049B002B4A
:1009A000FFF6D0AD012000F057F9049B213B122B3C
:1009B0003FF6C5AD01A252F823F000BF5B05000869
:1009C00081050008170600083F0500083F050008DC
:1009D0003F050008A7060008A30800086B070008E9
:1009E0000308000835080008630800083F050008F0
:1009F0007B0800083F050008F5080008CF0500083F
:100A00003F05000835090008A086010070B50F4BAE
:100A10000C4619780131C9B2012906460FD80C4895
:100A200003681D6A4FF47A73534331462246A84740
:100A3000844204D1074B00221A70012070BD4FF48C
:100A4000FA7000F07FFF002070BD00BF0C22002074
:100A5000502500209023002007B502AB002203F8A8
:100A6000012D012102461846FFF7D0FF20B19DF865
:100A7000070003B05DF804FB4FF0FF30F9E700001A
:100A80000A4608B50421FFF7C1FF80F00100C0B29B
:100A9000404208BD30B4054C2368DD69044B0A466A
:100AA000AC460146204630BC604700BF50250020C0
:100AB000A086010070B501F017FA094C094E20809C
:100AC000002530682388834208D901F007FA33688B
:100AD00005440133B5F5404F3360F2D370BD00BF1C
:100AE000922300206423002001F0ACBA00F10060E2
:100AF00000F540400068704700F10060920000F58A
:100B0000404001F037BA0000054B1A68054B1B88BE
:100B10009B1A834202D9104401F0E0B900207047CB
:100B2000642300209223002038B5074D044628682E
:100B3000204401F0DBF928B928682044BDE838409A
:100B400001F0ECB938BD00BF6423002010F00303AE
:100B500008D1B0F5047F05D200F10050A0F508409F
:100B60000068704700207047014BC058704700BFB5
:100B7000107AFF1F064991F8243033B10023082270
:100B8000086A81F82430FFF7B7BF0120704700BF23
:100B900068230020014B1868704700BF002004E064
:100BA00070B52A4B1C68C4F30B03240C63B140F2EC
:100BB0001342934231D040F2194293422FD040F277
:100BC000214293422DD10323214A0C2505FB032307
:100BD0005D6893F9082042F201039C4224D0B4F5E9
:100BE000805F23D041F201039C4221D041F20303F4
:100BF0009C421FD041F207039C4208BF3122441E91
:100C00000C44013D0B46A3421ED215F9016F581C3E
:100C100096B1034600F8016CF5E70123D4E70223FF
:100C2000D2E73F220B4DD6E73322E3E74122E1E74B
:100C30005A22E4E75922E2E72C2584421D7001D9AB
:100C4000981C5A70401A70BD1846FBE7002004E05B
:100C500070340008643400087047000070470000DA
:100C60007047000010B50023934203D0CC5CC454FD
:100C70000133F9E710BD000030B5441E14F9010F2F
:100C80000B4660B193F90050854201F1010106D194
:100C90001AB993F90020801A30BD013AEEE7002A14
:100CA000F7D1104630BD000002460346981A13F9EA
:100CB000011B0029FAD1704702440346934202D037
:100CC00003F8011BFAE770472DE9F047234C94F82D
:100CD000243005468846174683BB2E46DFF87C90B5
:100CE000C7B394F824302BB92022FF21484626624E
:100CF000FFF7E2FF94F82400C0F10805BD4228BFC9
:100D00003D465FFA85FAAD0041462A4604EB800075
:100D1000FFF7A8FF94F82430A7EB0A079A445FFA7C
:100D20008AFABAF1080F2E44A844FFB284F824A02E
:100D3000D6D1FFF71FFF0028D2D108E0266A06EBC4
:100D40008306B042CAD0FFF715FF0028C5D10020A6
:100D5000BDE8F0870120BDE8F08700BF68230020D0
:100D6000024B1A78024B1A70704700BF9023002084
:100D70000C22002038B5104D104C284600F0F8F831
:100D80002146284600F020F924680D48626DD2F80B
:100D9000043843F00203C2F8043800F0D3FD0949D7
:100DA000204600F01DFA626DD2F8043823F00203E9
:100DB000C2F8043838BD00BF502500206435000853
:100DC00040420F008C35000870470000FEE700002D
:100DD00000B59BB0EFF3098168226846FFF742FF38
:100DE000EFF30583044B9A6BDA6A9A6A9A6A9A6AF5
:100DF0009A6A9A6A9B6AFEE700ED00E000B59BB034
:100E0000EFF3098168226846FFF72CFFEFF30583B3
:100E1000044B9A6B9A6A9A6A9A6A9A6A9A6A9B6A65
:100E2000FEE700BF00ED00E000B59BB0EFF30981E5
:100E300068226846FFF716FFEFF30583034B5A6BF2
:100E40009A6A9A6A9A6A9A6A9B6AFEE700ED00E0DB
:100E500030B5084D0A4491420BD011F8013B0924EA
:100E60005840013CF7D040F300032B4083EA500088
:100E7000F7E730BD2083B8ED026843681143016095
:100E800003B118477047000013B5446BD4F894348D
:100E90001A681178042915D1217C022912D11979F7
:100EA000128901238B4013420CD101A904F14C009B
:100EB00001F04EFFD4F89444019B2179024620684A
:100EC00000F0DAF902B010BD143001F0D1BE00001C
:100ED0004FF0FF33143001F0CBBE00004C3001F076
:100EE000A3BF00004FF0FF334C3001F09DBF000066
:100EF000143001F09FBE00004FF0FF31143001F0BC
:100F000099BE00004C3001F06FBF00004FF0FF327F
:100F10004C3001F069BF0000D0F8942438B5136854
:100F200019780429054601D0012038BD017C022929
:100F3000FAD112795C89012090400440F4D105F186
:100F4000140001F031FE02460028EDD0D5F894548B
:100F50004FF480732868697900F07CF9204638BD29
:100F6000406BFFF7D9BF00000020704770470000BA
:100F70007FB5124B0360002343608360C36001258B
:100F800002260F4B057404460290019300F184027F
:100F9000294600964FF48073143001F0E1FD094BAF
:100FA0000193029400964FF4807304F5237229464E
:100FB00004F14C0001F0A8FE04B070BDC03400087C
:100FC000610F0008890E00080B68202282F3118847
:100FD0000A7903EB820290614A79093243F82200D0
:100FE0008A7912B103EB8203986102230374C0F87B
:100FF0009414002383F311887047000038B5037FF1
:10100000044613B190F85430ABB9201D01250221DC
:10101000FFF732FF04F1140025776FF0010100F0B3
:10102000B9FC84F8545004F14C006FF00101BDE8A4
:10103000384000F0AFBC38BD10B501210446043083
:10104000FFF71AFF0023237784F8543010BD000007
:1010500038B504460025143001F09AFD04F14C0027
:10106000257701F069FE201D84F854500121FFF717
:1010700003FF2046BDE83840FFF74EBF90F84430EC
:1010800003F06003202B19D190F84520212A0AD0C3
:10109000222A4FF000030ED0202A0FD1084A826383
:1010A0000722C26304E0064B83630723C363002364
:1010B0000364012070478363C363F9E7002070472E
:1010C0000D220020D0F8943437B51A68117804291D
:1010D00004461AD1017C022917D1197912890123FA
:1010E0008B40134211D100F14C05284601F0E4FE7B
:1010F00058B101A9284601F02BFED4F89444019B75
:1011000021790246206800F0B7F803B030BD000036
:1011100000EB8103F7B59C6905460E46F4B1202328
:1011200083F3118805EB8607201D0821FFF7A4FE35
:10113000FB685B691B684C3413B1204601F016FE56
:1011400001A9204601F004FE024648B1019B314648
:10115000284600F091F8002383F3118803B0F0BD16
:10116000FB685A691268002AF5D01B8A013B1340BC
:10117000F1D105F14402EAE7093138B550F82140D0
:10118000DCB1202383F31188D4F8942413685279B6
:1011900003EB8203DB689B695D6845B1042160183D
:1011A000FFF76AFE294604F1140001F007FD20460E
:1011B000FFF7B2FE002383F3118838BD70470000AB
:1011C00001F0B0B80123037000234360C361836260
:1011D0000362C3624362036303814381704700007B
:1011E00038B50446202383F3118800254160C5608B
:1011F00005614561856101F0A5F80223237085F33F
:10120000118838BD70B500EB810305465069DA607E
:101210000E46144618B110220021FFF74DFDA069BB
:1012200018B110220021FFF747FD31462846BDE8DE
:10123000704001F051B90000028902F00102028100
:10124000428902F001024281002202614261826110
:1012500001F0D6B9F0B400EB81044789E4680125B8
:10126000A4698D403D43458123600023A2606360F3
:10127000F0BC01F0F1B90000F0B400EB8104078983
:10128000E468012564698D403D43058123600023A6
:10129000A2606360F0BC01F06BBA000070B502237D
:1012A000002504460370A0F84C5080F84E5080F89A
:1012B0004F5005814581C56005614561856180F8B4
:1012C000345001F0A5F863681B6823B12946204615
:1012D000BDE87040184770BD037880F85030052392
:1012E000037043681B6810B504460BB1042198478E
:1012F00000232381638110BD436890F850201B6850
:1013000002700BB1052118477047000090F8343087
:1013100070B5044613B1002380F8343004F1440260
:10132000204601F08FF963689B6863BB94F84450D2
:1013300015F0600615D194F8453005F07F0545EAB3
:10134000032540F202339D4200F00E815BD8022D4E
:1013500000F0DC803FD8002D00F08780012D00F0E8
:10136000CF800021204601F0C7FB0021204601F07C
:10137000B9FB63681B6813B1062120469847062312
:1013800084F8343070BD204698470028CED094F8B9
:101390004B2094F84A3043EA0223E26B934238BF71
:1013A000E36394F94430E56B002B4FF0200380F2A7
:1013B000FD80002D00F0EC80092284F8342083F3B6
:1013C00011880021E36BA26B2046FFF755FF002335
:1013D00083F3118870BDB5F5817F00F0B180B5F55C
:1013E000407F49D0B5F5807FBBD194F84630012BC2
:1013F000B7D1B4F84C3023F00203A4F84C30A66304
:10140000E6632664C3E740F201639D421ED8B5F54A
:10141000C06F3BD2B5F5A06FA3D1B4F84430B3F59B
:10142000A06F0ED194F8463084F84E30204601F07B
:1014300047F863681B6813B10121204698470323CE
:1014400023700023A363E3632364A0E7B5F5106F63
:1014500032D040F602439D4252D0B5F5006F80D1A4
:1014600004F14F03A363012324E004F14C03A363BD
:101470000223E36325648AE794F84630012B7FF466
:1014800070AFB4F84C3043F00203B6E794F849204B
:10149000616894F848304D6894F8471043EA022395
:1014A000204694F84620A84700283FF45AAF4368E6
:1014B000A3630368E363A4E72378042B10D12023FC
:1014C00083F311882046FFF7B7FE86F3118863681F
:1014D00084F84F601B68032121700BB120469847A8
:1014E00094F84630002BACD084F84F30042323709E
:1014F00063681B68002BA4D0022120469847A0E710
:10150000374BA3630223E36300239DE794F848105D
:1015100011F0800F204601F00F010ED001F084F889
:10152000012806D002287FF41CAF2E4BA363E06392
:1015300067E72D4BA363E56363E701F067F8EFE727
:1015400094F84630002B7FF40CAF94F8483013F039
:101550000F013FF476AF1A06204602D501F0E0FAFB
:101560006FE701F0D3FA6CE794F84630002B7FF474
:10157000F8AE94F8483013F00F013FF462AF1B0649
:10158000204602D501F0B8FA5BE701F0ABFA58E764
:10159000142284F8342083F311882B462A462946E6
:1015A0002046FFF757FE85F3118870BD5DB1152207
:1015B00084F8342083F311880021E36BA26B20466A
:1015C000FFF748FE03E70B2284F8342083F31188E9
:1015D0002B462A4629462046FFF74EFEE3E700BF8A
:1015E000F0340008E8340008EC34000838B590F80E
:1015F00034300446152B29D8DFE803F03E2828288C
:1016000028283E28280B293928282828282828284F
:101610003E3E90F84B1090F84A20C36B42EA0122FC
:101620009A4214D9C268128AB3FBF2F502FB15354F
:101630006DB9202383F311882B462A462946FFF7EC
:101640001BFE85F311880A2384F8343038BD142337
:1016500084F83430202383F3118800231A46194676
:101660002046FFF7F7FD002383F3118838BD036C94
:1016700003B198470023E7E7002101F03DFA00217C
:10168000204601F02FFA63681B6813B1062120463B
:1016900098470623D8E7000090F83420152A38B57B
:1016A000044622D80123934040F6416213421DD1E3
:1016B00013F480150FD19B0217D50B2380F834301B
:1016C000202383F311882B462A462946FFF7D4FDB1
:1016D00085F3118838BDC3689B695B682BB9036CBF
:1016E00003B19847002384F8343038BD002101F05D
:1016F00003FA0021204601F0F5F963681B6813B175
:101700000621204698470623EDE70000024B002201
:101710001B605B609A607047942300200023037471
:101720008268054B1B6899689142FBD25A68036036
:1017300042601060586070479423002008B5202351
:1017400083F31188037C032B05D0042B0DD02BB918
:1017500083F3118808BD436900221A604FF0FF33FC
:101760004361FFF7DBFF0023F2E790E80C001A600B
:1017700002685360F2E70000002303748268054B9F
:101780001B6899689142FBD85A68036042601060F8
:101790005860704794230020054B19690874186835
:1017A00002681A605360186101230374FEF7ACBD30
:1017B0009423002030B54B1C87B005460A4C10D04E
:1017C00023690A4A01A800F001F92846FFF7E4FF5F
:1017D000049B13B101A800F04BF92369586907B0C5
:1017E00030BDFFF7D9FFF8E7942300203D1700082C
:1017F00038B50C4D41612B6981689A689142044665
:1018000003D8BDE83840FFF789BF1846FFF7B4FF9B
:1018100001232C61014623742046BDE83840FEF7C1
:1018200073BD00BF94230020044B1A681B699068A5
:101830009B68984294BF00200120704794230020A9
:1018400010B5084C236820691A6822605460012290
:1018500023611A74FFF790FF01462069BDE810402C
:10186000FEF752BD94230020FEE7000010B50C4C9B
:10187000FFF74CFF00F09CF880220A49204600F058
:1018800021F8012344F8180C037400F067FC0023CE
:1018900083F3118862B60448BDE8104000F034B804
:1018A000BC230020F4340008FC34000800F01AB90E
:1018B000034B59685A68521A9042FBD8704700BFD0
:1018C000001000E08260022202740022427470471D
:1018D0008368A3F17C0243F80C2C026943F83C2C8A
:1018E000426943F8382C074A43F81C2CC26843F875
:1018F000102C022203F8082C002203F8072CA3F175
:10190000180070472103000810B5202383F31188C5
:10191000FFF7DEFF00210446FFF76AFF002383F391
:101920001188204610BD0000024B1B6958610F2032
:10193000FFF732BF94230020202383F31188FFF7A1
:10194000F3BF000008B50146202383F31188082067
:10195000FFF730FF002383F3118808BD49B1064B20
:1019600042681B6918605A60136043600420FFF7E7
:1019700021BF4FF0FF307047942300200368984246
:1019800006D01A680260506059611846FFF7C6BE5B
:101990007047000038B504460D462068844200D1E7
:1019A00038BD036823605C604561FFF7B7FEF4E76C
:1019B000054B03F114025A619A614FF0FF32DA616C
:1019C00000221A62704700BF94230020F8B5274F09
:1019D0000361C2600D46044601F0A2FA3B46022DA7
:1019E00053F8142F294638BF02219A423E461D461D
:1019F0000AD138627C61BC61084422606260A160E7
:101A0000BDE8F84001F07ABAD7F820E0A0EB0E0369
:101A10005F181FD300279068834217D8376AAA42FD
:101A20001F44376201D0C01A906073699A6891426E
:101A300019D85A682360626014605C60A16098687D
:101A4000411A99604FF0FF33F361F8BD97601B1A9C
:101A50001268E0E793689F4203D20EEB070001F0A3
:101A60005BFA3946E1E7891A1B68DFE79423002017
:101A700038B51B4B01685A6990421D4603F11402A8
:101A80000CD0446821600368002193425C60C1600F
:101A900025D09A6881680A449A6038BD59614A60C5
:101AA0005B6900219342C16003D1BDE8384001F079
:101AB0002DBA9A6881680A449A602C6A01F030FA5B
:101AC0006A699268001B824209D9111A012998BFDC
:101AD000821C286ABDE83840104401F01DBA38BDA8
:101AE000942300202DE9F84F204C0027656904F16C
:101AF0001406B84601F014FA236AA0EB030AAB6897
:101B000053451DD84FF02009236AAA68D5F80CB0B8
:101B100013442362AB68AAEB030A2B68B3425E60EE
:101B20006361EF6001D101F0F1F988F31188286950
:101B3000D84789F311886569AB689A45E4D2D9E73B
:101B40006369B34210D020629A68A2EB0A029A60DD
:101B5000226AAB68821A9B1A022B2CBFC018023073
:101B6000BDE8F84F01F0D8B9BDE8F88F9423002004
:101B700000207047FEE70000704700004FF0FF3084
:101B800070470000022906D0032906D00129064823
:101B900018BF0020704705487047032A9ABF0448C1
:101BA00000EBC20000207047E83500089C350008B3
:101BB0001C22002070B59AB001AD064608462946A1
:101BC000144600F0BDF82846FFF76EF8C0B2431C7B
:101BD0005B0086E81800237003236370002302343F
:101BE0001946DAB2904204F1020401D81AB070BD6D
:101BF000EA5C04F8022C04F8011C0133F1E7000050
:101C000008B5202383F311880348FFF75BFA00230C
:101C100083F3118808BD00BF5025002090F84430A0
:101C200003F01F02012A07D190F845200B2A03D1A7
:101C300000238363C36312E003F06003202B11D100
:101C4000B0F8483073B990F84520212A03D0222AF1
:101C5000EFD0202A06D1044A82630722C2630364BC
:101C600001207047FFF70ABA1422002010B504467D
:101C7000052916D8DFE801F016150316161D2023D6
:101C800083F311880E4A0121FFF7BCFA20460D4A62
:101C90000221FFF7B7FA0C48FFF7DAF9002383F3C4
:101CA000118810BD202383F311880748FFF7A6F998
:101CB000F4E7202383F311880348FFF7BDF9EDE72C
:101CC0001C350008403500085025002038B50C4D63
:101CD0000C4C0D492A4604F10800FFF76BFF05F193
:101CE000CA0204F110000949FFF764FF05F5CA7242
:101CF00004F118000649BDE83840FFF75BBF00BF9C
:101D0000182A00201C2200206C35000876350008B7
:101D10008135000870B5044608460D46FEF7C4FF3D
:101D2000C6B22046013403780BB9184670BD32465E
:101D30002946FEF7A1FF0028F3D1012070BD000065
:101D40002DE9F04704460D46FEF7AEFF2D49C6B219
:101D50002046FFF7DFFF08B10836F6B22A492046D1
:101D6000FFF7D8FF08B11036F6B2632E0BD8DFF8B4
:101D70009480DFF89490254FDFF89CA0267846B930
:101D80002E70BDE8F08721462846BDE8F04701F0F7
:101D90005DBB252E31D1072241462046FEF76CFF60
:101DA00080B91B4B2A4603F10C0153F8040B42F88F
:101DB000040B8B42F9D119889B78118093700734FA
:101DC0000F35DBE7082249462046FEF755FFA0B94C
:101DD000104BAA1C13F8011F09095345C95D02F8ED
:101DE000021C197801F00F0102F10202C95D02F82C
:101DF000031CEFD118350834C0E72E7001340135CB
:101E0000BCE700BF0836000881350008203600080E
:101E1000103600080F7AFF1F1B7AFF1FBFF34F8F8A
:101E2000024AD368DB03FCD4704700BF003C024089
:101E300008B5094B1B7873B9FFF7F0FF074B1A6918
:101E4000002ABFBF064A5A6002F188325A601A68F7
:101E500022F480621A6008BD762C0020003C02400B
:101E60002301674508B50B4B1B7893B9FFF7D6FFE5
:101E7000094B1A6942F000421A611A6842F4805212
:101E80001A601A6822F480521A601A6842F480625A
:101E90001A6008BD762C0020003C02400B2870B56B
:101EA00013D80B4A0B4C137863B90B4E4FF00061FB
:101EB00044F8231056F8235001330C2B2944F7D152
:101EC0000123137054F8200070BD002070BD00BFC6
:101ED000A82C0020782C002034360008014B53F841
:101EE00020007047343600080C2070470B2810B5CE
:101EF000044601D9002010BDFFF7D0FF064B53F870
:101F000024301844C21A0BB9012010BD12680132E6
:101F1000F0D1043BF6E700BF343600080B2810B5BB
:101F2000044621D8FFF77AFFFFF782FF0F4AF32319
:101F3000D360C300DBB243F4007343F002031361C8
:101F4000136943F480331361FFF768FFFFF7A6FFBF
:101F5000074B53F8241000F0DDF8FFF783FF20460D
:101F6000BDE81040FFF7C2BF002010BD003C02409A
:101F7000343600082DE9F84312F00103154640D12C
:101F80008218B2F1016F3CD22C4B1B6813F0010395
:101F900037D02B4CFFF74CFFF323E360FFF73EFFF6
:101FA00040F20127032D01D9830713D0244C0F469B
:101FB000401A40F20118EB1B0B44012B00EB070603
:101FC000236924D823F001032361FFF74BFF01208D
:101FD000BDE8F883236923F44073236123693B43FD
:101FE000236151F8046B0660BFF34F8FFFF716FFB4
:101FF00003689E4208D0236923F001032361FFF7A1
:1020000031FF0020BDE8F883043D0430CAE723F423
:1020100040732361236943EA08032361B94637F813
:10202000023B3380BFF34F8FFFF7F8FE3688B9F8D5
:102030000030B6B2B342BED0DDE700BF0038024088
:10204000003C0240084908B50B7828B153B9FFF7A6
:10205000EFFE01230B7008BD23B1BDE808400870F6
:10206000FFF700BF08BD00BF762C002010B502446A
:10207000064B0439D2B2904200D110BD441C00B2CC
:1020800053F8200041F8040FE0B2F4E75028004074
:10209000104B30B51C6F240407D41C6F44F400743B
:1020A0001C671C6F44F400441C670B4C236843F40A
:1020B000807323600244094B0439D2B2904200D1AC
:1020C00030BD441C00B251F8045F43F82050E0B228
:1020D000F4E700BF00380240007000405028004084
:1020E00007B5012201A90020FFF7C0FF019803B046
:1020F0005DF804FB13B50446FFF7F2FFA04206D0DB
:1021000002A9012241F8044D0020FFF7C1FF02B0EF
:1021100010BD000070470000034B1B689B0042BFCE
:10212000024B01221A70704774380240A92C00201B
:10213000014B1878704700BFA92C0020EFF30983EA
:1021400005494A6822F001024A60683383F309882E
:10215000002383F31188704730EF00E0202080F3E4
:10216000118862B60B4B0C4AD96821F4E06109046E
:10217000090C0A430949DA60CA6842F08072CA60F1
:1021800007490A6842F001020A601022DA7783F8F0
:102190002200704700ED00E00003FA05F0ED00E0DA
:1021A000001000E010B5202383F311880E4B5B680C
:1021B00013F4006314D0F1EE103AEFF30984683C95
:1021C0004FF08073E361094BDB68236684F3098871
:1021D000FFF72AFB10B1064BA36110BD054BFBE7CF
:1021E00083F3118810BD00BF00ED00E030EF00E088
:1021F000330300083603000870470000FEE70000C4
:10220000084A094B09498B4204D3094A00219342E9
:1022100005D3704752F8040F43F8040BF3E743F873
:10222000041BF4E7C8370008A42D0020A42D0020CB
:10223000A42D0020836D70B5446D9E6800214FF081
:10224000FF354A01A3180131D3F800090028BEBFA9
:10225000D3F8000940F08040C3F80009D3F8000B20
:102260000028BEBFD3F8000B40F08040C3F8000B3D
:10227000A3188E42C3F80859C3F8085BE1D24FF0A7
:102280000113C4F81C3870BD890141F020010161BF
:1022900003699B06FCD41220FFF70ABB204B03EB1B
:1022A00080022DE9F047D2F80CE05D6DDEF81420D5
:1022B000461CD2F800C005EB063605EB4018516805
:1022C00061450BD3D5F83428012303FA00F022EA44
:1022D0000000C5F834081846BDE8F087BEF8104085
:1022E000ACEB0103A34228BF2346D8F81849A4B297
:1022F000B3EB840F10D894681F46A4F1040959F871
:1023000004AFC6F800A0042F01D9043FF7E71C442E
:102310000B4494605360D2E70020BDE8F08700BF13
:10232000AC2C002010B5054C2046FEF74BFF4FF0BB
:10233000A0436365024BA36510BD00BFAC2C002019
:10234000883600080378012B70B5054650D12A4B1A
:10235000446D98421BD1294B5A6B42F080025A635C
:102360005A6D42F080025A655A6D5A6942F08002F5
:102370005A615A6922F080025A610E2143205B693A
:1023800000F0D8FB1E4BE3601E4BC4F8003800235E
:10239000C4F8003EC02323606E6D4FF40413A363A2
:1023A0003369002BFCDA012333610C20FFF780FA3C
:1023B0003369DB07FCD41220FFF77AFA3369002B6C
:1023C000FCDA0026A6602846FFF734FF6B68C4F8E5
:1023D0001068DB68C4F81468C4F81C684BB90A4B71
:1023E000A3614FF0FF336361A36843F00103A3606F
:1023F00070BD064BF4E700BFAC2C00200038024053
:102400004014004003002002003C30C0083C30C0B3
:10241000F8B5446D054600212046FFF735FFA96D4C
:1024200000234FF001128F68C4F834384FF0006673
:10243000C4F81C284FF0FF3004EB431201339F42D5
:10244000C2F80069C2F8006BC2F80809C2F8080BAC
:10245000F2D20B686A6DEB65636210231361166933
:1024600016F01006FBD11220FFF722FAD4F800383C
:1024700023F4FE63C4F80038A36943F4402343F017
:102480001003A3610923C4F81038C4F814380A4BA8
:10249000EB604FF0C043C4F8103B084BC4F8003B5E
:1024A000C4F81069C4F80039EB6D03F1100243F46D
:1024B0008013EA65A362F8BD64360008408000100E
:1024C000426D90F84E10D2F8003823F4FE6343EAD0
:1024D0000113C2F8003870472DE9F0410EB200EB4D
:1024E00086080D46D8F80C100F6807F00303022B7E
:1024F00050D0032B50D03D4A3D4F012B18BF1746FB
:10250000446D4FEA451E04EB0E030022C3F8102B66
:102510008A6905F1100C002A40D04A8A05F1580357
:102520005B013A43E2500123D4F81C2803FA0CF370
:102530001343A6444A69C4F81C380023CEF8103966
:1025400005F13F03002A39D00A8A898B92080129B4
:1025500088BF4A43C16D04EB8303561841EA024227
:10256000C66529465A602046FFF78EFED8F80C3023
:102570001B8A43EA85531F4305F148035B01E7507B
:102580000123D4F81C2803FA05F51543C4F81C5898
:10259000BDE8F081174FB3E7174FB1E704EB4613DF
:1025A000D3F8002B22F40042C3F8002BD4F81C28E7
:1025B000012303FA0CF322EA0303BAE704EB8303D3
:1025C0000E4A5A6004EB461629462046FFF75CFE89
:1025D000D6F8003923F40043C6F80039D4F81C3883
:1025E000012202FA05F523EA0505CFE70080001075
:1025F000008004100080081000800C10000400020D
:10260000826D1268C265FFF715BE00005831436D38
:1026100049015B5813F4004004D013F4001F14BFA9
:1026200001200220704700004831436D49015B588A
:1026300013F4004004D013F4001F14BF0120022043
:102640007047000000EB8101CB68196A0B681360CA
:102650004B6853607047000000EB810330B5DD68C4
:10266000AA691368D36019B9402B84BF4023136053
:102670006B8A1468426D1C44013CB4FBF3F4634361
:10268000033323F0030302EB411043EAC44343F056
:10269000C043C0F8103B2B6803F00303012B09B2C1
:1026A0000ED1D2F8083802EB411013F4807FD0F835
:1026B000003B14BF43F0805343F00053C0F8003B8D
:1026C00002EB4112D2F8003B43F00443C2F8003B56
:1026D00030BD00002DE9F041244D6E6D06EB401336
:1026E0000446D3F8087BC3F8087B38070AD5D6F828
:1026F0001438190706D505EB84032146DB68284604
:102700005B689847FA072FD5D6F81438DB072BD526
:1027100005EB8403D968CCB98B69488A5E68B6FB3F
:10272000F0F200FB12628AB91868DA6890420DD2A2
:10273000121A83E81400202383F311880B482146E2
:10274000FFF78AFF84F31188BDE8F081012303FAC3
:1027500004F26B8923EA02036B81CB6823B1214623
:102760000248BDE8F0411847BDE8F081AC2C0020DC
:1027700000EB810370B5DD68436D6C692668E66027
:102780004A0156BB1A444FF40020C2F810092A68C7
:1027900002F00302012A0AB20ED1D3F8080803EBB3
:1027A000421410F4807FD4F8000914BF40F0805028
:1027B00040F00050C4F8000903EB4212D2F80009BF
:1027C00040F00440C2F80009D3F83408012202FAAC
:1027D00001F10143C3F8341870BD19B9402E84BF0C
:1027E0004020206020682E8A841940F00050013C6F
:1027F0001A44B4FBF6F440EAC440C6E7F8B5044610
:102800001E48456D05EB4413D3F80869C3F8086901
:10281000F10717D5D5F81038DA0713D500EB840384
:10282000D9684B691F68DA68974218D2D21B002713
:102830001A605F60202383F311882146FFF798FF19
:1028400087F31188330617D5D5F834280123A34020
:10285000134211D02046BDE8F840FFF71FBD012309
:1028600003FA04F2038923EA020303818B68002B35
:10287000E8D021469847E5E7F8BD00BFAC2C002022
:1028800097482DE9F84F456D6E69AB691E4016F407
:10289000805F6E61044605D0FEF700FDBDE8F84F8D
:1028A000FFF780BC002E12DAD5F8003E8C489B075B
:1028B0001EBFD5F8003E23F00303C5F8003ED5F84F
:1028C000043823F00103C5F80438FEF715FD370579
:1028D00005D58348FFF7AEFC8148FEF7FDFCB00448
:1028E0000CD5D5F8083813F0060FEB6823F47053B5
:1028F0000CBF43F4105343F4A053EB60310704D5ED
:102900006368DB680BB176489847F2025AD4B30289
:102910000CD5D4F85480DFF8C8A100274FF0010986
:10292000A36D9B68F9B28B4280F08780F70619D5BA
:10293000616D0A6AC2F30A1702F00F0302F4F01283
:10294000B2F5802F00F0A180B2F5402F0AD104EB40
:10295000830301F58051DB68186A00231A469F4201
:1029600040F087803003D5F8184813D5E10302D52D
:102970000020FFF7AFFEA20302D50120FFF7AAFE59
:10298000630302D50220FFF7A5FE270302D503202B
:10299000FFF7A0FE750381D5E00702D50020FFF701
:1029A0002DFFA10702D50120FFF728FF620702D5FE
:1029B0000220FFF723FF23077FF570AF0320FFF707
:1029C0001DFF6BE7D4F85480DFF814A100274FF007
:1029D0000109A36D9B685FFA87FB5B4597D308EB02
:1029E0004B13D3F8002902F44022B2F5802F22D1F4
:1029F000D3F80029002A1EDAD3F8002942F09042C9
:102A0000C3F80029D3F80029002AFBDB5946606D82
:102A1000FFF73AFC228909FA0BF322EA0303238128
:102A200004EB8B03DB689B6813B15946504698470B
:102A30005846FFF733FC0137CBE708EB4112D2F8D9
:102A4000003B03F44023B3F5802F10D1D2F8003BB4
:102A5000002B0CDA628909FA01F322EA030363818D
:102A600004EB8103DB68DB680BB150469847013704
:102A700056E79C0708BF0A68072B98BF027003F14E
:102A800001039CBF120A013069E7023304EB8302A1
:102A900001F58051526890690268D0F808C040681A
:102AA000A2EB000E0022104697420AD104EB8304E9
:102AB00063689B699A683A449A605A6817445F60F1
:102AC00050E712F0030F08BF0868964588BF8CF8DE
:102AD000000002F1010284BF000A0CF1010CE3E7DF
:102AE000AC2C0020436D03EB4111D1F8003B43F4C3
:102AF0000013C1F8003B7047436D03EB4111D1F85F
:102B0000003943F40013C1F800397047436D03EBFB
:102B10004111D1F8003B23F40013C1F8003B70478A
:102B2000436D03EB4111D1F8003923F40013C1F8D0
:102B30000039704700F1604300F01F02400903F5BF
:102B4000614309018000C9B200F1604083F80013BD
:102B500000F5614001239340C0F880310360704765
:102B600030B5039C0172043304FB0325C361049B4D
:102B700003630021059B00604060C1604261026107
:102B80008561046242628162C162436330BD0000BC
:102B90000022416A41610161C2608262C2626FF0DB
:102BA0000101FEF7F7BE000003694269934203D1B9
:102BB000C2680AB100207047181D70470369196088
:102BC000C2680132C260C2691344826903619342E0
:102BD00024BF436A03610021FEF7D0BE38B5044626
:102BE0000D46E3683BB16269131D1268A36213448A
:102BF000E362002038BD237A33B929462046FEF728
:102C0000ADFE0028EDDA38BD6FF00100FBE70000F3
:102C1000C368C269013BC36043691344826943616D
:102C2000934224BF436A436100238362036B03B171
:102C30001847704770B52023044683F31188866ACD
:102C40003EB9FFF7CBFF054618B186F31188284639
:102C500070BDA36AE26A13F8015BA362934202D3D8
:102C60002046FFF7D5FF002383F31188EFE700002C
:102C70002DE9F84F04460E4690469946202787F3E3
:102C800011880025AA46D4F828B0BBF1000F09D15D
:102C900049462046FFF7A2FF20B18BF31188284652
:102CA000BDE8F88FA16AE36AA8EB050B5B1A9B45A8
:102CB00028BF9B46BBF1400F1BD9334601F14002B0
:102CC00051F8040B43F8040B9142F9D1A36A403345
:102CD0004036A3624035A26AE36A9A4202D3204694
:102CE000FFF796FF8AF311884545D8D287F31188FC
:102CF000C9E730465A46FDF7B5FFA36A5B445E4418
:102D0000A3625D44E7E7000010B5029C0172043342
:102D100003FB0421C36100238362C362039B03633B
:102D2000049B00604060C460426102618161046292
:102D30004262436310BD0000026AC260426A42619F
:102D4000026100228262C2626FF00101FEF722BEC0
:102D5000436902699A4203D1C2680AB100207047F0
:102D6000184650F8043B0B6070470000C368C26906
:102D70000133C3604369134482694361934224BFB2
:102D8000436A43610021FEF7F9BD000038B50446EF
:102D90000D46E3683BB123691A1DA262E269134440
:102DA000E362002038BD237A33B929462046FEF776
:102DB000D5FD0028EDDA38BD6FF00100FBE700001B
:102DC00003691960C268013AC260C269134482692A
:102DD0000361934224BF436A036100238362036B50
:102DE00003B118477047000070B5202304460E4613
:102DF00083F31188856A35B91146FFF7C7FF10B113
:102E000085F3118870BDA36A1E70A36AE26A01335C
:102E10009342A36204D3E16920460439FFF7D0FF4F
:102E2000002080F3118870BD2DE9F84F04460D464F
:102E300091469A464FF0200888F311880026B34641
:102E4000A76A4FB951462046FFF7A0FF20B187F38C
:102E500011883046BDE8F88FA06AE76AA9EB06033F
:102E60003F1A9F4228BF1F46402F1BD905F1400340
:102E700055F8042B40F8042B9D42F9D1A36A403346
:102E8000A3624036A26AE36A9A4204D3E16920460B
:102E90000439FFF795FF8BF311884E45D9D288F39B
:102EA0001188CDE729463A46FDF7DCFEA36A3B448C
:102EB0003D44A3623E44E5E7026943699A4203D177
:102EC000C3681BB9184670470023FBE7836A002BD1
:102ED000F8D0043B9B1AF5D01360C368013BC36074
:102EE000C3691A44836902619A4224BF436A036139
:102EF000002383620123E5E700F090B84FF08043A0
:102F0000002258631A610222DA6070474FF0804352
:102F10000022DA60704700004FF08043586370472A
:102F20004FF08043586A70474B6843608B688360FA
:102F3000CB68C3600B6943614B6903628B69436271
:102F40000B6803607047000008B5224B22481A69DD
:102F500040F2FF110A431A611A6922F4FF7222F04B
:102F600001021A611A691A6B0A431A631A6D0A433D
:102F70001A651A4A1B6D1146FFF7D6FF184802F171
:102F80001C01FFF7D1FF174802F13801FFF7CCFF12
:102F9000154802F15401FFF7C7FF144802F1700110
:102FA000FFF7C2FF124802F18C01FFF7BDFF114885
:102FB00002F1A801FFF7B8FF0F4802F1C401FFF7C3
:102FC000B3FF0E4802F1E001FFF7AEFFBDE8084095
:102FD00000F0AAB800380240000002409436000811
:102FE0000004024000080240000C024000100240B1
:102FF0000014024000180240001C02400020024061
:1030000008B500F007FAFEF731FCFFF785F8BDE8D8
:103010000840FEF75BBE000070470000104B1A6CC2
:1030200042F001021A641A6E42F001021A660D4A59
:103030001B6E936843F0010393604FF0804353226B
:103040009A624FF0FF32DA6200229A615A63DA60C4
:103050005A6001225A6108211A601C20FFF76ABDDC
:1030600000380240002004E04FF0804208B51369A8
:10307000D1680B40D9B2C9439B07116107D5202302
:1030800083F31188FEF712FC002383F3118808BD37
:1030900008B5FFF7E9FFBDE80840FFF783B8000077
:1030A0001F4B1A696FEAC2526FEAD2521A611A694B
:1030B000C2F308021A614FF0FF301A695A69586169
:1030C00000215A6959615A691A6A62F080521A627B
:1030D0001A6A02F080521A621A6A5A6A58625A6A66
:1030E00059625A6A1A6C42F080521A641A6E42F09F
:1030F00080521A661A6E0B4A106840F48070106095
:10310000186F00F44070B0F5007F1EBF4FF48030A0
:1031100018671967536823F40073536000F05AB9B5
:103120000038024000700040334B4FF080521A6468
:10313000324A4FF4404111601A6842F001021A60AD
:103140001A689207FCD59A6822F003029A602A4B0B
:1031500019469A6812F00C02FBD1186800F0F900C9
:1031600018609A601A6842F480321A600B689B03F8
:10317000FCD54B6F43F001034B671F4B5A6F900711
:10318000FCD51F4A5A601A6842F080721A601B4AC6
:1031900053685904FCD5184B1A689201FCD5194A9A
:1031A0009A60194B1A68194B9A42194B21D1194A46
:1031B0001168194A91421CD140F205121A60144A52
:1031C000136803F00F03052BFAD10B4B9A6842F0FA
:1031D00002029A609A6802F00C02082AFAD15A6C2C
:1031E00042F480425A645A6E42F480425A665B6EE0
:1031F000704740F20572E1E700380240007000407D
:103200000854400700948838002004E0116400202E
:10321000003C024000ED00E041C20F41084A08B501
:10322000536911680B4003F00103536123B1054A50
:1032300013680BB150689847BDE80840FEF7B2BF6D
:10324000003C0140242D0020084A08B5536911684C
:103250000B4003F00203536123B1054A93680BB19D
:10326000D0689847BDE80840FEF79CBF003C01408D
:10327000242D0020084A08B5536911680B4003F05B
:103280000403536123B1054A13690BB15069984790
:10329000BDE80840FEF786BF003C0140242D002019
:1032A000084A08B5536911680B4003F008035361DD
:1032B00023B1054A93690BB1D0699847BDE808402E
:1032C000FEF770BF003C0140242D0020084A08B5DD
:1032D000536911680B4003F01003536123B1054A91
:1032E000136A0BB1506A9847BDE80840FEF75ABF11
:1032F000003C0140242D0020174B10B55C691A6872
:10330000144004F478725A61A30604D5134A936AF0
:103310000BB1D06A9847600604D5104A136B0BB105
:10332000506B9847210604D50C4A936B0BB1D06BB8
:103330009847E20504D5094A136C0BB1506C9847C5
:10334000A30504D5054A936C0BB1D06C9847BDE832
:103350001040FEF727BF00BF003C0140242D002095
:103360001A4B10B55C691A68144004F47C425A6127
:10337000620504D5164A136D0BB1506D98472305AD
:1033800004D5134A936D0BB1D06D9847E00404D572
:103390000F4A136E0BB1506E9847A10404D50C4A26
:1033A000936E0BB1D06E9847620404D5084A136F30
:1033B0000BB1506F9847230404D5054A936F0BB1A6
:1033C000D06F9847BDE81040FEF7ECBE003C0140CE
:1033D000242D0020062108B50846FFF7ABFB062187
:1033E0000720FFF7A7FB06210820FFF7A3FB062114
:1033F0000920FFF79FFB06210A20FFF79BFB062110
:103400001720FFF797FB06212820BDE80840FFF7AB
:1034100091BB000008B5FFF743FE00F00BF8FDF785
:10342000CFFEFDF7A3FDFFF7F7FDBDE80840FFF76E
:1034300063BD0000002304491A465A50C8180833D7
:10344000802B4260F9D17047242D0020034611F8EB
:10345000012B03F8012B002AF9D170471210121327
:103460001211000053544D3332463F3F3F000000DD
:1034700000000000643400083F0000001304000056
:10348000A03400083F00000019040000AA3400081E
:103490003F00000021040000B43400083F00000099
:1034A00053544D3332463430780053544D33324602
:1034B0003432780053544D33324634343658580041
:1034C00000000000E50E0008D10E00080D0F0008F6
:1034D000F90E0008050F0008F10E0008DD0E0008C7
:1034E000C90E0008690F000800000000010000007C
:1034F000000000006D61696E0000000014350008D6
:10350000D823002050250020010000006918000881
:103510000000000069646C6500000000020000000B
:10352000000000001111000879110008400040005F
:10353000E8290020F8290020020000000000000017
:103540000300000000000000BD11000800000000A2
:1035500010000000082A0020000000000100000008
:1035600000000000AC2C00200101020041726475D3
:1035700050696C6F740025424F415244252D424CD6
:10358000002553455249414C250000006D1C0008A0
:10359000851B00081D1C0008011C000843000000DA
:1035A000A435000809024300020100C032090400EA
:1035B00000010202010005240010010524010001A0
:1035C000042402020524060001070582030800FF07
:1035D00009040100020A0000000705010240000082
:1035E000070581024000000012000000F0350008CD
:1035F00012011001020000400912415700020102AD
:10360000030100000403090425424F4152442500F0
:103610004D616D62614634303555532D493243005A
:1036200030313233343536373839414243444546F8
:1036300000000000004000000040000000400000CA
:103640000040000000000100000002000000020035
:103650000000020000000200000002000000020062
:1036600000000200000000000D130008ED15000826
:1036700099160008400040000C2D00200C2D002061
:10368000010000001C2D002080000000400100000F
:10369000030000000000800200000000AAAAAAAAFD
:1036A00000000000FFFF00000000000000A00A0072
:1036B0000000000000000000AAAAAAAA0000000062
:1036C000FFFF0000000000000000000000000050AC
:1036D00000000000AAAAAAAA00000000FF3F000004
:1036E00000000000000000000000000000000000DA
:1036F000AAAAAAAA00000000FFFF00000000000024
:10370000000000000000000000000000AAAAAAAA11
:1037100000000000FFFF00000000000000000000AB
:103720000000000000000000AAAAAAAA00000000F1
:10373000FFFF00000000000000000000000000008B
:1037400000000000AAAAAAAA00000000FFFF0000D3
:103750000000000000000000000000000000000069
:103760000A0000000000000003000000000000004C
:103770000000000000000000000000000000000049
:103780000000000000000000000000000000000039
:103790000E0400000000000000400F00FF00960033
:1037A000000000080096000000000800040000006F
:1037B00004360008000000000000000000000000C7
:1037C000000000000000000000000000FFFFFFFFFD
:1037D000FFFFFFFFFFFFFFFFFFFFFFFFFFFFFFFFF9
:1037E000FFFFFFFFFFFFFFFFFFFFFFFFFFFFFFFFE9
:1037F000FFFFFFFFFFFFFFFFFFFFFFFFFFFFFFFFD9
:10380000FFFFFFFFFFFFFFFFFFFFFFFFFFFFFFFFC8
:10C0000000060020B5D2000895EF0908F1EE0908F6
:10C010005DEF0908F1EE090829EF0908B7D2000819
:10C02000B7D20008B7D20008B7D20008E1180C0850
:10C03000B7D20008B7D20008B7D20008B7D20008BC
:10C04000B7D20008B7D20008B7D20008B7D20008AC
:10C05000B7D20008B7D20008FD2A0C08252B0C081F
:10C060004D2B0C08752B0C089D2B0C0899D40B0834
:10C07000C1D40B08EDD40B0819D50B0845D50B0816
:10C080006DD50B0899D50B081DD40B08B7D2000845
:10C09000B7D20008B7D20008B7D20008C52B0C08E9
:10C0A000112D0C08152D0C08292D0C082D2D0C0810
:10C0B000B7D20008312D0C08452D0C0825DB0B08E4
:10C0C000CDDC0B08B7D20008B7D20008B7D2000801
:10C0D000B7D20008992C0C08AD2C0C08C12C0C0808
:10C0E000292C0C08B7D20008B7D20008B7D2000834
:10C0F000B7D20008B7D20008B7D20008C5D50B08E0
:10C10000B7D20008B7D20008592D0C08B7D20008E2
:10C11000D52C0C08E92C0C08B7D20008B7D20008BF
:10C12000F1D50B0819D60B0845D60B0871D60B08AC
:10C130009DD60B08B7D20008B7D20008B7D20008C6
:10C14000B7D20008B7D20008B7D200080D200C08FB
:10C15000C5D60B08F1D60B081DD70B08FD2C0C0813
:10C16000B7D20008B7D20008B7D20008B7D200088B
:10C17000B7D20008B7D20008B7D20008B7D200087B
:10C18000B7D20008B7D20008B7D20008B7D200086B
:10C19000B7D20008B7D20008B7D20008B7D200085B
:10C1A000B7D20008B7D20008B7D20008B7D200084B
:10C1B000B7D20008B7D20008B7D20008B7D200083B
:10C1C000B7D20008B7D20008B7D20008B7D200082B
:10C1D000B7D20008B7D20008B7D20008B7D200081B
:10C1E00069F500087D260108D960010871C40108BD
:10C1F0009D0D020865950208191404089DD20508D2
:10C20000A5D80508BD220608A1740608657C0608A5
:10C210009D7F06080DE5060845060708C5DA0708EC
:10C22000894D080849E80908E1F40A08754F0B0828
:10C2300045760B0869800B08C5AF0B08EDB50B08F8
:10C2400081F0004102E000BF83F0004330B54FEAC7
:10C2500041044FEA430594EA050F08BF90EA020F34
:10C260001FBF54EA000C55EA020C7FEA645C7FEAC7
:10C27000655C00F0E2804FEA5454D4EB5555B8BFEA
:10C280006D420CDD2C4480EA020281EA030382EA5B
:10C29000000083EA010180EA020281EA0303362DED
:10C2A00088BF30BD11F0004F4FEA01314FF4801CC0
:10C2B0004CEA113102D0404261EB410113F0004FD2
:10C2C0004FEA03334CEA133302D0524263EB430389
:10C2D00094EA050F00F0A780A4F10104D5F1200E27
:10C2E0000DDB02FA0EFC22FA05F2801841F1000182
:10C2F00003FA0EF2801843FA05F359410EE0A5F156
:10C3000020050EF1200E012A03FA0EFC28BF4CF086
:10C31000020C43FA05F3C01851EBE37101F000453C
:10C3200007D54FF0000EDCF1000C7EEB00006EEB49
:10C330000101B1F5801F1BD3B1F5001F0CD34908D3
:10C340005FEA30004FEA3C0C04F101044FEA44522A
:10C3500012F5800F80F09A80BCF1004F08BF5FEAB1
:10C36000500C50F1000041EB045141EA050130BD91
:10C370005FEA4C0C404141EB0101013C28BFB1F5A3
:10C38000801FE9D291F0000F04BF01460020B1FAEE
:10C3900081F308BF2033A3F10B03B3F120020CDAC1
:10C3A0000C3208DD02F1140CC2F10C0201FA0CF09F
:10C3B00021FA02F10CE002F11402D8BFC2F1200C04
:10C3C00001FA02F120FA0CFCDCBF41EA0C019040BA
:10C3D000E41AA2BF01EB0451294330BD6FEA040403
:10C3E0001F3C1CDA0C340EDC04F11404C4F12002EE
:10C3F00020FA04F001FA02F340EA030021FA04F300
:10C4000045EA030130BDC4F10C04C4F1200220FA56
:10C4100002F001FA04F340EA0300294630BD21FA94
:10C4200004F0294630BD94F0000F83F4801306BF5A
:10C4300081F480110134013D4EE77FEA645C18BF4E
:10C440007FEA655C29D094EA050F08BF90EA020FE5
:10C4500005D054EA000C04BF1946104630BD91EADD
:10C46000030F1EBF0021002030BD5FEA545C05D1E0
:10C470004000494128BF41F0004130BD14F580041F
:10C480003CBF01F5801130BD01F0004545F0FE4193
:10C4900041F470014FF0000030BD7FEA645C1ABFC8
:10C4A000194610467FEA655C1CBF0B46024650EAFF
:10C4B000013406BF52EA033591EA030F41F400212B
:10C4C00030BD00BF90F0000F04BF0021704730B5B1
:10C4D0004FF4806404F132044FF000054FF0000186
:10C4E00050E700BF90F0000F04BF0021704730B547
:10C4F0004FF4806404F1320410F0004548BF40421C
:10C500004FF000013EE700BF42004FEAE2014FEA70
:10C5100031014FEA02701FBF12F07F4393F07F4F4B
:10C5200081F06051704732F07F4208BF704793F04E
:10C530007F4F04BF41F40021704730B54FF4607461
:10C5400001F0004521F000411CE700BF50EA010264
:10C5500008BF704730B54FF000050AE050EA01020D
:10C5600008BF704730B511F0004502D5404261EB7D
:10C5700041014FF4806404F132045FEA915C3FF4BE
:10C58000D8AE4FF003025FEADC0C18BF03325FEA5B
:10C59000DC0C18BF033202EBDC02C2F1200300FA0C
:10C5A00003FC20FA02F001FA03FE40EA0E0021FA31
:10C5B00002F11444BDE600BF70B54FF0FF0C4CF41F
:10C5C000E06C1CEA11541DBF1CEA135594EA0C0FD1
:10C5D00095EA0C0F00F0DEF82C4481EA030621EA0C
:10C5E0004C5123EA4C5350EA013518BF52EA033547
:10C5F00041F4801143F4801338D0A0FB02CE4FF0F9
:10C600000005E1FB02E506F00042E0FB03E54FF028
:10C610000006E1FB03569CF0000F18BF4EF0010E20
:10C62000A4F1FF04B6F5007F64F5407404D25FEA1C
:10C630004E0E6D4146EB060642EAC62141EA5551CF
:10C640004FEAC52040EA5E504FEACE2EB4F1FD0C11
:10C6500088BFBCF5E06F1ED8BEF1004F08BF5FEA8F
:10C66000500E50F1000041EB045170BD06F0004641
:10C6700046EA010140EA020081EA0301B4EB5C04EE
:10C68000C2BFD4EB0C0541EA045170BD41F48011E6
:10C690004FF0000E013C00F3AB8014F1360FDEBF0B
:10C6A000002001F0004170BDC4F10004203C35DAE7
:10C6B0000C341BDC04F11404C4F1200500FA05F36A
:10C6C00020FA04F001FA05F240EA020001F000420B
:10C6D00021F0004110EBD37021FA04F642EB060181
:10C6E0005EEA430E08BF20EAD37070BDC4F10C04AB
:10C6F000C4F1200500FA04F320FA05F001FA04F26F
:10C7000040EA020001F0004110EBD37041F100015A
:10C710005EEA430E08BF20EAD37070BDC4F1200565
:10C7200000FA05F24EEA020E20FA04F301FA05F2CD
:10C7300043EA020321FA04F001F0004121FA04F275
:10C7400020EA020000EBD3705EEA430E08BF20EA45
:10C75000D37070BD94F0000F0FD101F0004640007F
:10C7600041EB010111F4801F08BF013CF7D041EA01
:10C77000060195F0000F18BF704703F00046520005
:10C7800043EB030313F4801F08BF013DF7D043EAD6
:10C790000603704794EA0C0F0CEA135518BF95EA8C
:10C7A0000C0F0CD050EA410618BF52EA4306D1D113
:10C7B00081EA030101F000414FF0000070BD50EA32
:10C7C000410606BF1046194652EA430619D094EABC
:10C7D0000C0F02D150EA013613D195EA0C0F05D1A6
:10C7E00052EA03361CBF104619460AD181EA0301FA
:10C7F00001F0004141F0FE4141F470014FF00000B2
:10C8000070BD41F0FE4141F4780170BD70B54FF04C
:10C81000FF0C4CF4E06C1CEA11541DBF1CEA1355CC
:10C8200094EA0C0F95EA0C0F00F0A7F8A4EB0504AE
:10C8300081EA030E52EA03354FEA013100F08880A5
:10C840004FEA03334FF0805545EA131343EA12636E
:10C850004FEA022245EA111545EA10654FEA002623
:10C860000EF000419D4208BF964244F1FD0404F5DC
:10C87000407402D25B084FEA3202B61A65EB030538
:10C880005B084FEA32024FF480104FF4002CB6EBF5
:10C89000020E75EB030E22BFB61A754640EA0C0075
:10C8A0005B084FEA3202B6EB020E75EB030E22BFB5
:10C8B000B61A754640EA5C005B084FEA3202B6EBF6
:10C8C000020E75EB030E22BFB61A754640EA9C00B5
:10C8D0005B084FEA3202B6EB020E75EB030E22BF85
:10C8E000B61A754640EADC0055EA060E18D04FEA43
:10C8F000051545EA16754FEA06164FEAC30343EAE3
:10C9000052734FEAC2025FEA1C1CC0D111F4801FAF
:10C910000BD141EA00014FF000004FF0004CB6E7A8
:10C9200011F4801F04BF01430020B4F1FD0C88BF47
:10C93000BCF5E06F3FF6AFAEB5EB030C04BFB6EB52
:10C94000020C5FEA500C50F1000041EB045170BD45
:10C950000EF0004E4EEA113114EB5C04C2BFD4EB72
:10C960000C0541EA045170BD41F480114FF0000EF6
:10C97000013C90E645EA060E8DE60CEA135594EA72
:10C980000C0F08BF95EA0C0F3FF43BAF94EA0C0F75
:10C990000AD150EA01347FF434AF95EA0C0F7FF4EA
:10C9A00025AF104619462CE795EA0C0F06D152EA3E
:10C9B00003353FF4FDAE1046194622E750EA410622
:10C9C00018BF52EA43067FF4C5AE50EA41047FF433
:10C9D0000DAF52EA43057FF4EBAE12E74FF0FF3C98
:10C9E00006E000BF4FF0010C02E000BF4FF0010C69
:10C9F0004DF804CD4FEA410C7FEA6C5C4FEA430CE2
:10CA000018BF7FEA6C5C1BD001B050EA410C0CBF30
:10CA100052EA430C91EA030F02BF90EA020F002092
:10CA2000704710F1000F91EA030F58BF994208BFF9
:10CA300090422CBFD8176FEAE37040F001007047B6
:10CA40004FEA410C7FEA6C5C02D150EA013C07D10D
:10CA50004FEA430C7FEA6C5CD6D152EA033CD3D058
:10CA60005DF8040B704700BF8446104662468C4652
:10CA70001946634600E000BF01B5FFF7B7FF002885
:10CA800048BF10F1000F01BD4DF808EDFFF7F4FFAE
:10CA90000CBF012000205DF808FB00BF4DF808ED39
:10CAA000FFF7EAFF34BF012000205DF808FB00BF5C
:10CAB0004DF808EDFFF7E0FF94BF012000205DF87E
:10CAC00008FB00BF4DF808EDFFF7CEFF94BF012033
:10CAD00000205DF808FB00BF4DF808EDFFF7C4FF2C
:10CAE00034BF012000205DF808FB00BF4FEA410C75
:10CAF0007FEA6C5C02D150EA013C0AD14FEA430C58
:10CB00007FEA6C5C02D152EA033C02D14FF0000094
:10CB100070474FF0010070474FEA410212F50012D2
:10CB200015D211D56FF47873B3EB625212D94FEA74
:10CB3000C12343F0004343EA505311F0004F23FA5E
:10CB400002F018BF404270474FF00000704750EAB3
:10CB5000013005D111F0004008BF6FF00040704770
:10CB60004FF00000704700BF4A0011D212F50012CA
:10CB700011D20DD56FF47873B3EB62520ED44FEA35
:10CB8000C12343F0004343EA505323FA02F07047B5
:10CB90004FF00000704750EA013002D14FF0FF30F3
:10CBA00070474FF0000070474FEA4102B2F1E04396
:10CBB00024BFB3F5001CDCF1FE5C0DD901F0004C84
:10CBC0004FEAC0024CEA5070B2F1004F40EB8300D4
:10CBD00008BF20F00100704711F0804F21D113F100
:10CBE0003872BCBF01F00040704741F480114FEA39
:10CBF0005252C2F11802C2F1200C10FA0CF320FAC2
:10CC000002F018BF40F001004FEAC1234FEAD323DE
:10CC100003FA0CFC40EA0C0023FA02F34FEA430348
:10CC2000CCE77FEA625307D150EA01331EBF4FF0D1
:10CC3000FE4040F44000704701F0004040F0FE40EC
:10CC400040F40000704700BF80F0004002E000BFE9
:10CC500081F0004142001FBF5FEA410392EA030FE7
:10CC60007FEA226C7FEA236C6AD04FEA1262D2EB31
:10CC70001363C1BFD218414048404140B8BF5B4236
:10CC8000192B88BF704710F0004F40F4000020F0CF
:10CC90007F4018BF404211F0004F41F4000121F0E5
:10CCA0007F4118BF494292EA030F3FD0A2F101022F
:10CCB00041FA03FC10EB0C00C3F1200301FA03F16D
:10CCC00000F0004302D5494260EB4000B0F5000F90
:10CCD00013D3B0F1807F06D340084FEA310102F14F
:10CCE0000102FE2A51D2B1F1004F40EBC25008BF01
:10CCF00020F0010040EA03007047490040EB0000CB
:10CD0000013A28BFB0F5000FEDD2B0FA80FCACF1CB
:10CD1000080CB2EB0C0200FA0CF0AABF00EBC250F8
:10CD200052421843BCBFD0401843704792F0000FE6
:10CD300081F4000106BF80F400000132013BB5E739
:10CD40004FEA41037FEA226C18BF7FEA236C21D0AF
:10CD500092EA030F04D092F0000F08BF0846704714
:10CD600090EA010F1CBF0020704712F07F4F04D1E2
:10CD7000400028BF40F00040704712F100723CBFF5
:10CD800000F50000704700F0004343F0FE4040F41F
:10CD9000000070477FEA226216BF08467FEA2363DD
:10CDA0000146420206BF5FEA412390EA010F40F4C8
:10CDB000800070474FF0000304E000BF10F0004314
:10CDC00048BF40425FEA000C08BF704743F09643FB
:10CDD00001464FF000001CE050EA010208BF704716
:10CDE0004FF000030AE000BF50EA010208BF70479D
:10CDF00011F0004302D5404261EB41015FEA010CB2
:10CE000002BF84460146002043F0B64308BFA3F1A9
:10CE10008053A3F50003BCFA8CF2083AA3EBC2538B
:10CE200010DB01FA02FC634400FA02FCC2F12002AA
:10CE3000BCF1004F20FA02F243EB020008BF20F0E1
:10CE40000100704702F1200201FA02FCC2F1200247
:10CE500050EA4C0021FA02F243EB020008BF20EA3C
:10CE6000DC7070477BB972B90029BEBF00204FF05B
:10CE7000004106E008BF00281CBF6FF000414FF0E2
:10CE8000FF3000F015BAADF1080C6DE904CE0029B1
:10CE900009DB002B1ADB00F0A3F8DDF804E0DDE984
:10CEA000022304B07047404261EB4101002B1BDBC1
:10CEB00000F096F8DDF804E0DDE9022304B040421A
:10CEC00061EB4101524263EB43037047524263EB13
:10CED000430300F085F8DDF804E0DDE9022304B047
:10CEE000404261EB41017047524263EB430300F063
:10CEF00077F8DDF804E0DDE9022304B0524263EB89
:10CF00004303704753B94AB9002908BF00281CBF22
:10CF10004FF0FF314FF0FF3000F0CAB9ADF1080C0F
:10CF20006DE904CE00F05CF8DDF804E0DDE90223F1
:10CF300004B0704730B1012390FAA0F0B0FA80F04D
:10CF40001844704708460029FBD02123F4E700BFAE
:10CF5000430803F05533C01A830803F0333300F05D
:10CF60003330184400EB101000F00F3000EB0020BD
:10CF700000EB0040000E704707EE900AF5EEC07A15
:10CF8000F1EE10FA01D400F00BB8F1EE677A08B5B3
:10CF900017EE900A00F004F8404261EB410108BD31
:10CFA000D0B5FFF7B1FA0C4B002206460F46FFF74B
:10CFB00003FBFFF7D9FD0446FFF784FA074B002275
:10CFC000FFF7FAFA02460B4630463946FFF73CF9BE
:10CFD000FFF7CAFD2146D0BD0000F03D0000F04142
:10CFE0002DE9F047089D04468E46002B4DD18A421C
:10CFF000944669D9B2FA82F252B101FA02F3C2F14F
:10D00000200120FA01F10CFA02FC41EA030E9440DF
:10D010004FEA1C48210CBEFBF8F61FFA8CF708FB00
:10D0200016E341EA034306FB07F199420AD91CEBD8
:10D03000030306F1FF3080F01F81994240F21C810A
:10D04000023E63445B1AA4B2B3FBF8F008FB103352
:10D0500044EA034400FB07F7A7420AD91CEB040487
:10D0600000F1FF3380F00A81A74240F20781644457
:10D07000023840EA0640E41B00261DB1D4400023DC
:10D08000C5E900433146BDE8F0878B4209D9002D40
:10D0900000F0EF800026C5E9000130463146BDE8CA
:10D0A000F087B3FA83F6002E4AD18B4202D3824234
:10D0B00000F2F980841A61EB030301209E46002DE3
:10D0C000E0D0C5E9004EDDE702B9FFDEB2FA82F238
:10D0D000002A40F09280A1EB0C014FEA1C471FFA96
:10D0E0008CFE0126200CB1FBF7F307FB131140EA7D
:10D0F00001410EFB03F0884208D91CEB010103F14A
:10D10000FF3802D2884200F2CB804346091AA4B20B
:10D11000B1FBF7F007FB101144EA01440EFB00FEDF
:10D12000A64508D91CEB040400F1FF3102D2A64544
:10D1300000F2BB800846A4EB0E0440EA03409CE7E3
:10D14000C6F12007B34022FA07FC4CEA030C20FA90
:10D1500007F401FA06F31C43F9404FEA1C4900FAB0
:10D1600006F3B1FBF9F8200C1FFA8CFE09FB18112D
:10D1700040EA014108FB0EF0884202FA06F20BD9A0
:10D180001CEB010108F1FF3A80F08880884240F2F0
:10D190008580A8F102086144091AA4B2B1FBF9F034
:10D1A00009FB101144EA014100FB0EFE8E4508D92F
:10D1B0001CEB010100F1FF346CD28E456AD90238B4
:10D1C000614440EA0840A0FB0294A1EB0E01A14299
:10D1D000C846A64656D353D05DB1B3EB080261EB07
:10D1E0000E0101FA07F722FA06F3F1401F43C5E9E1
:10D1F000007100263146BDE8F087C2F12003D84017
:10D200000CFA02FC21FA03F3914001434FEA1C4758
:10D210001FFA8CFEB3FBF7F007FB10360B0C43EA4A
:10D22000064300FB0EF69E4204FA02F408D91CEBFA
:10D23000030300F1FF382FD29E422DD902386344F8
:10D240009B1B89B2B3FBF7F607FB163341EA034198
:10D2500006FB0EF38B4208D91CEB010106F1FF38E7
:10D2600016D28B4214D9023E6144C91A46EA0046DE
:10D2700038E72E46284605E70646E3E61846F8E670
:10D280004B45A9D2B9EB020864EB0C0E0138A3E7B9
:10D290004646EAE7204694E74046D1E7D0467BE79A
:10D2A000023B614432E7304609E76444023842E712
:10D2B000704700BF02E000F000F8FEE772B63748A2
:10D2C00080F30888364880F3098836483649086074
:10D2D00040F20000CCF200004EF63471CEF20001B4
:10D2E0000860BFF34F8FBFF36F8F40F20000C0F2B2
:10D2F000F0004EF68851CEF200010860BFF34F8F68
:10D30000BFF36F8F4FF00000E1EE100A4EF63C7154
:10D31000CEF200010860062080F31488BFF36F8FFF
:10D32000B4F03CFBB5F086FA4FF055301F491B4A6C
:10D3300091423CBF41F8040BFAE71D49184A91425B
:10D340003CBF41F8040BFAE71A491B4A1B4B9A42AF
:10D350003EBF51F8040B42F8040BF8E700201849CF
:10D36000184A91423CBF41F8040BFAE7B4F01AFBAB
:10D37000B5F0B4FA144C154DAC4203DA54F8041B62
:10D380008847F9E702F0E0F8114C124DAC4203DA9D
:10D3900054F8041B8847F9E7B4F002BB00060020EC
:10D3A0000022002000C0000808ED00E0000000207E
:10D3B00000060020A0E10E0800220020742C0020AE
:10D3C000782C0020584C0120E0C1000840C2000821
:10D3D00040C2000840C200082DE9F04F2DED108A30
:10D3E000C1F80CD0C3689D46BDEC108ABDE8F08F33
:10D3F000002383F311882846A0470020B3F050FA99
:10D40000FEE7B3F0ADF800DFFEE7000001F0FF013A
:10D41000102A2BDB10F0070F08D010F8013B013A5F
:10D420008B422DD010F0070F42B3F6D1F0B441EA91
:10D43000012141EA014122F007047FF000070023A7
:10D44000F0E80256083C85EA010586EA010685FAFD
:10D4500047F5A3FA87F586FA47F6A5FA87F68EB957
:10D46000EED1F0BC01F0FF0102F0070232B110F87A
:10D47000013B013A83EA010313B1F8D10020704760
:10D4800001387047002D06BF35460338073815F0C0
:10D49000010F07D1013015F4807F02BF013015F470
:10D4A000C03F0130F0BC0138704700BF10F8012BBD
:10D4B00011F8013B012A28BF9A42F7D0D01A7047D1
:10D4C000034613F8012B002AFBD1181A01387047C4
:10D4D00038B50022002304460D46FFF7DFFA28B9CD
:10D4E00020462946BDE8384000F00AB8204605F13C
:10D4F000004100F005F8404261EB410138BD00BF3A
:10D50000D0B50C4B002206460F46FFF755F8FFF743
:10D510002BFB0446FEF7D6FF074B0022FFF74CF823
:10D5200002460B4630463946FEF78EFEFFF71CFBDF
:10D530002146D0BD0000F03D0000F041036800220C
:10D540001B6818477FB503914021054680F058FAC3
:10D55000039A18B90124204604B070BD134E0392FB
:10D5600096F9E632002BF5D061F006FA437A039A79
:10D5700053B961F001FA847A039A2CB90C4B40211B
:10D58000284680F045FAE6E7D6F8DC3CB6F9E81222
:10D59000B3F906309942DDDD064B00934021064B7E
:10D5A000284680F035FA0024D5E700BF804C0020E3
:10D5B000509F0C086F9F0C085D9F0C08F0B50D463E
:10D5C0009DB02021044680F01BFA002800F09D80C9
:10D5D0004F4E96F9E632ABB1D6F8DC2CB6F9E8320C
:10D5E000B2F90A1003F10A02914203DD40F28D32D2
:10D5F000934207DC474B2A462021204680F008FA58
:10D60000002080E096F9D532022B05D1424B2A4604
:10D610002021204680F0FCF9B6F8A832A3F57A73F1
:10D620009BB241F6583293420DD83C4F96EDC57AE5
:10D63000D7F81C3DD3ED097AB4EEE77AF1EE10FA93
:10D6400003DD374BD7E7374BD5E796EDC67AD3EDF9
:10D650000B7AB4EEE77AF1EE10FAF2DCB6F9E232C8
:10D66000002B01DC304BC6E796F874230D2A06D850
:10D670000123934013F4215F01D02C4BBBE72C48CE
:10D6800010F0CCF9012806D1D7F8280D87F00EFA52
:10D6900098B101281AD00021602204A80391B8F0A3
:10D6A00041F92449D7F8240D642303AA86F020FE0B
:10D6B00000BB03AB0093204B02E0204B0093204BB8
:10D6C0002A462021204680F0A3F999E796F8F03CFD
:10D6D00073B11C48192150F059FA48B11948D6F8CD
:10D6E000C062192150F078FA8642D4DD164BE5E786
:10D6F000164BE3E71649D7F81C0D642303AA83F001
:10D70000B7FC0028D5D01DB0F0BD0120FBE700BF5D
:10D71000804C0020789F0C088B9F0C08806C0020A8
:10D72000C39F0C08B39F0C08DD9F0C08F29F0C08E8
:10D73000588200206CA00C0870A00C0837A00C08C0
:10D7400012A00C08C039002056A00C0847A00C08F5
:10D7500082A00C0807B5044888F000FD00F0010025
:10D7600003B05DF804FB00BF807900202DE9F04391
:10D77000DFF844910446D9F8EC000368A5B01B69B2
:10D780000D469847804615F069FC00210746602247
:10D790000CA80B91B8F0C6F864230BAA4146384692
:10D7A00014F050FF064648B93A4A0BAB29462046CA
:10D7B00080F050FB304625B0BDE8F083A9F56B60E2
:10D7C0006EF0E2FBB8F1000F03D194F91E30012B8B
:10D7D0000AD1314812F02CFC80B9304A2946204643
:10D7E00080F038FB0026E5E710F0060FE2D0A9F53F
:10D7F000405012F01DFC08B9294AEFE703A938464A
:10D8000014F052FD28B19DF80D305B0601D5254A74
:10D81000E4E7DFF8A880D8EDC17AF5EEC07AF1EE42
:10D8200010FA4FF00003C5DD089309930A930DF138
:10D83000200907AB019305AA06AB04A9CDF8009017
:10D84000384615F013F9484630F0BAFDD8EDC17AE4
:10D85000B4EEE70AF1EE10FA01DB134ABEE79DEDE4
:10D86000057AF4EEC77AF1EE10FA01D80F4AB5E75F
:10D870009DED047AF4EEC77AF1EE10FA01D80C4A65
:10D88000ACE79DED067AF4EEC77AF1EE10FA91D886
:10D89000084AA3E788A00C08802C002091A00C085F
:10D8A000A8A00C08CEA00C08DCA00C08F1A00C0865
:10D8B00007A10C081DA10C08805C0020804C0020F2
:10D8C00008B5064B93F805319B0704D5044A80F050
:10D8D000C1FA002008BD0120FCE700BF805C0020E9
:10D8E00034A10C0870B50C4C0546D4F8EC00036864
:10D8F0005B690E46984710B10124204670BDA4F51F
:10D90000405012F0A7FB04460028F5D1034A3146E7
:10D91000284680F09FFAF0E7805C002044A10C08C4
:10D920002DE9F046464ED6F8103193F8CB509BB017
:10D9300081468A4665B9434B1B68986A03685B6BEE
:10D940009847044640B9404A5146484680F082FA1A
:10D9500028461BB0BDE8F08661F00EF8202162F089
:10D9600081F858B161F008F81F2162F07BF888B3A4
:10D97000364A5146484680F06DFA002496F8E23067
:10D9800003F01403142B05D1314A5146484680F068
:10D9900061FA00245146484681F02AF90021884264
:10D9A0004FF0600202A808BF0C460191B7F0BAFF21
:10D9B000D6F81001036801AA1B6864219847054640
:10D9C00080B9244A01AB5146484680F043FA2C46C0
:10D9D0002546BDE760F0D0FFA52162F043F800289E
:10D9E000C6D1CBE7002CF3D0D9F808303BB9D9F831
:10D9F000003051465B6B484698470446E8E751467D
:10DA00004846FFF7DBFD514607464846FFF758FFFB
:10DA10003840C4B251464846FFF794FD5146044091
:10DA20004846FFF75FFF51460440484680F03AFA07
:10DA300051460440484681F0F3F80440C8E700BF6F
:10DA4000805C0020E084002058A10C086FA10C0825
:10DA500089A10C08A1A10C0808B5FFF761FF054AD0
:10DA600092F8E01060F3041182F8E010024A90711D
:10DA700008BD00BF805C0020BD860020F7B50546CC
:10DA80000F467FF0F9FF044678B1022128467FF067
:10DA9000B7FF064648B1154888F060FBC205C0F3E1
:10DAA0000723C0F3002403D53446204603B0F0BD5D
:10DAB0009B07F9D50D4888F05FFB0D4B03F6CC436F
:10DAC000D3ED007AF8EEE77A30EE670ADFED097AF7
:10DAD000B0EEC00AB4EEE70AF1EE10FAE4DD064B50
:10DAE0003A46022128467FF093FFDEE78079002046
:10DAF000806C00200000C842ACA10C08F8B50446B8
:10DB00000F4680F06FFA1021054620467FF078FF1F
:10DB100058B12046FFF71EFE064630B9044B3A4680
:10DB2000102120467FF074FF35462846F8BD00BF1F
:10DB3000C0A10C0870B505460E467FF005FF0446EF
:10DB400078B1802128467FF05BFF50B1074B93F8F6
:10DB5000AD3643B1064B3246802128467FF058FF50
:10DB60000024204670BD0446FBE700BF805C002017
:10DB7000D4A10C0838B50D4D0446D5F8280D86F013
:10DB800095FF012810D0D5F8280D86F08FFF0228C8
:10DB900004D02046BDE838407FF0D8BE04480FF0DE
:10DBA0003DFF0128F5D138BD0020FCE7806C002046
:10DBB00058820020F0B5134C04F5005385B0D3F81B
:10DBC000D42C0092D3F8D82C0192D3F8DC2C0292FA
:10DBD000D3F8E03C03936A4606460F4680F0BAFF4E
:10DBE0003946054630467FF06DFF04F54054284025
:10DBF00094F8E03060F3C303C3F3C00084F8E0306E
:10DC000005B0F0BD802C00202DE9F84306462748DA
:10DC1000DFF8A890DFF8A8800F466EF0B5F904464B
:10DC2000D9F8EC0003681B699847054630B914F031
:10DC3000060F03D1D9F82031022B09D139463046DD
:10DC400080F02CF8054618B9002488F807400AE04F
:10DC500039463046FFF78AFD04460028F4D02DB936
:10DC6000012388F807302046BDE8F88308213046B4
:10DC70007FF0C6FE0028F3D00D4823F033FC0028C7
:10DC8000EED00C4B93F81424B02101FB023203F5C3
:10DC90000053B2F81E22B3F9D6329A42E0DD064BA9
:10DCA0003A46082130467FF0B3FECDE7D04D002044
:10DCB000A02D0020802C0020E8A10C08805C002012
:10DCC000BD8600202DE9F3410E46054615F0C6F944
:10DCD000804614F0ABFA044640B9514A0121284667
:10DCE00080F0B8F8204602B0BDE8F0814D4FD7F87B
:10DCF000EC00036831469B699847044658B9D7F849
:10DD0000EC0003681B6C9847474A034601212846EC
:10DD100080F0A0F8E6E7AB68002BE3D0102128469E
:10DD20007FF06EFE20B3D8ED937A98ED920A20EE44
:10DD3000270AB5F099FBDFED3D7AA7F5805320EE79
:10DD4000270AB3F9A832DFED3A7A20EE270A07EE68
:10DD5000903AF8EEE77AB4EEE70AF1EE10FA07DD52
:10DD6000344B0122102128467FF052FE0024B9E7EF
:10DD7000402128467FF044FE38B3012E1ED0232ECA
:10DD80001CD0042E1AD02C4CD4F8DC3CB3F908304B
:10DD900000EE103AA4F50050B8EEC00A00F0BCFB4B
:10DDA000B5EEC00AF1EE10FA1DDD244B00930122FE
:10DDB000234B402128467FF02BFED7E7D7F8EC0015
:10DDC0000368DB6B98470028DDD01E4B1B68D86AC0
:10DDD0000368DB6998470128014619D11A4A284689
:10DDE00080F038F8C2E7D7F8EC0003685B69984721
:10DDF00030B1D4F8DC3CB3F90830002BE5DDD4E7D2
:10DE0000D7F8EC0003681B6898470B28DDD1F0E7D2
:10DE10003146284602B0BDE8F04180F0ABBB00BF00
:10DE2000F8A10C08805C002009A20C08E02E6542D5
:10DE30000000C8421DA20C08804C00206F9F0C08F7
:10DE400025A20C08E084002031A20C0870B505461C
:10DE50000E46FFF78BFC084B0446D8713146284626
:10DE6000FFF740FD31460028284608BF002480F017
:10DE700059FD204070BD00BFBD8600202DE9F04156
:10DE80004E4F3B78002B40F096804D4CD4F810510B
:10DE900095F8CB5001263E701DB13B702846BDE879
:10DEA000F08180F06BFF054630B9464A3870137830
:10DEB00043F001031370F1E756F084F8314655F052
:10DEC000BBF9A4F5405006F047FD3F4B1E710B26F1
:10DED0004AF094FF013E4AF05FFF16F0FF06F7D1CB
:10DEE0003A4800F083FF15F0B9F8D0F80022C4F8E2
:10DEF000382190F87C32DA074DD414F019FC56F032
:10DF000061F83C2155F09AFF0023C4F8F830002155
:10DF10002E482F4E00F0F0FF2C4812F089F80146F1
:10DF20002C488CF08DF82C4B1B68D86A03680121B3
:10DF30001B689847D4F8100103689B6A9847012131
:10DF4000D4F8100189F0C4F856F03CF88046D4F8B3
:10DF5000EC0003681B68984796F868220146404623
:10DF600055F042FBA6F5005006F0E8FC53F024FA09
:10DF700052F060FD00233B7091F042F8B4F8E230BB
:10DF800006F5005623F4087343F02003C6F8340D59
:10DF9000A4F8E23082E79B07B9D431460B4804F07D
:10DFA0005FFD0E4888F0E8F8DFED0D7A20EE270AD5
:10DFB00084ED3E0AABE7002570E700BF782C002017
:10DFC000805C0020DC860020BD860020802C0020A4
:10DFD000804C00205C570020E084002080790020E5
:10DFE0000AD7233C2DE9F043374DD5F8103193F88B
:10DFF000CB3087B0002B64D062B1012901D0232936
:10E0000008D195F9E030002B04DB0024204607B04E
:10E01000BDE8F08380F05EFF04460028F5D015F0DF
:10E020001DF807461CF078F88046384613F008FEC5
:10E03000D8B198F92430022B17D100264FF00009EF
:10E04000F1B203AA38460191CDF80C90CDF81090AA
:10E05000CDF8149014F092F9019918B103AA404632
:10E060001BF00AFD0136032EEAD11848012106F003
:10E07000DFFE1648012106F00FFE0021D5F8100141
:10E0800089F026F8124832F0BFFE55F09BFF0021C0
:10E0900055F0D2F80F4B1B68D86A036800211B6843
:10E0A000984795F8E230D5F8EC100B486FF345131C
:10E0B00085F8E2300B1A594259413C308FF0A6F9ED
:10E0C000A4E70124A2E700BF805C0020802C002090
:10E0D000447C0020E0840020E07D002010B5064C48
:10E0E000D4F8EC0003685B6A984718B1D4F8103193
:10E0F00093F8CB0010BD00BF805C002030B52DED43
:10E10000028B89B00C46B0EE408AFFF7E7FF054668
:10E11000002838D0B4EE488AF1EE10FA7CBFDFED6B
:10E120001C8ADFED1C7A226863689FED1A0A68BFBB
:10E13000DFED198A029278BF68EE288A02A878BFBC
:10E1400068EEA78AD4ED027A0393F1EE677ACDEDFB
:10E15000047A2FF037FDB4EE488A00220123F1EE55
:10E1600010FACDE900238DED050ACDED060A9FEDED
:10E170000A0A0A488DED071AF0EE680A68BF1346CE
:10E1800005A90DF029FD284609B0BDEC028B30BD74
:10E19000E02E65420000C84200000000FC80002024
:10E1A00007B50191FFF79AFF30B10199044803B018
:10E1B0005DF804EB00F0F6BA03B05DF804FB00BFB5
:10E1C000802C002001486EF06BB800BFD04D0020BD
:10E1D00008B500F5405090F8E030C3F340128A4291
:10E1E0000BD061F3451380F8E03031B155F0EAFE11
:10E1F000BDE808400F2155F021BE08BD70B500F5FF
:10E2000040560546D6F820318B420C4612D00129E3
:10E2100011D0022916D059B955F0D4FE1B2155F062
:10E220000DFE0D4A05F53A500621383057F0C8FF6B
:10E23000C6F8204170BD55F0C5FE1A2155F0FEFD0F
:10E24000064AEFE7012100F057FE55F0BBFE1D2105
:10E2500055F0F4FD024AE5E79CA20C08B1A20C08B7
:10E26000ACA20C0810B500F540520C4692F80531EE
:10E2700003F00101A14209D064F3000382F80531E3
:10E28000DB0704D405F038FF024B9C7210BD06F08A
:10E2900019F9F9E7BD86002000F5405090F80531E6
:10E2A00061F3410380F80531014B1973704700BFDA
:10E2B000BD86002010B5044660F05EFB202161F0B1
:10E2C000D1FB04F54053003893F8E22018BF012039
:10E2D00060F3820283F8E22010BD000010B504460E
:10E2E00053F06AF804F54052436FD2F8102104F558
:10E2F0008044D360D4F81C2D9366D4F8242DC2F842
:10E30000FC32D4F81C0D03685B6D9847D4F81C0DE3
:10E310000368BDE810409B6D1847000070B52DEDF7
:10E32000028B00F540550446D5F8103193F8CB30F8
:10E33000002B71D095F9E030002B6DDB00F58046A5
:10E3400096F8E83E002B67D1D5F8EC0003685B69CE
:10E350009847002860D1324BD3F8EC0003681B6863
:10E3600098470B2858D0D6F8243D9FED2E7AD3ED50
:10E37000DB7AF0EEE77AF4EEC77AF1EE10FA4BD5DD
:10E38000D5F81001443057F051FA0346DFED260A64
:10E3900093ED000A9F20B7EE001A2CF0BDF9B5EE00
:10E3A000C00AF1EE10FA37DD04F59A4087F0F0FE6E
:10E3B000DFED1E7AB0EEC00AB4EEE70AF1EE10FA15
:10E3C0002AD504F58054D6F81C0DD4F8A83407EEED
:10E3D000903A0368D3F89830B8EEE78A984738EE59
:10E3E000400ADFED137AB0EEC00AB4EEE70AF1EEB0
:10E3F00010FA11D5D4F8AC3440F2E63203F2F3133C
:10E40000934209D8BDEC028BD5F810019FED090AA3
:10E41000BDE870408AF0DEB8BDEC028B70BD00BF75
:10E42000805C00200000003400000000000070420A
:10E430000000FA430AD7233C08B500F54050D0F855
:10E44000100103681B699847F6EE007A20EE270A50
:10E45000B5EEC00AF1EE10FA48BF9FED010A08BD03
:10E460000000000038B52DED028B00F58045044614
:10E47000D5F81C3DDFED110A93ED370A04F5405441
:10E480007120B7EE001A2CF047F9D4F81001D5F836
:10E49000245D03681B69B0EE408A984738EE400A55
:10E4A000BDEC028BDFED067A05F50575284620EEFA
:10E4B000270ABDE8384078F04DBB00BF00000000DF
:10E4C00000007A4400F5A853D3ED005AD2ED007A4B
:10E4D000D3ED036A91ED006A26EEE77A67EEA57A3E
:10E4E000A6EE257AE6EE267A81ED007AC2ED007A74
:10E4F0007047000000F50050B0F98C3B33B9B0F91B
:10E50000E2020028B8BF404280B2704783EAE3705D
:10E51000A0EBE370F8E7000070B52DED028B00F57D
:10E52000405382B093F8051111F00106044605D05E
:10E530009FED2E0A02B0BDEC028B70BD8DED010A7D
:10E5400060F01AFA037F002BF2D0DFED298ADFEDAD
:10E55000270A9DED010AB0EE681A4E202CF0DCF877
:10E5600004F500554FF4C8723146B5F9EA02B0EE31
:10E57000408A2CF00FF9A5F8EA02204611F006FBBC
:10E58000B5F9EA3207EE900AB8EEE77A07EE903A6C
:10E59000F8EEE77A77EE676AB4EEE68AF1EE10FA03
:10E5A0000DD52046FFF7A6FF07EE900A38EE668AE3
:10E5B000B8EEE70A20EE088A88EE260ABAE777EE78
:10E5C000877AB4EEE78AF1EE10FAB1DDB5F9E232FE
:10E5D00000EE103A38EE678AB8EEC00A78EEE77AB5
:10E5E00020EE088A88EE270AA4E700BF000000009A
:10E5F00000007A44002070470020704770470000F8
:10E6000000F50B50383070470048704798D20C081E
:10E6100000F54050D0F8EC0003681B681847000074
:10E62000034808603221117008221A60704700BF49
:10E6300058A60C0800F54050D0F8EC000368DB6CDD
:10E640001847000000F54050D0F8EC0003689B6CC0
:10E650001847000000F5405300F59F40D3F8EC3018
:10E6600008301B1A584258417047000010B500F599
:10E6700040500C46D0F8EC000368DB6D984707EE7D
:10E68000900A9FED057AF8EE677A012067EE877AA7
:10E69000C4ED007A10BD00BF0AD7233C10B500F5C9
:10E6A00040500C46D0F8EC0003689B6D984707EE8D
:10E6B000900A9FED057AF8EEE77A012067EE877AF7
:10E6C000C4ED007A10BD00BF0AD7233C10B500F599
:10E6D00040500C46D0F8EC0003681B6E9847DFED05
:10E6E000047A20EE270A012084ED000A10BD00BF45
:10E6F0000AD7233C66F070BF6AF0B8BB62F0E8BB93
:10E7000052F0A4BD29F042BF54F014BF18F07CBBF6
:10E7100062F05EBF5FF08ABD5DF094BE10F0CEBEC9
:10E7200011F028BB06F0B8BD12F040BB05F038BDB3
:10E7300005F084BA05F0AAB968F0CEBC10F00CB8A8
:10E74000FFF7ECBD10F0FEBF11F06CBA03F03EB95C
:10E7500010F082BF10F0FABE60F05CB84BF042BD22
:10E7600024F06EB906F064B902F0F8BC62F040BF64
:10E7700011F076BA06F048BD04F05EB906F0A0BE0E
:10E7800005F016BA06F004BA10F024BEFFF7A6BDD5
:10E790002AF01ABA05F014BF0AF072BA0AF05CB98E
:10E7A0000AF0F0B81FB500F540530446D3F8EC006A
:10E7B000039103685B6A984760B1DFED070A03992C
:10E7C000002304F5A8400093B0EE600A1A467C309E
:10E7D0000DF058F804B010BD0000000010B52DED8C
:10E7E000028B00F540530446D3F8EC0003685B6AE3
:10E7F000B0EE408A984720B90024BDEC028B204639
:10E8000010BD9FED080A04F5A84028EE000A7C30F0
:10E810000CF002FB04460028EED003480121FFF76C
:10E82000D7FCEAE70000C842802C00200A4A92F98F
:10E83000E020002A0B4605DA00228A604A600A605E
:10E840000120704700F58040D0F81C2D783207CAAF
:10E8500083E80700F4E700BF805C002070B5204B20
:10E86000036000F500531F4AC3F8B82E00F540536B
:10E870000446586F08B11AF087FE1B4B236004F55D
:10E88000805393F8342F42B9D3F8305F2DB1284626
:10E8900028F084FC28461AF073FE04F58D501C30D5
:10E8A0007EF0F8FA04F58650043062F045FD04F677
:10E8B000F44504F69446B54204D0183D284628F0A5
:10E8C000C3F8F8E7094BC4F8C83804F6C41056F08A
:10E8D00089FC04F5136056F085FC204670BD00BF2E
:10E8E00050AA0C08E4B40D0888950D08C05F0D0807
:10E8F00038B54B4B044640F8043B66F08DFF04F1FD
:10E90000100017F01DFF04F1680052F02DFA04F515
:10E91000907022F0F7FC04F58C6016F02BFC04F2EA
:10E9200084501AF033FE04F6C80029F0D3FC04F535
:10E93000476066F04FFD04F554604FF04DF804F564
:10E940007F6054F0D9FB04F5855008306CF0FEFD73
:10E9500004F58650043062F0D7FC04F5885019F0B5
:10E9600037FC04F58D501C307EF080FA04F58E5093
:10E97000183052F0BBFD04F591500C3068F0F6F8F9
:10E9800004F580530025274A83F8505204F592532A
:10E99000103304F5935013604AF072F804F5955063
:10E9A0002946103012F03CFE04F5C85078F010FBF8
:10E9B00004F5EE5004307BF079FA04F5F6501C3083
:10E9C0007DF0AEFB04F5FA507DF0E4FF04F5FC5059
:10E9D000183012F027FC04F50350383079F034F881
:10E9E00004F5055010306DF073F904F5085010303F
:10E9F0007EF0D8FD04F5005304F50A5083F8685200
:10EA0000094D7EF0F1FE2B6813B1084890F0C6FA6C
:10EA1000204607494DF0A6FE2C60204638BD00BFB9
:10EA200088950D089C900020A4870020C0A20C08A7
:10EA300090940D0810B511F01DF85FF09DFF03686C
:10EA4000BDE810405B681847FFF7F4BF10B50446F7
:10EA500006F03AF9204611F013FB204603F03CFE85
:10EA60002046BDE8104003F09DBF0000FFF7EEBF59
:10EA700070B500F544553C350446284617F03AFD7C
:10EA80001BF04AFB90F9213093B390F840337BB3ED
:10EA900004F5405304F28456D3F81001443056F084
:10EAA000C5FE0346DFED130A93ED000A9F20B7EE83
:10EAB000001A2BF031FE94F9B835012B284608BF17
:10EAC00086ED0E0A002117F0A9FADFED0B7A04F2A9
:10EAD000DC7494ED287A20EE270ADFED087AA7EEA1
:10EAE000270A304684ED280ABDE870401BF024BA9E
:10EAF00070BD00BF00000000CDCCCC3D6666663F17
:10EB0000FFF7B6BF10B50121044611F0F5FA60B168
:10EB1000114BD3F8EC0003689B6A984728B920464C
:10EB200002F02AFA204602F037FA4FF4001120468C
:10EB300011F0E2FA18B12BF0C1F829F0A7FA4FF45E
:10EB40008021204611F0D8FA28B12BF0B7F8BDE8A3
:10EB5000104029F0A9B910BD805C0020FFF7D2BF9A
:10EB600070B500F580450446D5F81C0D9FED5A0A96
:10EB700086B06C302FF026F804F5955003A91030BC
:10EB80008DED030ACDED040A8DED051A12F0F4FBAC
:10EB90000221204611F0B0FA70B10121204611F097
:10EBA000ABFA48B94D4BD3F8EC0003689B6A984721
:10EBB00010B9204602F0E0F90121204611F09CFA3C
:10EBC00048B9464BD3F8EC0003689B6A984710B9E4
:10EBD000204602F0E1F90121204611F08DFA10B92A
:10EBE000204602F031FA4FF40031204611F084FA49
:10EBF00030B104F54053D3F8100103685B6C9847BB
:10EC00004021204611F078FA60B104F57F60019050
:10EC100053F030FE04F58053019893F9C4300BB1E2
:10EC200053F06AFF4FF48061204611F065FA18B185
:10EC300004F57F6053F0B8FE2021204611F05CFA05
:10EC400058B104F54056D6F8EC0003681B699847A4
:10EC500018B3D5F8240D84F087FA8021204611F0EE
:10EC60004BFA38B32BF02AF829F042F9102120464C
:10EC700011F042FA18B1D5F81C0D80F0BBFF4FF42B
:10EC80000041204611F038FA18B304F59B403C309F
:10EC900006B0BDE8704062F0DDBD20460DF0ACFC72
:10ECA0000028D6D1D6F8EC0003685B6998470028A5
:10ECB000CFD0D2E74FF48021204611F01DFA002872
:10ECC000D0D14FF40021204611F016FA0028C9D106
:10ECD000CCE706B070BD00BFE02E6542805C00202E
:10ECE000FFF73EBF10B50121044611F005FA10B13F
:10ECF000204602F0A9F98021204611F0FDF958B113
:10ED00004FF48021204611F0F7F928B92AF0D6FFF8
:10ED1000BDE8104029F0C8B810BD0000FFF7E2BF01
:10ED200010B5044605F020FD204605F06BFB20469B
:10ED300005F060FD204612F0A9F82046BDE810401D
:10ED400003F0A6BCFFF7ECBF70B54FF6FF710446A9
:10ED500011F0D2F904F5405528B1D5F8E02007218B
:10ED6000204602F0A1F9D5F8103193F8CB308BB9D9
:10ED70002046FFF79FFAD5F8100104F5005302680A
:10ED800093F87413166A93F8FE22B047D5F8100171
:10ED900089F0ECFB61F050FC61F04CF9204612F078
:10EDA00073F895F8E0300F4A04F58044DB43D4F85B
:10EDB0001C5DC3F3C01353712B681E6F52F0FCFA35
:10EDC00051F064FF2846B047D4F8244D52F0F4FACD
:10EDD00004F5057451F05AFF2046BDE8704077F005
:10EDE0001FBD00BFBD860020FFF7AEBF70B500F5A8
:10EDF000A85300F540551B68C5F8243100F580562E
:10EE000006F20C5304461B68C5F82831D6F8B00446
:10EE100000F58C4050302BF053FCD5F82431C5F868
:10EE20003031D5F82831C5F82C01C5F834314FF60A
:10EE3000FF71204611F060F938B1D6F8B0242046B1
:10EE40000921BDE8704002F007B970BD30B500F58A
:10EE50004053D3F82041002C4CD093F8E120D10747
:10EE600048D56FF3000283F8E12000F50052012C31
:10EE7000D2F8D41CD2F8D85CB1F908400BBFD3ED5E
:10EE80004A5AD3ED4D5AD3ED497AD3ED4C7A07EE79
:10EE9000104AB5F9084006EE904A0CBFF8EEE66A53
:10EEA000F8EEE66AB8EEC77A25EEE66A00F5A853F2
:10EEB000A7EE276A67EEA67AD3ED006AE7EE257A19
:10EEC00093ED037A27EE877AA6EE267ABDEEC77A0F
:10EED00017EE104A0C8193ED007AD2F8D82C67EE29
:10EEE000877A93ED037AE6EE477AFDEEE77A17EE3E
:10EEF000903A138130BD000038B505462DED028BE8
:10EF000000F5405471B1284610F03CFCD4F82C3187
:10EF10001B1A03F2F31340F2E63293420CD8BDEC15
:10EF2000028B38BDD4F82031022BF8D110F00EFC42
:10EF3000B0F57A7FE7D2F2E7C4F82C0100F58C40F7
:10EF40005030642390FBF3F308EE103ADFED097ABA
:10EF5000B8EEC88A28EE278AB0EE480AB4F09AF8CC
:10EF600084ED4C0AB0EE480AB4F01AFA84ED4D0A6A
:10EF7000D5E700BF35FA8E3C00F5955001211030E1
:10EF800013F0D0BFFFF7F8BF10B5044610F004FE31
:10EF90001021204611F0B0F870B1204601F048FF72
:10EFA0004FF40011204611F0A7F828B92AF086FE88
:10EFB000BDE8104029F06AB810BD0000FFF7E4BFBB
:10EFC000F8B50446254606F0A3F9224B45F83C3B2C
:10EFD000214BA465C4E91734204BC4E91934204BF4
:10EFE000E36604F1800019F03FFF04F19C0019F082
:10EFF0003BFF04F1B80019F037FF4FF6FF76194BCD
:10F00000C4F8CC30A4F8D06004F1D40019F02CFF7F
:10F010004FF0FF37144B1549C4F8307128461D6076
:10F020004DF0A0FBA4F87870A4F8946004F5A270E9
:10F0300019F01AFF04F5B07019F016FF04F5BE7050
:10F0400019F012FF002384F89031C4F8B43120463F
:10F05000F8BD00BF4CFF0C0899E700089DE70008C9
:10F06000A1E700080000FFFF88860020A46C0D08BF
:10F0700010B5044606F04CF90A4B23600123A38720
:10F0800004F1400019F0F0FE04F1500019F0ECFE1C
:10F0900004F1600019F0E8FE04F1700019F0E4FEDC
:10F0A000204610BD30090D082DE9F047044688B010
:10F0B000FFF71EFCA44B236004F50C50203004F530
:10F0C000005502F027F904F50B532C3304F53356A1
:10F0D000C5F8E83C062385F8EC3C4FF07C5705A9C1
:10F0E00006F13800059756F093FC06F150008FF0BA
:10F0F00031F9002304F59A4985F8283D192304A91C
:10F1000085F8343D04F53456C5F8309D04F5355086
:10F11000049756F07DFC06F158008FF01BF901268C
:10F12000182304F5365004F5375785F87C3D3837F9
:10F1300085F8706DC5F8789D103061F0F7FC3846A1
:10F140007EF00EFC814B8DF8186006AEC5F8F83DD8
:10F150003146381D4EF01CF904F5385030304AF075
:10F16000FFFF04F5395030307EF0E4FB784B794FE7
:10F17000C5F8703E04F53A5031460830069756F00F
:10F1800047FC04F53A5031461430069756F040FCDF
:10F1900004F53A503146203004F53A5A06970AF100
:10F1A000380A56F035FC6C4BC5F8B83E0AF114002D
:10F1B0008FF0D0F804F53B5704F53D58303708F18F
:10F1C0001408384614375BF005FAB845F9D104F550
:10F1D00040580723C8F878300023A8F87C304FF453
:10F1E000CB701AF0CBF9C8F8740004F542508FF0D8
:10F1F000B1F804F5435004308FF0ACF8574B1A685F
:10F200000AB9C3F800A004F5AC47554BC5F8B83EA1
:10F21000643704F54350C8F8EC7030307FF07AFE64
:10F22000504B07934FF07E554F4BC8F82451C8F808
:10F2300030510694009304F5445096E80C004FF4C6
:10F2400000713C3016F09CFD04F55A50303070F0DF
:10F25000E7FC04F5994003A95030039556F0FEFBF6
:10F2600004F5994003A96430039556F0D1FB04F5E9
:10F27000994004F58045703019F0F6FD05F60C5301
:10F280000026C9F80060C9F80460C9F808601E606B
:10F290005E609E6004F595531033C5F8183D04F583
:10F2A0009A40002385F8393D4FF400413C3017F077
:10F2B00031FB04F59B403C3062F074F904F59C404E
:10F2C00040306EF03BFE04F59C407C304EF096F9E9
:10F2D000264BC5F87C3E04F59D40254B2549103052
:10F2E00004F59D48186008F130084DF03BFAFF2303
:10F2F00085F8C03E85F8C83E1F4940464DF032FAB9
:10F300001E4A136813B11E488FF048FE1D491E485F
:10F31000C2F8008004F59D42583208604FF0140E88
:10F320001FFA83FC0EFB0C010133097C0029F7D185
:10F33000164BA3F800C0164BD3F80080B8F1000FAD
:10F340002AD01448E0E700BF50AA0C0848A20C08D5
:10F3500088A20C080000A040E4B40D08EC8A00204C
:10F36000D0AA0C0895E7000840AA0C0898A20C083F
:10F37000A4900020B0C90D08485C0E083891002008
:10F38000D4A20C0860870020B8EC0C085C87002031
:10F3900018870020F5A20C0804F59D401A6003A907
:10F3A000584B03936C3056F033FB04F59E400C3001
:10F3B00005F0AEFF544BC5F80C3F04F59E404C30B1
:10F3C00005F0A6FF04F5A249504BC5F84C3F04F5E3
:10F3D0009F4009F16009083004F5A045FFF7F0FDF2
:10F3E000484605F095FF4A4BC5F8603109F13C00ED
:10F3F0008CF094FC474BC5F89C3104F5A6402030B6
:10F4000005F086FF444BC5F8203304F5A640643070
:10F4100005F07EFF414BC5F8643304F5A74085F83D
:10F42000A083243005F074FF3D4BC5F8A43304F5E8
:10F43000A740603005F06CFF3A4BC5F8E03305F2A9
:10F440001C4304F5A8401E605E609E60343005F0E9
:10F450005FFF354BC5F8343404F5A840C5F8708417
:10F460007C3005F055FF314BC5F87C3404F5A940DC
:10F47000C5F8B884403005F04BFF2D4BC5F8C034BB
:10F4800004F5AA40083005F043FF2A4BC5F80835BB
:10F4900004F5AA40443005F03BFF274BC5F844353E
:10F4A00005F2BC5304F5AB401E605E605830FFF7B8
:10F4B000DFFD384605F02CFF204BC5F8643604F517
:10F4C000AD40203005F024FF1D4BC5F8A03604F5F3
:10F4D000AD40A5F8DC867030FFF7CAFD194BC5F8C2
:10F4E000F036012385F8793704F5AF4318461E60DE
:10F4F0005E609E600C300AF04BFD204608B0BDE80F
:10F50000F08700BFCDCC4C3D44FB0C08E8FB0C0859
:10F51000F0FF0C0880000D083C010D08DC010D080F
:10F520007C020D0814030D0850050D08F0050D08A8
:10F5300080060D0818070D08B8070D088C0A0D087D
:10F54000280C0D08E8090D0838B5054B1C68236820
:10F550000A461D68034B01462046A847002038BDD7
:10F56000E0840020802C002010B58FF069F9064C53
:10F57000064B18602046FFF797FD2046044A0549D0
:10F58000BDE81040B3F060BC802C0020E084002077
:10F59000D4E500205DE800080120704790F89C3019
:10F5A0008B4286BF283150F82100002070470000B0
:10F5B00090F89C308B4286BF283150F82100002003
:10F5C00070470000FA207047014B93F8AE02704775
:10F5D000804C0020034BD3F82001431E5842584171
:10F5E000704700BF805C0020034BD3F82001831ECE
:10F5F00058425841704700BF805C0020034BD3F84D
:10F60000100108B187F05CBE01487047805C0020A3
:10F61000BCAA0C0838B5C36A2E4D43F4E052C2624E
:10F62000026B42F4E0520263426B42F4E0524263E6
:10F63000D5F8242D0446E2B143F4F843C362D5F86B
:10F64000240D83F051F938B1236B43F480432363D5
:10F65000636B43F480436363D5F8240D83F066FA4B
:10F6600038B1236B43F400532363636B43F40053BB
:10F670006363194B1D6845B1192128464EF086FA7F
:10F6800018B1E36A43F48073E362144B93F8F03CDF
:10F690006BB1236B43F48073236345B11921284672
:10F6A0004EF0ACFA18B1636B43F480736363E36AA2
:10F6B00043F08043E362236B43F080432363084BB2
:10F6C000D3F8103193F8C1301BB9636B43F080431A
:10F6D000636338BD806C002070870020804C002060
:10F6E000805C002013B54FF44470CDE9002119F07F
:10F6F0003FFF044628B1DDE900215DF075FE024BB5
:10F700002360204602B010BD14AD0C0800207047E5
:10F71000704700000320704708207047014B93F8A2
:10F72000B0027047804C0020034B93F96803003807
:10F7300018BF0120704700BF804C0020014B93F997
:10F74000B2027047804C00207047000070470000F4
:10F7500008B50C4BD3F8240D70B910230A4AD2F81F
:10F76000102143F0400022B192F8CB200AB143F0BF
:10F77000C00040F0010008BD83F0B6F80028ECD0CE
:10F780001823EBE7806C0020805C002038B5C5783A
:10F790000B46352D044628BF352535220021184655
:10F7A000B6F0C0F82A4604F10C01BDE83840B6F0C6
:10F7B0006FB800001FB5184C94F8E610A4F168006B
:10F7C00011F01AFD78B194F8E610A4F1680011F078
:10F7D00015FD40B194F8E610A4F1680004B0BDE84E
:10F7E000104011F00DBD002301930293039313F019
:10F7F00035FC01A913F0FEF920B101A82EF0E0FDBF
:10F8000004B010BD23F05AF990F8F432B02202FB94
:10F81000030090ED3B0AF3E7804C002008B50D4B48
:10F82000D3F81001A8B1443056F000F8034693ED28
:10F83000000ADFED090A9F20B7EE001A2AF06CFFDC
:10F84000DFED067A20EE270ABDEEC00A10EE103A70
:10F8500018B208BD805C0020000000000000C84213
:10F860002DE9F04FDFF8D880344F8DB004460425E1
:10F8700008F5005617F8019BB8F9083309F1FF3A6B
:10F8800043FA0AF3D90742D5207C57F063FC83463C
:10F89000207C58F063FB00F121039B4505D2207CBE
:10F8A0000DB0BDE8F04F56F0ABBEBAF1030F2ED845
:10F8B000DFE80AF00234393ED6F81C0D03689B6875
:10F8C000984700F194035A69D3F800A0D3F804E0F4
:10F8D000D8681969D3F818C008925A6A1B6ACDF81B
:10F8E0002520CDF8293062222123CDE9003206906F
:10F8F0000791207CCDF80CA0192303AAC221CDF8D2
:10F9000010E0CDF814C08DF8249057F08DFC013D27
:10F9100015F0FF05AED10DB0BDE8F08FD6F81C0D87
:10F920000368DB68CCE7D6F81C0D03681B69C7E7E2
:10F93000D6F8243D03F52A73C5E700BFE8AD0C08EF
:10F94000804C002013B504460748019108F0CCFF15
:10F9500030B90199204602B0BDE8104058F03EBDD4
:10F96000042002B010BD00BF087C0020014808F050
:10F9700097BD00BF087C002037B504460D460648F9
:10F98000019211468AF08EFF019A2946204603B063
:10F99000BDE830405CF0F6BB1858002010B588B0C8
:10F9A000044659F019FF0C4BD3F8100138B90B4A33
:10F9B0000621204608B0BDE8104059F0F5BE694662
:10F9C0001E2287F081FC064A6B460621204659F02C
:10F9D000EBFE08B010BD00BF805C002008AB0C0837
:10F9E000C2F80C08034A92F8D03C013382F8D03CAC
:10F9F00058F0B6BF804C002007B50846019119F0B9
:10FA000009FB38B10448019902F0DEFC002003B084
:10FA10005DF804FB0420FAE7EC840020F7B58B8B3B
:10FA2000CD2B06460C4617461DD1D1ED067AFCEECD
:10FA3000E77ACDED017A9DF80430022B13D10E4DFB
:10FA400095F8351E05F6BC5061F0E2FD58B195F809
:10FA5000351E05F6BC5061F0E3FD20B994ED020AB5
:10FA6000064802F091FC3A462146304603B0BDE814
:10FA7000F04059F007B800BF806C0020EC840020F3
:10FA8000162A10B40C4605D0542A03D05DF8044B56
:10FA900058F0C0BC0323237001205DF8044B70476D
:10FAA00008B558F013FF40F41C6040F00D0008BD8D
:10FAB00010B5044619F064FD204610BD10B50C4C7D
:10FAC00094F9E030002B0FDBD4F8EC000368DB6C1A
:10FAD000984758B9D4F8EC0003689B6C9847002805
:10FAE0000CBF0220032010BD0120FCE70420FAE730
:10FAF000805C002010B44C69012C05D101465DF8F2
:10FB0000044B034802F0F4BF5DF8044B58F042BFC9
:10FB1000802C00202DE9F341B1F90430002B06467A
:10FB20000C46154635DB4FF00008CDE900281A4F8A
:10FB3000B1F902209FED190AD7F8D41C4FF47A735B
:10FB40005CF008FE0123CDE900539FED140AB4F9DF
:10FB50000020D7F8D81C4FF47A7330465CF0FAFDD9
:10FB60009FED0F0AB4F90420D7F8DC1C4346304659
:10FB7000CDE900585CF0EEFDCDE900589FED070A95
:10FB8000B4F90620D7F8E01C4FF47A7330465CF0E5
:10FB9000E1FD02B0BDE8F081804C00200000FA4495
:10FBA00000007A44044B187820B9044B93F8E20023
:10FBB000C0F38010704700BF58860020805C002092
:10FBC0000B4B93F8AD267AB993F8052192060BD129
:10FBD00093F9E020002A09DB93F8E13013F0200FBD
:10FBE00014BF042001207047052070470320704790
:10FBF000805C002008B5074B93F9FC32032B03D03F
:10FC0000BDE8084059F048BE034A022159F0CCFD36
:10FC1000042008BD804C002020AB0C08094BD3F811
:10FC20006C23920701D458F0E9BB03F5005303F6A7
:10FC3000F44393ED000ADFED047AB8EEC00A20EE3B
:10FC4000270A7047804C00200AD7233C10B594B097
:10FC5000044603A819F008F91C4BD3F8EC0003681C
:10FC600003A95B6D984778B3002103A819F094F9B4
:10FC700050B3247C8FF0C4F9059BDDED047A089322
:10FC8000069B09930023F8EEE77A9FED117A0B9318
:10FC90000C930D930E930F931093119312934FF6B1
:10FCA000F853ADF84C300023962267EE877A8DF832
:10FCB0004E303323CDE90032079007AA5721204662
:10FCC000CDED0A7A57F0B0FA14B010BD805C002078
:10FCD0000AD7233C30B52DED0A8B774C0546D4F876
:10FCE000EC00036899B05B6A984700285BD004F584
:10FCF0000054D4F8B834062B00F2C980DFE803F0D2
:10FD00000404045788AB53006C489FED6D8A0BF0D8
:10FD100081FF9FED6C0A0168426883680D930BA810
:10FD20000B910C922DF04EFFF0EE489AB0EE40CAC7
:10FD3000F0EE60BAB0EE419AB0EE48AAF0EE488A12
:10FD4000F0EE48AAB0EE48BA40F6F8542D7C8FF099
:10FD500057F900231593169301238C228DF85E30FA
:10FD60003323CDE900320B90B1EE499AF1EE688A67
:10FD7000B1EE488A0BAA552128468DED0CCACDED6F
:10FD80000DBA8DED0E9A8DED0FBACDED10AACDED19
:10FD9000118A8DED12AACDED139A8DED148AADF86E
:10FDA0005C4057F041FA19B0BDEC0A8B30BD4348B6
:10FDB0000BF030FF9FED430A0168426883680D93A2
:10FDC0000BA80B910C922DF0FDFE3C48F0EE60BAB2
:10FDD000B0EE419AB0EE40CA0BF020FF9FED390A19
:10FDE0002DF0F0FE3548B0EE40BAF0EE60AAF0EE2D
:10FDF000418A0BF017FF9FED330A2DF0E3FE4FF41D
:10FE00004064B0EE40AAF0EE609AB0EE418A9DE701
:10FE10002A489FED2B9A0BF001FF9FED2A0A2DF047
:10FE2000D1FE2648B0EE40BAF0EE60AAF0EE418A6C
:10FE30000BF0F8FE9FED230A2DF0C4FEF0EE49BA58
:10FE4000B0EE40AAF0EE609AB0EE418AB0EE49CA38
:10FE500040F607447AE71948DFED198A0BF0E2FE15
:10FE60009FED180A2DF0AEFEF0EE68AAB0EE40AAA3
:10FE7000F0EE609AB0EE418AB0EE68BAB0EE689AE1
:10FE8000F0EE68BAB0EE68CA40F63F445EE79FED18
:10FE90000C8A0024F0EE489AB0EE48AAF0EE488AA8
:10FEA000F0EE48AAB0EE48BAB0EE489AF0EE48BA82
:10FEB000B0EE48CA4AE700BF805C0020FC8000200A
:10FEC000000000000AD7233C2DE9F0412DED068B00
:10FED0003B4D95F8E13099068CB004466AD505F59E
:10FEE00080579FED380AD7F81C0DDFED378A6C304C
:10FEF0002DF068FE8DED041A21EE281AD5F8EC607D
:10FF00008DED020ABDEEC11ACDED030A11EE103AD5
:10FF10001DB2336894F810809B6D304660EE289ACD
:10FF200020EEA89A984707EE900AF8EEE77A304656
:10FF300067EEA87AFDEEE77A17EE903A1CB23368C6
:10FF4000DB6D984707EE900AB8EE678AD7F8243D34
:10FF5000DFED1E7A93ED0FAA336828EE288A1B6E18
:10FF6000B4EEE78AF1EE10FA58BFB0EE678A304679
:10FF70009847BCEEC88A0023089318EE103AB722BF
:10FF80002AEE28AA20EE280AADF82C301A23CDE953
:10FF900000323E2105AA4046CDED059A8DED069A28
:10FFA0008DED07AA8DED090AADF82850ADF82A406D
:10FFB00057F03AF90CB0BDEC068BBDE8F08100BFFC
:10FFC000805C00209F0CB3450AD7233C00FF7F478D
:10FFD0002DE9F04F2DED028B1A4B047CD3F81C3D1C
:10FFE0008DB0D3F88480D3F88870D3F88C60D3F8C0
:10FFF000905093ED258AD3F898B0D3F89CA0D3F80D
:020000040801F1
:10000000DC908EF0FDFF00238DF82C301622252386
:10001000CDE90032029002AA532120468DED078AD5
:10002000CDF820B0CDF824A0CDF82890CDF80C80E4
:1000300004970596069557F0F7F80DB0BDEC028BC6
:10004000BDE8F08F806C002070B58A7A4B7A43EA65
:100050000223CA7A43EA02439D2B06460C4621D16D
:10006000134D95F8351E05F6BC5061F0D1FAC8B1B4
:1000700095F8351E05F6BC5061F0DEFA022811D164
:1000800095F8351E05F6BC5061F0CAFA50B9D4EDAA
:10009000057A9FED080A0848F8EEE77A27EE800A0D
:1000A00002F072F921463046BDE8704058F058BB66
:1000B000806C00200AD7233CEC840020054BD3F849
:1000C00010312BB193F8CA00002808BF02207047F6
:1000D00002207047805C002008B5034BD3F8EC0089
:1000E00003681B68984708BD805C0020024B93F8AA
:1000F000E100C0F340107047805C002070B52C4ECA
:100100002DED028B0546D6F8EC0091ED018A0368CF
:1001100086B05B6A0C46984750B9BDEEC88A18EEA7
:10012000103ADB0704D4022006B0BDEC028B70BD90
:10013000D4E904012BF0A0FB0028F4D002A818F0A9
:1001400093FE02AA214628465CF074FA0028EAD001
:10015000184902A818F06AFF03460028E3D1DFED32
:10016000160A00900246B0EE600A144802A90BF08D
:1001700089FBD8B1D6F8EC0003685B6A984704465F
:1001800008B10020D0E70E480222042105F058FCF7
:1001900060B1DFED090A094800942346B0EE600A19
:1001A000224602A90BF06EFB0028EAD10420BBE72F
:1001B000805C00207079002000000000FC8000209E
:1001C000802C002008B591F82030032B1CD1D1EDF4
:1001D000027A9FED0E7A91ED060A0D4BF0EEE77A6A
:1001E000F4EEC77ADFED0B7AD3F8EC00F1EE10FAFB
:1001F0004CBF0121002120EE270A10F095FA0028BB
:1002000014BF0020042008BD0220FCE700000034D9
:10021000805C00200000C84210B52DED028BD1EDAE
:10022000007AF5EEC07AF1EE10FA82B00C4604DAEC
:10023000042002B0BDEC028B10BD9FED197AF4EEE4
:10024000C77AF1EE10FAF3D891ED030A9FED158A03
:10025000F0EEC07AF4EEC87AF1EE10FA19D5D4EDCA
:10026000037A1148D4ED010A94ED000AF4EEC87A3D
:10027000D4ED027AFDEEE77AF1EE10FACDED017AD7
:100280009DF90410ACBF0122002201F0DFFF002025
:10029000CFE7F7EE000A2AF03BF90028C8D0DEE7E6
:1002A0000000B44300000034EC84002091ED010A0A
:1002B000B5EEC00AF1EE10FA08B501DC042008BD65
:1002C0009FED107A104BD1ED007AD3F8EC0020EEC0
:1002D000070A9FED0E7A0368F4EEC77AF1EE10FA82
:1002E00005DDDB6E98470028E8D00020E7E79FEDAA
:1002F000087AF4EEC77AF1EE10FACCBF9B6E5B6E13
:10030000F0E700BF0000C842805C00209A993940A5
:100310003333F33F08B5D1ED007A9FED157AF0EE57
:10032000E77AF4EEC77AF1EE10FA1DD5D1ED017A35
:10033000F0EEE77AF4EEC77AF1EE10FA14D50D4834
:100340000222032105F07CFB80B10A480121FDF760
:100350003FFF094890F8C83F012B03D000F6C47056
:1003600030F0A8FF002000E0022008BD0420FCE7D8
:1003700000000034802C0020806C002010B5D1EDEE
:10038000007AFCEEE77A17EE903A9CB2012C02D08C
:10039000022C06D04CB90648214667F01FF8002011
:1003A00010BD044803F05CF9F9E70420F8E700BF4A
:1003B000107B0020802C00201FB5D1ED017A0B7C32
:1003C000FCEEE77ACDED027AD1ED007A0093FCEEF7
:1003D000E77AD1ED030ACDED037A91ED020A9DF89B
:1003E00008309DF80C20014602480EF059FF05B078
:1003F0005DF804FB802C002010B50A4C94F8053100
:10040000DB070CD402220521A4F5405005F018FBAF
:1004100028B902221146A4F5405005F011FB002036
:1004200010BD00BF805C002010B5D1ED007AFCEE5D
:10043000E77A044617EE903A13F0FF030FD10F4B03
:10044000D3F8EC0003689B6F984708B1002010BDFB
:100450000B4A2046062159F0A7F90420F7E7012BA3
:1004600009D1064BD3F8EC000368DB6F98470028EE
:10047000ECD1044AEDE70220E9E700BF805C0020F0
:1004800044AB0C0854AB0C089FED0B7A01F10C0344
:10049000F1EC017AF4EE677AF1EE10FA0AD6F0EE9A
:1004A000E77AF4EEC77AF1EE10FA03DC9942EFD165
:1004B000012070470020704700007A4430B52DEDD0
:1004C000028B8DB00023054603930493059312F02D
:1004D000C5FD03A912F08EFB58B312F0BFFD00F565
:1004E0005A7393E8070006AC84E80700DDED060ABE
:1004F0009DED070A2D7CF1EE600AB1EE400AB3F0E3
:100500001BF82046B0EE408A2DF05AFFDFED0B7A43
:10051000089B0B93012228EE278A0C23CDE9003299
:10052000A82109AA28468DED098A8DED0A0A56F000
:100530007BFE0DB0BDEC028B30BD00BFE02E6542EE
:10054000242938B505460FD003D81B2907D101242B
:1005500012E04029FBD0A1F14203012BF7D9284634
:10056000BDE838405CF052BA0C2156F05BF8044606
:1005700010B12846FFF7A2FF204638BD38B5194C08
:1005800094F80531DB070D460AD4D4F8103193F8FE
:10059000CB303BB901221146A4F50270FDF76EFC89
:1005A000002038BD94F9E030002B4FF0020212DA3F
:1005B0000521A4F5405005F043FA0028F0D095ED50
:1005C000000ADFED097AD4F8EC0020EE270A0121B9
:1005D00010F0AAF8E4E70921A4F5405005F030FA3C
:1005E000DEE700BF805C00200000C84210B5214C4F
:1005F00094F80531DB070ED4D4F8103193F8CB30E2
:100600004BB194F9E030002B07DA01220821A4F560
:100610000270FDF7E7FC002010BDD1ED007A9FEDE0
:10062000167AF0EEE77AF4EEC77AF1EE10FA0BD50F
:1006300012480222112105F003FAA0B90222114644
:100640000E4805F0FDF9E6E7D4F8EC0003681B68F6
:1006500098470428DFD0D4F8EC0003681B6898475B
:100660001428E5D1D7E7064840F6C41108F03EFE4D
:10067000D1E700BF805C002000000034802C002007
:10068000A07F002073B58B8BC12B05460C4644D848
:10069000BB2B0DD8202B63D02ED8113B99B2052946
:1006A00018D92146284602B0BDE870405DF0A0BAD6
:1006B000BC3B052BF5D801A151F823F0FB0701083D
:1006C00005080108A3060108A3060108930701080D
:1006D0009F070108052BE4D801A151F823F000BFC2
:1006E000E1070108A3060108A3060108F5070108B0
:1006F00007070108B5070108732B2CD006D8542B27
:1007000058D0552BCDD1022209216BE0B22BC8D194
:1007100002B0BDE87040FFF7C9BD4AF21146B342CE
:1007200054D00BD8D12B40D0B3F5967F53D0D02BDB
:10073000B7D102B0BDE87040FFF720BE4AF21246C2
:10074000B3423ED04AF21346B342AAD102B0BDE84A
:100750007040FFF74BBF02B0BDE87040FFF75CBDD3
:10076000D1ED007AF5EEC07AF1EE10FA4FDD9FED93
:10077000297AF4EEC77AF1EE10FA48D8FCEEE77A5F
:10078000254ACDED017A9DF80430A2F89A3B00206D
:100790002EE0214602B0BDE87040FFF7AFBC214615
:1007A00002B0BDE87040FFF73FBE02B0BDE8704048
:1007B000FFF702BE2146284602B0BDE87040FFF7B1
:1007C00001BD02B0BDE87040FFF7D8BE02B0BDE881
:1007D0007040FFF711BE02B0BDE87040FFF79ABD50
:1007E000022205210D4805F02BF90028CFD1042065
:1007F00002B070BD02220621F4E70221084806F08B
:1008000097FAF2E70221064806F05CFAEDE70220CB
:10081000EEE700BF00007F43804C0020802C0020CA
:10082000087C002008B591ED007AF6EE007AB4EE6F
:10083000E77AF1EE10FA06DD044801220521FDF702
:10084000D1FB002008BD0420FCE700BF785A00203F
:1008500030B52DED028BCD7893B0272D28BF2725FD
:100860000C462722002108A8B5F05CF82A4604F1BE
:100870000C0108A8B5F00CF8424BD3F8EC00036863
:100880005B6A9847002841D09DF8465068063DD4E1
:1008900000244FF07E532906049307940694059490
:1008A00027D504A82CF038FCEA070194029403949D
:1008B00005F006032ED4002B2ED10D9B01930E9B29
:1008C00002930F9B039330480AF08AFD9DED100AB6
:1008D000044630B340F2ED40B7EE001AFFEE000AD6
:1008E00029F01AFF2848234601AA04A90AF080FD2E
:1008F0000CE0099B04930A9B05930B9B069304A8A9
:100900000C9B07932CF00EFC0028CDD113B0BDEC4E
:10091000028B30BD062BD6D001211B480AF0FCFC0F
:10092000F4E7DFED1A0A4FF49E60B7EE001A29F0E3
:10093000F3FEF6EE000AB0EE408A29F0E9FDE8B9D0
:10094000B6EE000A124BB4EEC08AF1EE10FAD3F8FC
:10095000283D08DD38EE400A30EE008A93ED070AA4
:1009600028EE000ABEE730EE480AD3ED087A30EEF2
:10097000000AF0EEE77A27EEC00AB3E79FED030A1C
:10098000B0E700BF805C0020FC8000200000000079
:10099000806C00202DE9F0439DB0814608460EA9E9
:1009A000FEF7F4FE844BD3F8EC0003685B6A9847CB
:1009B00050B19DF86C30012B09D0DA1F022A06D9FC
:1009C0007E4801210AF0A8FC1DB0BDE8F083BDF807
:1009D0006840A20504F0070604F0380704F4E07547
:1009E00001D5002DF0D04FF00008CDF81480CDF8DF
:1009F0001880CDF81C803EBB9FED716A9DED107A8A
:100A0000DDED117ADDED0F6A27EE067A67EEC67A24
:100A100066EE866A083B012BCDED056A8DED067A00
:100A2000CDED077A04D8674806AA05A9FDF74AFD67
:100A30009DF86C30073B022B06D8634885F098FB85
:100A4000014605A82DF0DEF8CDF82080CDF82480F1
:100A5000CDF82880F7B9DDED147A129B0893F1EEFA
:100A6000677A139B099308A94846CDED0A7AFFF7E8
:100A70000BFD0028A4D09FED520A08A82DF0F6F82F
:100A80009DF86C30083B012B04D84E4809AA08A9F0
:100A9000FDF718FDCDF82C80CDF83080CDF83480EE
:100AA000EDB99FED476A9DED167ADDED177ADDED24
:100AB000156A9DF86C3027EE067A67EEC67A66EE08
:100AC000866A083B012BCDED0B6A8DED0C7ACDEDDE
:100AD0000D7A04D83B480CAA0BA9FDF7F3FC14F4DB
:100AE000806233D1DFED397A9DED180A9DF86C10E4
:100AF00020EE270ADFED327A0839012920EE270A95
:100B00008CBF0021012114F4006305BFDFED2F7AB3
:100B1000DDED190ADFED2E0A60EEA70A04BFDFED56
:100B2000287A60EEA70AAEB9002F35D1B3FA83F365
:100B3000B2FA82F25B0952090291019300920BAB67
:100B400008AA05A91D480AF055FD3DE79FED200ABA
:100B50000021D8E77FB9B3FA83F35B090120009342
:100B6000B2FA82F3CDE901105B0914480BAA08A977
:100B70000AF0D8FF28E7002D7FF422AF0120B3FA56
:100B800083F3B2FA82F2CDE900105B090B485209F7
:100B90000BA90AF06FFF17E7002D3FF411AFB3FA6E
:100BA00083F3B2FA82F2CDE900165B09520905A976
:100BB00002480AF0A1FD07E7805C0020FC800020CD
:100BC0000000C842802C002080790020E02E654281
:100BD000000000002DE9F047A2B08046084614A9A5
:100BE000FEF7D4FD7E4BD3F8EC0003685B6A9847B0
:100BF000C0B1BDF88040A30504F0070904F4E07714
:100C000000D57FB10CAE304618F02EF9B9F1000FC7
:100C100029D1DDE915012AF02FFE30B971480121F3
:100C20000AF07AFB22B0BDE8F0879DF8841009AA8B
:100C300040465BF0E9FC0028F0D0DDED177A9FED2F
:100C40006A7A099B009367EE877A10ADFDEEE77A2A
:100C5000DDE9151217EE903A284618F025F995E8C7
:100C60000F0086E80F00002514F0380A0695079556
:100C7000089514D1DDED1A7A189B0693F1EE677A88
:100C8000199B079306A94046CDED087AFFF7FCFBB8
:100C90000028C3D09FED540A06A82CF0E7FF099561
:100CA0000A950B959FB99FED506A9DED1C7ADDED7D
:100CB0001D7ADDED1B6A27EE067A67EEC67A66EED0
:100CC000866A8DED0A7ACDED096ACDED0B7A14F4C2
:100CD000806805BFDFED457A9DED1E0A9FED440A51
:100CE00020EE270A04BFDFED407A20EE270A14F435
:100CF000006405BFDFED3D7ADDED1F0ADFED3C0A44
:100D000060EEA70A04BFDFED387A60EEA70AB9F1FA
:100D1000000F31D1BAF1000F52D13046CDED050AA6
:100D20008DED040A18F0D0F803289DED040ADDEDDE
:100D3000050A3FF473AF10A93046CDED050A8DEDDD
:100D4000040A10951195129518F01EFA00283FF428
:100D500065AFB4FA84F46409B8FA88F3DDED050AE6
:100D60009DED040ACDF804A000945B0906AA10A921
:100D70001C480AF0AFFC55E7BAF1000F0FD1012370
:100D8000B4FA84F4CDE901A36409B8FA88F31548EC
:100D900000945B0909AA06A90AF0C4FE42E7002FE5
:100DA0007FF43CAF0123CDE90073B8FA88F2B4FABE
:100DB00084F30C485B09520909A90AF05BFE31E78C
:100DC000002F3FF42BAFB4FA84F3B8FA88F2CDF8D1
:100DD00000905B095209314602480AF053FD21E7B1
:100DE000805C0020FC8000200000C842E02E6542AC
:100DF0000000000010B44B7A8C7ACA7A43EA0423CC
:100E000043EA0243542B07D0562B09D0522B0BD167
:100E10005DF8044BFFF71CBD5DF8044BFFF7BABD4E
:100E20005DF8044BFFF7D6BE5DF8044B5CF0BCB830
:100E30002DE9F0432DED028B00F540590446D9F819
:100E4000EC00DFED4A8A036891B05B69984704F5CE
:100E500080470026002840F08480D7F8243DD3ED59
:100E6000DE7A93EDD88AFDEEE77A28EE288A17EE2F
:100E7000903A1DB204F5365801A940460EF0F4FF31
:100E800018B953F09FF83A4B01933722002102A87A
:100E9000B4F048FDA3238DF8083095238DF8093070
:100EA0008EF0B6F8D7F81C3DCDF80B00D9F810013C
:100EB000D3F8DC20D3F8E030CDF80F104430CDF873
:100EC0001320CDF8173054F0B1FC0346DFED290AAA
:100ED00093ED000AB7EE001A9F2029F01DFC10EEDA
:100EE000103AD9F81001CDF81B3003681B699847F8
:100EF00010EE103A04F59A49CDF81F3018EE103A6A
:100F00004846CDF8233085F037F920EE280A4046D0
:100F100010EE103ACDF82730D7F8CC3CCDF82B3076
:100F2000019BCDF82F300EF0C1FF10EE103A48466D
:100F3000CDF83330CDF83760ADF83B5085F028F967
:100F4000BDEEC00A372210EE103A02A904F57F6008
:100F5000ADF83D3052F088F911B0BDEC028BBDE820
:100F6000F08308EE106A002584E700BF0AD7233C0F
:100F70002292CA7F0000000010B500F58044D4F82A
:100F80001C0D7DF0E1FFD4F8241DD4F81C0DBDE844
:100F900010407EF03FB8000070B54FF48051044619
:100FA0000FF0AAF800284ED004F5804604F57F65BE
:100FB000D6F81C0D03689B689847692100F19402DC
:100FC000284651F0E9FFD6F81C0D0368DB68984706
:100FD0006A2100F19402284651F0DEFFD6F81C0D7C
:100FE00003681B6998476B2100F19402284651F071
:100FF000D3FFD6F8242D6C21284602F52A7251F031
:10100000CBFF202120460FF077F8E0B104F54053E4
:10101000D3F8EC0003681B69984778B1D6F8242D03
:10102000284690326E2151F0B7FFD6F8242D28467D
:10103000BC32BDE870406F2151F0AEBF20460BF0CE
:10104000DBFA0028EAD170BD08B512F007F8BDE858
:10105000084011F081BD00007FB50E464FF6FF71CC
:10106000044615460FF048F8E0B11022002168460A
:10107000B4F058FCA3238DF8003095238DF801308F
:1010800003238DF802308DF0C3FF1022CDF803004A
:10109000CDF8071004F57F6069468DF80B60039565
:1010A00052F062F904B070BD7FB50E464FF6FF7185
:1010B000044615460FF020F8E0B1102200216846E2
:1010C000B4F030FCA3238DF8003095238DF8013067
:1010D00004238DF802308DF09BFF1022CDF8030021
:1010E000CDF8071004F57F6069468DF80B60039515
:1010F00052F03AF904B070BD30B52DED048B87B0D5
:1011000004460D46182200216846B0EE409AF0EEE3
:10111000608AB0EE418AB4F005FCA3238DF800305C
:1011200095238DF8013006238DF802308DF070FF85
:101130001822CDF80300CDF8071004F57F6069464A
:101140008DF80B508DED039ACDED048A8DED058A57
:1011500052F08AF807B0BDEC048B30BD10B54FF4E7
:10116000801104460EF0C8FF30B104F595501030E0
:10117000BDE8104010F0DAB910BD00002DE9F043D1
:101180008FB01446054689463122002101A8DDE9C9
:1011900016769846B4F0C6FBA3238DF80430952349
:1011A0008DF8053008238DF806308DF031FF236867
:1011B000049363680593A36806933B68CDF81D30DC
:1011C0007B68CDF82130BB68CDF825303368CDF889
:1011D00029307368CDF80700CDF80B10CDF82D300D
:1011E0003122B3688DF80F9001A905F57F608DF865
:1011F0001C80CDF8313052F037F80FB0BDE8F083E5
:1012000070B52DED068B8CB0144605460E462C228B
:10121000002101A8B0EE409AF0EE608AB0EE418A5B
:10122000B0EE61AAF0EE429AB4F07CFBA3238DF8F5
:10123000043095238DF805300B238DF806308DF0A2
:10124000E7FEDFED1A7A94ED007ACDF8070027EE7D
:10125000277A29EE279A8DED077A94ED017ACDF859
:101260000B1027EE277A68EEA78A8DED087A94EDA9
:10127000027A8DF80F6028EE278A67EE277A2C22F3
:1012800001A905F57F608DED049ACDED058A8DED00
:10129000068ACDED097A8DED0AAACDED0B9A51F0B3
:1012A000E3FF0CB0BDEC068B70BD00BFE02E6542C5
:1012B000A020704730B5154B89B004466946D3F875
:1012C000100104F57F651E2285F0FEFF6A46104975
:1012D000284652F065F904F54053D3F8EC00036852
:1012E0001B68984704F50053014693F86822284686
:1012F00052F07AF904F59550103012F015F904F512
:10130000907020F045FC09B030BD00BF805C00202B
:10131000C2F80C082E4B2F4A70B54360002343617E
:101320008361C361C3632C4B426303644FF080420B
:101330002A4B43640446826358305DF09DF9284E81
:10134000284BA365A82560195DF04CFB665130352C
:10135000B5F56A7FF7D1244D04F56A705FF044F863
:10136000002104F2BC7088F09FFBC4F8705804F6AA
:101370007800A5F5BE6589F06DF89FED1C1ADFEDCC
:101380001C0A9FED1C0AC4F8085904F61C107EF0D4
:10139000CDFB9FED161A9FED180AF0EE410A04F6F8
:1013A00034107EF0C3FB9FED111A9FED130AF0EE8F
:1013B000410A04F64C107EF0B9FB20460F494BF071
:1013C000D1F920460E494BF0CDF9204670BD00BF43
:1013D000F03800200000C8410AD7233C0000E0405C
:1013E0002CF60C0840F60C080C84002000000000CD
:1013F0009A99993E0000B44300804A43A8E90C083A
:1014000028EC0C0870B54C4D4C49ADF50E7DD02242
:1014100006465AA8B4F03CFA0FCD0EAC0FC40FCD5F
:101420000FC40FCD0FC495E80F0084E80F0000240F
:101430005AAB18190021B7EE000A10344AF04EFEDC
:10144000D02CF5D13E4B0FCB02AC84E80F0001A9A4
:1014500020464AF0F7FD90B19DF90430DFED396A7E
:10146000E06807EE103AB8EEC77AF0EE007AE7EEE1
:10147000267AB7EE000A80EE270A4BF013FD00240F
:101480000EAB181900211034B7EE000A4AF026FE00
:10149000402CF5D12C49902236A8B4F0F9F900225D
:1014A000092136A84AF0C6FE96F9A469D6B9274D97
:1014B0000FCD1EAC0FC40FCD0FC40FCD0FC495E8D8
:1014C0000F0084E80F00324604211EA84AF0B2FE45
:1014D0009FED1F0A1F484BF0E5FC1F48B7EE000ABE
:1014E0004BF0E0FC1D4C9FED1E0A0FCC06AD0FC566
:1014F00094E80F0085E80F00002106A84AF0EEFDF1
:101500009FED170A002128464AF0E8FD04F110017A
:1015100060221EA8B4F0BCF900241EAB18190021EB
:10152000B7EE000A10344AF0D9FD602CF5D15EF018
:10153000E7FC0DF50E7D70BDB09B0C08E09A0C0821
:10154000F09B0C08CDCCCC3D009C0C08909C0C086A
:101550000000000090E80C089FE80C08D09C0C08E4
:10156000000034422DE9F04790B00DF106011D2036
:101570005EF0BAFD002800F09E809DF80630614ABA
:101580000133DBB211210BA88DF806308CF008FF77
:1015900000220DF107010BA84AF086FA9DF80630EB
:1015A000594A112105460BA88CF0FAFE00220DF1D4
:1015B00007010BA84AF078FA9DF80630534A11212A
:1015C00006460BA88CF0ECFE00220DF107010BA8DB
:1015D0004AF06AFA9DF806304D4A03F03F031121A4
:1015E00007460BA88CF0DCFE00220DF107010BA8CA
:1015F0004AF05AFA8046002D5DD0002E5BD0002FB5
:1016000059D0002857D028464AF066FC002852D10D
:1016100030464AF061FC00284DD138464AF05CFC67
:10162000002848D140464AF057FC002843D1394CA5
:1016300094E80F000DF10C0C10348CE80F0094E8C6
:101640000F000DF11C0989E80F0002A960464AF05D
:10165000F9FC98B3BDF8084002A948464AF0F2FCEC
:1016600000284AD0BDF8083054BB23B340F2E2440E
:101670009C420FFA84FA0FFA83F927D80DF10A0178
:101680003046ADF80A904BF003FF0DF10A012846F1
:10169000ADF80AA04BF0FCFE0DF10A013846ADF89A
:1016A0000AA04BF0F5FE00230DF10A014046ADF80B
:1016B0000A304BF007FF10B0BDE8F0870024CBE7FD
:1016C00040F2D662002B08BF1346D1E70DF10A01A4
:1016D0003046ADF80AA04BF0DBFE0DF10A012846BA
:1016E000ADF80A904BF0D4FE0DF10A013846ADF882
:1016F0000A904BF0CDFE0123D6E7002CDBD040F260
:10170000D663B5E7B0E80C08BCE80C08C8E80C08DC
:10171000D5E80C08509D0C0837B500F50A51782221
:101720002C31044650F06CF900220C2126484AF076
:1017300081FD2046FFF716FF0022B7EE000A0221C6
:1017400004F50B504AF0FEFD012504F505511F4A32
:1017500000950023103145204AF070FD1C4A1368A3
:10176000D90709D41B49156004F5035338330B60BE
:1017700004F585530833CB6004F50C50154902225B
:10178000203001254AF0ACFD134A0095002304F5F2
:101790007F61FD204AF052FD104B1A68D20705D434
:1017A0000F4A1D6004F58E54183414600C48012152
:1017B0004AF0B2FD4BF0DCF90A4A138843F001030A
:1017C000138003B030BD00BFE8E80C08A0560E0837
:1017D000E484002000220020249C0D08E8840020DE
:1017E000182200204C8700200F299DBF302303FBC7
:1017F0000100503000207047014B93F9F30270470D
:10180000804C0020024B93F8050100F00100704766
:10181000805C0020044BB3F8B832DB075ABF006984
:10182000C0F3401000207047804C0020014BD3F8DB
:10183000E00C7047804C002008B503689B6898470F
:1018400030B9044B93F90401B0FA80F0400908BDA7
:101850000020FCE7805C002038B50D1E2DDB174C06
:1018600094F8EC2CEBB29A4227D3D4F8E83C01224E
:10187000595DA4F5005004F0E3F8F0B15DF07CF898
:1018800003215EF0EFF8C0B95DF076F80D215EF04F
:10189000E9F890B994F9D832EB40DB075CBF94F9D2
:1018A000F212E940A4F5005048BF0221BDE83840DB
:1018B00058BF01F00101FCF7A1BC38BD804C0020ED
:1018C000022A10B50C4605D1BDE810400948352262
:1018D00004F0B6B8084BD3F8EC0003681B689847CF
:1018E000A04205D15DF048F8BDE810405CF0CEBFE5
:1018F00010BD00BF802C0020805C002029B102298F
:1019000007D1044BC3F8E4107047024B0122C3F81F
:10191000E4207047805C002031B1022907D1044BDC
:10192000012283F8E8207047014B83F8E8107047E4
:10193000805C002010B500F50053DFED186AD3F885
:10194000D82CD3F8D43CB2F90820B3F908309FED75
:10195000147A07EE902AF8EEE77A0446C7EEA60A54
:1019600000F595500121103007EE903AF8EEE77A35
:1019700060EE870A87EEA60A20EE070A11F00CFC3B
:1019800052F020FB262152F059FA04F53A50054A4C
:10199000BDE810400621383054F012BC0000C842A7
:1019A00035FA8E3CFCF30C0800F58042002382F8E7
:1019B000383D044A00F53A5013720621024A383085
:1019C00054F0FEBBBD86002008F40C0870B500F58D
:1019D0008045044695F8381D002957D02C4B2D4AD8
:1019E000D3F8EC00904204D1D3F8103193F8CB3007
:1019F00023B92046BDE87040FFF7D6BF264E95F8C4
:101A0000390D04F54053012293F9E0303272D0BB16
:101A1000002B3BDB85F8392D0139C9B204F50053A1
:101A200085F8381DD3F8D82CD3F8D43CB2F9082067
:101A3000DFED1A6AB3F908309FED197A07EE902AA4
:101A4000F8EEE77AB1FA81F1C7EEA60A04F59550EF
:101A50004909103007EE903AF8EEE77A60EE870A0F
:101A600087EEA60A20EE070A11F096FB95F8383D9E
:101A700063B904F53A5033720A4ABDE87040062152
:101A8000383054F09DBB002BC6DAB2E770BD00BF02
:101A9000805C0020E4820020BD86002000007A45A2
:101AA00035FA8E3C1CF40C086D2900F3E380012903
:101AB00001DC5DF001BE8B1E6B2BFAD80FF2040C1B
:101AC0005CF823F0D31C0108CD1C0108D31C0108CD
:101AD000D31C0108B31A0108D31C0108B31A01086A
:101AE000B31A0108CD1C0108B31A0108D31C010860
:101AF000CD1C0108CD1C0108B31A0108D31C010834
:101B0000D31C0108D31C0108B31A0108B31A010839
:101B1000CD1C0108D31C0108CD1C0108B31A010813
:101B2000CD1C0108CD1C0108B31A0108B31A010825
:101B3000B31A0108B31A0108B31A0108CD1C010831
:101B4000D31C0108B31A0108B31A0108B31A01081B
:101B5000D31C0108B31A0108CD1C0108B31A0108EF
:101B6000B31A0108D31C0108CD1C0108B31A0108DF
:101B7000B31A0108B31A0108D31C0108D31C0108C9
:101B8000D31C0108B31A0108B31A0108D31C0108B9
:101B9000B31A0108B31A0108D31C0108D31C0108A9
:101BA000D31C0108B31A0108B31A0108D31C010899
:101BB000D31C0108B31A0108B31A0108B31A0108AB
:101BC000B31A0108B31A0108B31A0108D31C01089B
:101BD000D31C0108D31C0108D31C0108D31C010825
:101BE000D31C0108B31A0108CD1C0108CD1C010843
:101BF000B31A0108B31A0108B31A0108B31A01088D
:101C0000B31A0108B31A0108D31C0108CD1C01083E
:101C1000B31A0108B31A0108B31A0108B31A01086C
:101C2000B31A0108B31A0108B31A0108B31A01085C
:101C3000B31A0108B31A0108B31A0108B31A01084C
:101C4000B31A0108B31A0108D31C0108B31A01081A
:101C5000B31A0108B31A0108B31A0108B31A01082C
:101C6000B31A0108B31A0108B31A0108B31A01081C
:101C7000CD1C0108A12921DC96297FF71AAFA1F11B
:101C800097030A2B3FF615AF0FF2040C5CF823F014
:101C9000D31C0108D31C0108B31A0108D31C010886
:101CA000B31A0108B31A0108B31A0108B31A0108DC
:101CB000CD1C0108CD1C0108D31C0108B42908D093
:101CC000DB2903D0B2297FF4F4AE704700235DF026
:101CD000C5BC704770B563298AB0034668DC01292A
:101CE00073DD881E612870D8DFE810F07C00840066
:101CF000940099006F00B3006F006F000C016F003B
:101D00006F008B001F016F000A013C0143016F004F
:101D10006F004B01520159016F006A0173016F009E
:101D20006F006F006F006F007C0189016F006F0012
:101D30006F008B016F006F006F006F008D016F00EF
:101D40006F006F006F006F006F006F006F006F001B
:101D500095016F006F004501470149016F006F0059
:101D60006F006F006F006F006F006F006F006F00FB
:101D70008F0191019301970199019B016F00BC01B3
:101D80009D016F006F006F006F006F006F006F00AC
:101D900001026F006F006F006F006F006F006F0037
:101DA0006F006F006F006F006F006F006F000D021B
:101DB000B22900F068810EDC9A2900F0B0819F29D9
:101DC00000F09D81982900F0A08118460AB0BDE876
:101DD00070405DF0AFB9B42900F0C680DB29F4D1C2
:101DE000012433E0022AFBD135220E21B04803F052
:101DF00027FEF5E7111E18BF0121AD48FCF7FEF9DB
:101E0000EEE7012A04D0022A14BF00210221F4E7E0
:101E10001146F2E706211846FFF752FDE0E7022AD5
:101E2000DED1A44DD5F8EC000368DB6A9847044680
:101E30000028D5D0A5F58053D3F8DC3CB3F90830A1
:101E4000002BCDD1A5F54050FFF774FD20460AB018
:101E500070BD022AC4D1974E974AD6F8EC10914231
:101E6000BED0D6F8102192F8CB20002AB8D006F5C3
:101E70008054A6F58056B4F9F82F2AB9D6F8DC3C80
:101E8000B3F90830002BABD01C22002103A805AD0C
:101E9000B3F048FD284616F0E7FFB4F9F83F93B9D0
:101EA0001623ADF80E30D4F8F43C8448642BB8BF48
:101EB000642303A906932CF02FFE20B152F082F880
:101EC000272151F0BBFF04F54F6494E80F0085E82B
:101ED0000F00D6F8DC3C7948B3F90830002BCCBFB2
:101EE0001023152303A9ADF80E302CF015FE0028A1
:101EF0003FF476AF52F066F8272151F09FFF6FE76D
:101F0000032188E7022A6E4D03D0002385F8F03CB8
:101F100066E71921A5F596504BF038FE04460028D7
:101F2000F3D0012385F8F03C90E7012A0BD0022A78
:101F300011D0002A7FF454AF614B83F81C2352F078
:101F400041F82B21D9E75E4B019283F81C2352F014
:101F500039F82C21D1E75A4B83F81C2352F032F880
:101F60002D21CAE70F2156E7564811468BF016FC83
:101F700036E709214FE704214DE705214BE71721FB
:101F800049E7901E414241414F4865F027FA27E753
:101F9000022A7FF425AF464801F062FB20E7012AC0
:101FA00006D0022A07D0002A7FF41AAF1146EBE7C9
:101FB00011460192E8E74448012165F00FFAEAE78B
:101FC000424B911ED3F81C3D4A424A4183F82020DF
:101FD00006E7931E594259413C4BD3F81C0D7EF045
:101FE000B1FEFDE6334B013A93F8E210012A8CBFB3
:101FF0000022012262F3041183F8E210F0E61121BD
:1020000009E7122107E7152105E7002103E7102161
:1020100001E70221FFE60121FDE61621FBE607218B
:10202000F9E60B21F7E6022A284B0ED1012483F8AA
:10203000E84E51F0C7FF4A2151F000FF5AF094FFDB
:10204000234A062154F0BCF800E7002283F8E82E6A
:1020500051F0B8FF4B2151F0F1FE5AF085FF1D4AB7
:10206000062121E0012A09D0022A0AD0002A7FF4A1
:10207000B7AE012118480DF02FFFB1E60192002103
:10208000F8E71146F6E75AB3022A7FF4A9AE094BE6
:10209000D3F8EC0003689B6F984700287FF4A0AE4C
:1020A0005AF062FF0D4A042154F08AF898E600BF06
:1020B000802C0020805C0020087C0020447C0020D4
:1020C000804C00201C7E0020107B0020806C0020B3
:1020D00034F40C0845F40C08005A002057F40C089E
:1020E000184BD3F8EC000368DB6F984778E6184686
:1020F0001146FFF703FC144804F054F870E611464B
:10210000FFF70AFC6CE61B2185E6022A7FF468AE25
:102110000E48FCF76BFE5AF027FF0D4AA0E7114668
:102120005CF0F2FE0B487BF05FFC044600283FF4B5
:1021300057AE044A92F8E33043F0020382F8E330EA
:1021400084E600BF805C00208C7B0020802C002077
:1021500070F40C08785A002010B50446044884F046
:1021600009F804F10801BDE8104029F003BB00BFE5
:102170008079002038B504462DED028B114883F09C
:10218000FFFF05462BF060FA0F48B0EE408A0DF0D5
:102190004FFF90B1DFED0D7AB4EEE78AF1EE10FA61
:1021A0000BDDD5ED000A95ED010AB1F0C5F9DFEDC3
:1021B000087A20EE270A84ED080ABDEC028B94ED24
:1021C000080A38BD80790020802C002000401C4681
:1021D000E02E6542074B93F9D902022805D0032867
:1021E00006D0003818BF0120704781F00100704709
:1021F00004207047804C002003688B4216D00429CD
:10220000C0E9001302D007290ED07047084B9FED9C
:10221000097A03F59663D3ED007AF8EEE77A67EE74
:10222000877AC0ED087A704700238362704700BF49
:10223000803C00200AD7233C08B50246FFF7CAFFBE
:10224000BDE8084001461046FFF7D6BF70B52DED3A
:10225000048B0446F0EE408AB0EE608A0D461646C6
:102260008CF0CEFE9FED329ADFED329AE06176B3CC
:10227000236843B9304B03F59663D3ED007AF8EE4B
:10228000E77AC4ED097A68EE898A002DB7EE000A74
:10229000FFEE007AB8BFB0EE670A68EE808AC4ED40
:1022A000058A264BB4EEE98AF1EE10FAD3F81C0D3C
:1022B00030DA7DF025FD20EE090A84ED060ABDEC3A
:1022C000048B20460321BDE87040FFF795BF94EDD5
:1022D000090A98EE890A28F0C9F9002D84ED050A4B
:1022E0000BDAB4EEE90AF1EE10FADADBDFED147A7C
:1022F00030EE670A84ED050AD3E7D2D0DFED117A1C
:10230000B4EEE70AF1EE10FACBD8DFED0D7A30EE3D
:10231000270AEFE77DF0F4FCB4EE480AF1EE10FA7C
:1023200048BFB0EE408A28EE098A84ED068AC6E7E7
:102330000000C84200000034803C0020806C002077
:1023400000A00C47000000B410B52DED028B044630
:10235000B0EE608AF0EE408A8CF052FEDFED090AA2
:10236000E06168EEA08A68EE200AC4ED098ABDEC3F
:10237000028BC4ED0A0A20460621BDE81040FFF793
:102380003BBF00BF0000C84210B52DED028B0446D4
:10239000B0EE408A8CF034FE94ED090ADFED097A44
:1023A000E061A8EE270A28F04BF9BDEC028B002370
:1023B00084ED090AA36220460621BDE81040FFF71C
:1023C0001BBF00BF0000C84270B54B68154D0646E4
:1023D0000C4673B98B6863B9C96851B91248FFF7E5
:1023E0002BFF95F8351E05F6BC50BDE870405FF038
:1023F00077BA95F8351E0D485FF012F948B906F125
:102400000801204616F0C0FE18B107480221FFF768
:10241000F3FE95F8351E05482246BDE870405FF092
:1024200053BA00BF806C0020EC8400203C7A00206E
:1024300008B50721FFF7E0FE80ED0A0A08BD00009D
:1024400008B50368032B23D1D0ED057A9FED127AEE
:10245000F0EEE77AF4EEC77AF1EE10FA1AD50F4BE8
:1024600090ED090A03F59663D3ED007AF8EEE77A6A
:1024700037EEC00A28F0FAF8DFED097AB0EEC00AAC
:10248000B4EEE70AF1EE10FA94BF0120002008BD77
:102490000120FCE70020FAE700000034803C002027
:1024A0000000484330B50368023B85B00446082B62
:1024B0006DD8DFE803F0050D30374B613F616100F7
:1024C000FFF74AFE84ED090A94ED090A05B030BD14
:1024D0008CF096FDE369DFED310AE061C31A07EE87
:1024E000903AF8EE677A94ED050A67EEA07AD4ED9B
:1024F000060AF12020EEA71A67EEE00A28F00CF990
:10250000D4ED057A77EEC07AC4ED057AD4ED097A78
:1025100037EE800AD6E7FFF72DFEDFED217A20EEB9
:10252000270ACFE71F4BD3ED4E7AF8EEE77AC0EDDE
:10253000097AC9E71C4DD5F8300D81F0B5FF0028A8
:10254000C2D0D5F8303D1B6B6362BDE78CF058FDFF
:10255000E3699FED127AD4ED0A6AE061C31A07EECF
:10256000903AF8EE677A67EE877A94ED097AA6EEEC
:10257000A77A84ED097AA7E70B4B9FED0C0AD3F8F5
:102580001C0D6C302BF01EFB84ED091A9CE7064BEA
:10259000D3F8243DD3F84433D6E700BF6F12833A13
:1025A0000000C842805C0020806C00209F0CB34576
:1025B0000368092B08D8DFE803F0050A05050505BF
:1025C000070705100023836290ED0A0A7047044B49
:1025D000D3F8243DD3F84833F5E7C36AF3E700BFE7
:1025E000806C0020F8B50023214FCB6297F80531AD
:1025F000204E13F0010F04460D462DD1D7F8EC0004
:1026000003685B6F984738B3D7F8EC0003F0CEFB54
:10261000DFED197A85ED0B0AB0EEC00AB4EEE70AD9
:10262000F1EE10FA03D409213046FFF7E5FD114819
:10263000FFF738FF0F4884ED000AFFF7B9FF336852
:1026400084ED010A0A2B0FD8DFE803F00C101010FC
:102650001010100C100C0C003368092BE7D1054842
:102660000021E2E70223A3602046F8BD0123FAE738
:10267000805C0020EC84002000000034034B012229
:102680001A6000229A60DA601A617047EC840020B8
:1026900013B501A904460DF067FB04F5804320B98A
:1026A000012283F8652E02B010BDDDED017ADFED69
:1026B000096A03F65862B8EEE77AD2ED007A67EE5F
:1026C000A67AB4EEE77AF1EE10FA54BF01220022A6
:1026D000E7E700BF0000C8422DE9F04F2DED068B63
:1026E00000F5005B00F595599BF92A338DB005463E
:1026F00000F5804409F1100933B100F54058D8F8CD
:10270000103193F8CB707FB90021A4F8DC1E484645
:1027100010F032FF94F8DD1E48460DB0BDEC068B7C
:10272000BDE8F04F10F032BF8CF06AFC0190D4F895
:10273000240D9FED948A90EDDBAA80F0D5F809AEC8
:10274000002800F0CA80D4F8243D03F55C7393E8B8
:10275000070086E8070030468DED0B8A2BF030FE2F
:10276000B0EE409A28460DF063FC05F59A4A002821
:1027700000F0B680504683F003FD07C886E80700E6
:1027800030468DED0B8A2BF01BFEF0EE409AD8F808
:10279000EC0003681B689847122840F0AA800023C9
:1027A00084F8DC3ED8F8EC0003685B69984728B1F0
:1027B000DBF8DC3CB3F90830002B0DDC98F9E03095
:1027C000002B09DA019BC4F8E03E504683F0D4FCAC
:1027D00004F6E46383ED000A94F8DC3E5BB1019BF0
:1027E000D4F8E00E181A41F28833984240F28F80F4
:1027F000002384F8DC3ED4F81C0D9FED630A6C3096
:102800002BF0E0F98DED090ACDED0A0A8DED0B1ADA
:1028100096E8070006AB03AE9FED5C0A83E807006D
:1028200086E8070030462BF0CDF92846B0EE408A06
:10283000F0EE608A8DED060ACDED070A8DED081ADF
:102840000DF0F6FB002874D0DFED517AF4EEE79A34
:10285000F1EE10FA94BF01250025D4F8240D80F084
:1028600043F830B1DFED4A7AB4EEE79AF1EE10FAB0
:1028700009D9002D64D1D8F8EC0003681B6898478B
:10288000022864D00027D4F8240D80F04FF90546C3
:10289000002873D0B5EEC0AAF1EE10FA6DD5DFEDC9
:1028A0003D7AB4EEE7AAF1EE10FAACBF012600269D
:1028B000504683F06DFC5EB9DFED377AB0EEC00AAA
:1028C000B4EEE70AF1EE10FA5AD8002D08BF00273F
:1028D00094F8DC1E84F8DD7E19E7B0EE489A41E7F3
:1028E00028460DF075FB00287FF444AFDFED259AF4
:1028F0004DE7D8F8103193F8CB30002B3FF452AFAE
:1029000098F9E030002BBFF64DAF012348E7504661
:1029100083F032FC04F6E463D3ED007A30EE670A0C
:10292000DFED1E7AB4EEE70AF1EE10FA3FF760AF82
:1029300061E728460DF04CFB0546002884D18CE762
:10294000D4F8240D7FF0D0FF002894D19BE7B0EE9F
:10295000680AB0F09FFBF0EE408AB0EE480AB0F093
:1029600099FBDFED0F7A20EE280AB4EEE70AF1EECC
:1029700010FACCBF0127002785E700252E4697E7F0
:102980003746A5E7000000009F0CB345D302373956
:102990000000FA420000C8C2000070420000484235
:1029A00055CF7D3F38B504460DF042FB04F59555F3
:1029B000103548B920460DF00BFB014620B92846DA
:1029C000BDE8384010F024B804F54054D4F8EC00C9
:1029D00003689B6C984720B9D4F8EC000368DB6C63
:1029E00098470146EBE7000030B5044689B06846D9
:1029F00004F5955516F038FA103504A816F034FA97
:102A00006946284610F0BEF898B104A9284610F08F
:102A100009F970B1059B019323680022DB6C6946BC
:102A20002046984728B104F52B5001211C3087F02F
:102A300007FB09B030BD000000F5805292F82C254C
:102A4000D2070BD400F54052D2F8102192F8CB10E7
:102A500009B1FFF7C9BF03689B6C184770470000B6
:102A600030B587B0044602A8019116F0FDF904F5CF
:102A7000955002A9103010F085F8019A18B9002578
:102A8000284607B030BD236802A9DB6C2046984772
:102A900005460028F3D004F52B5001211C3087F0A7
:102AA000CFFAEDE7F0B5044685B004F595566846D3
:102AB00010360F46154616F0D7F96946304610F025
:102AC000B1F810B9002005B0F0BD394630460FF01E
:102AD00011FF0028F6D0002DF5D004F580542846CB
:102AE00094F82C3543F0020384F82C35EBE7000012
:102AF0002DE9F04F2DED0A8BBDB0044624220D4682
:102B000018A80021B2F00EFF2422002121A8B2F063
:102B100009FF242200212AA8B2F004FF04F5405640
:102B20002422002133A8B2F0FDFE0023CDE90D33AD
:102B30000F9396F8E13013F0080839D104F50059E5
:102B400043F0080399F8D02C079286F8E13017F08B
:102B5000E3FA90F9213003B390F84033EBB104F27B
:102B60008457384617F0E8F9C34694F8A6355FFA5B
:102B70008BF18B421FD9384617F0BCF90BF1010BD2
:102B800082460028F1D1C94A0221284656F00CFE9F
:102B900096F8E1306AF3C30308E0C54A02212846EB
:102BA00056F002FE96F8E1306FF3C30386F8E13089
:102BB0004FF001083EE304F537533833012118463E
:102BC0000BEE903AFAF7F6FF824608B9B94ADBE70E
:102BD00020460CF04FFFD9F8DC3CB3F908A0BAF15D
:102BE000000F01D0B44AD9E796F9E030002B01DBA1
:102BF000B24AC9E7204601F0AFFE04F544533C3326
:102C0000184652460CA90CEE103A13F057FA002859
:102C100014BF022301230393F123CDE9133A8F213B
:102C20000A23CDE9003113AA287CADF854A0032370
:102C30004D2154F0F9FAA24B9FEDA28A01225A725B
:102C40000621A14A284656F0AFFD039B022B0CBF7C
:102C50009E4A9F4A062128464FF0000A56F0A4FDDE
:102C600089F8E6A25146384617F0B0F894F8A63530
:102C70005FFA8AF18B420CD913AA38468DED138A7C
:102C80008DED148A8DED158A0AF1010A16F020FFE8
:102C9000ECE7384617F050F94FF0000A4FF07C0B84
:102CA00094F8A6255FFA8AF94A4519D94946384663
:102CB00016F000FEC0B20BFB00403CAA0C2300F251
:102CC000146003FB092C07C8ACF1900C8CE80700DA
:102CD0003CAA02EB890909ED2F8A0AF1010ADFE714
:102CE00041F288310AA823F0FBFFD6F810019FEDCE
:102CF000759A03689FED77AA9B6ADFED77AA9847DC
:102D0000D6F81001012184F0E3F9744B1B6802939B
:102D1000D86A036801211B6898478CF071F9059007
:102D20008CF06EF9F0EE499A0690002604F50059F1
:102D3000079A99F8D03C934240F0D88094F8C6188E
:102D4000384617F0D7F8002800F0D08004F5405B33
:102D5000DBF8103193F8CB300493002B00F0C680E1
:102D600041F288310BA823F0BBFF8CF049F9059B99
:102D7000C01A132840F2D9808CF042F90590204601
:102D80000CF078FE5DF058FC82465DF0EBFBD9F864
:102D9000DC3CDBF81001B3F9083000EE103AB8EE75
:102DA000C00A20EE0A0A85F005FE50465DF0E2FBFF
:102DB000384617F0C1F81CEE100A13F09BFBD9F847
:102DC000DC3CDFED400AB3F9083000EE103AB8EE13
:102DD000C00AA22020EE0A0AB7EE001A27F09CFCD7
:102DE000B4EEE90AF1EE10FA1CEE100A4FF0000200
:102DF0000CA958BFF0EE409AF0EE408A13F05EF94D
:102E000008B900230C939DED0C8ADFED357AB4EE02
:102E1000498AF1EE10FAF4EEE78A48BFB0EE498A2B
:102E2000F1EE10FA80F28F809FED2E9ADFED2E8A60
:102E30004FF0000A94F8A6355FFA8AFB5B4540F232
:102E400096814FF00C0918AB09FB0BF903EB090055
:102E5000B0EE490A2AF0B6FE59463846CDED110AC1
:102E60008DED121A8DED100A16F024FD7C23C0B2F0
:102E700003FB0040B0EE680A00F214602AF0A2FEE4
:102E80003CAB13A910A899448DED130ACDED140A9B
:102E90008DED151A2AF06AFE0AF1010A09ED240ADD
:102EA00049ED230A09ED221AC4E700BF6DF60C08AC
:102EB0005CF60C08DF0C0D087BF60C088DF60C0890
:102EC000BD8600200000000098F60C08ADF60C0846
:102ED0006F9F0C086F12833A0000C842E084002004
:102EE00000000034A4707D3F0AD7233C04F540590C
:102EF000D9F8100103689B6A9847D9F8100100219E
:102F000084F0E6F8029BD86A036800211B689847A2
:102F1000002E40F05F812846C94A052156F044FC46
:102F20003146384616F052FF70E1029B986A0368FA
:102F300005215B6898470BA823F0DEFEB0EE498AB6
:102F4000B0EE489AF2E64FF000094FF00C0B04F592
:102F5000B86A94F8A6255FFA89F39A4222D91946ED
:102F60003846089316F0A6FC089B0BFB03F13CAB1C
:102F70005A18A2F16C034FF07C0CC0B2CDE90832B4
:102F80000CFB00A018AB194454302AF005FE089B36
:102F9000099A09F1010902ED1B0AC3ED010A83ED4B
:102FA000021AD6E7039B012B4FF0000A46D19FED92
:102FB000A5BA9FEDA59A4FF00C0B94F8A6355FFAD1
:102FC0008AF6B34240F286800BFB06F63CAB03EB7D
:102FD0000609A9F14803089321ABB0EE680A9819D5
:102FE0002AF000FE089B09ED120AC3ED010A83EDE9
:102FF000021A33ABB0EE4B0A98192AF0E3FD2AAB64
:1030000098198DED100AB0EE490ACDED110A8DED3B
:10301000121A2AF0D7FD13A910A88DED130ACDEDD1
:10302000140A8DED151A2AF0B7FD0AF1010A09ED0F
:10303000090A49ED080A09ED071ABEE79FED819AD2
:103040009FED81BAF0EE088A94F8A6355FFA8AF906
:103050004B4564D99DED0C0AB4EEE80AF1EE10FA86
:1030600035DB0C2303FB09F93CAB03EB090621AB71
:1030700003EB09002AF0B6FD33AB46ED110A06ED6D
:10308000101A06ED120A03EB0900B0EE490A2AF005
:1030900099FD2AAB03EB09008DED100AB0EE4B0A47
:1030A000CDED110A8DED121A2AF08CFD13A910A88E
:1030B0008DED130ACDED140A8DED151A2AF06CFD75
:1030C00006ED090A46ED080A06ED071A049E0AF104
:1030D000010AB9E74FF000094FF00C0A94F8A63541
:1030E0005FFA89F6B34241D933AB0AFB06302BF0C5
:1030F00067F91BEE900AF0EE408A7AF071FC07EE59
:10310000900AB8EE677A3CABC8EE877A03EB860686
:1031100009F1010967EEAA7A46ED2F7ADEE74FF052
:10312000000A4FF00C0B94F8A6355FFA8AF94B456C
:103130001DD933AB0BFB09302BF042F9C8EE297ACD
:103140000AF1010A1BEE900A67EE808A7AF048FCC9
:1031500007EE900AB8EE677A3CABC8EE877A03EBCD
:10316000890967EEAA7A49ED2F7ADCE7049E8BF095
:1031700047FF069BC01AB0F5FA7F27D98BF040FFB6
:1031800004F50053DDED0D7AD3F8DC3C0C9A1B8975
:103190001392FCEEE77A339A1492ADF85C30349ACD
:1031A000159217EE903A359A1692ADF85E30F022ED
:1031B0001423CDE90032B121069013AA287C54F0E3
:1031C00033F874F005FC297C74F0F4FA0BA823F0B2
:1031D00093FDB5E60399384616F0F8FD00264FF04A
:1031E0000C0A94F8A635F1B28B4207D933AB0AFB2F
:1031F0000132384616F06CFC0136F2E7384616F01C
:1032000079FC124A0621284656F0CEFA104B0025CA
:1032100020465D7201F092FB04F50B50263049F018
:1032200077FB99F8E13065F3C30389F8E1300AA828
:1032300023F062FD40463DB0BDEC0A8BBDE8F08F47
:10324000A1A70E08A4707D3F0AD7233CB5F60C0851
:10325000BD860020F0B5534FD7F8983CDA0785B00B
:10326000044600F19C8000F54055D5F8103193F8E4
:10327000C120002A40F0938093F8CB30002B00F05F
:103280008B8095F9E030002BC0F2868000F58046F7
:1032900096F8E83E002B40F08280D6F81C0D9FED9A
:1032A000420A6C302AF08EFCCDED020A60EEA00AD4
:1032B000DFED3E7A8DED010AE0EE000A8DED031A96
:1032C000F4EEE70AF1EE10FA66DCD6F81C3D9FED4D
:1032D000387AD3ED377AF4EEC77AF1EE10FA04D5E6
:1032E000D5F810311B7A002B56D0B5EE007AF4EEEB
:1032F000C77AF1EE10FA4FD404F59A4082F048FFF5
:10330000DFED2C7AB4EEE70AF1EE10FA44D8D6F8E5
:103310001C3D9FED297AD3ED367A67EE877AB3EEBE
:103320000E7AF4EEC77AF1EE10FA35DA234AB4F9E0
:10333000A410138801339BB2138019B9B4F8A210FA
:10334000A4F8A410B4F8A410994228D80026168036
:1033500050F038FE0122192150F090FDD5F81001EF
:1033600003685B699847431C04F53A50144A314698
:10337000383052F025FFD5F81031012283F8C120F2
:10338000D7F8983C5B070AD504F58550083005B09E
:10339000BDE8F04068F01EB9084B00221A8005B065
:1033A000F0BD00BF804C00209F0CB3454054094A3B
:1033B0006666663F000000B4E02E65422685002068
:1033C000CCF60C0870B52DED028B4A4BD3F8983C27
:1033D0009B0784B004461FD400F58045DFED468A84
:1033E000D5F81C0D03681B699847D0ED017AF4EEFF
:1033F000E87AF1EE10FA0FDB04F5405304F59D4630
:10340000D3F8102192F8C1106C3649B1002303A9FA
:103410003046039352F00CFA04B0BDEC028B70BD41
:1034200092F8CB20002AF1D093F9E030002BEDDBAD
:1034300095F8E83E002BE9D1D5F81C0D03681B690F
:103440009847D0F8A430D5F81C0D039303681B6986
:10345000984704F58C7200F1A401304652F0E6FA68
:10346000DDED037AB0EEC08AF0EEE77AF4EEC87ACA
:10347000F1EE10FA03D503A9304652F0D9F9D5F888
:103480001C0D03681B699847D0ED040AF4EEE80AA6
:10349000F1EE10FAC0DBF6EE087A60EEA77AF4EEF1
:1034A000C87AF1EE10FA1DD58BF0AAFDD5F8F83EDA
:1034B00042F21072C31A9342AED9DFED107AC5F80A
:1034C000F80E68EE277A04F53A5417EE900AF9F7E9
:1034D0001BF83834CDE90001094A0021204652F09A
:1034E0006FFE99E79DED030A27F012F80028DBD163
:1034F00092E700BF804C0020000000340000C8426A
:10350000E8F60C0810B5044600F59D40103063F055
:1035100077FF04F59D400121BDE8104030306CF08C
:103520003BBA0000F8B500F58045044695F9903E99
:1035300043B300F5405695F8A42E96F8E030DB43EF
:10354000C3F3C01363F3C30285F8A42E00F59D47AF
:1035500000F59A4082F01CFEDFED3D7A103720EE38
:10356000670A384663F0CCFF95F8E83E53B9384611
:1035700063F072FFD6F8103193F8CB301BB9354B9E
:1035800000221A80F8BD95F8A43EDB07FAD4D6F8DD
:10359000EC0003689B6B98470028F0D096F9E03068
:1035A000002BECDB2B4E33884BB9B5F9963E33B18B
:1035B000642213FB02F3D5F8F42C9A42E2DB38467E
:1035C00063F0BAFFD5F81C3D9FED237AD3ED367A30
:1035D00067EE877AB3EE0E7AF4EEC77AF1EE10FA60
:1035E00005D83388002BCDD0013B3380CAE7B4F92E
:1035F000A4301BB9B4F8A230A4F8A4303388B4F8CE
:10360000A420B4F9A400154993423CBF0133338090
:103610003388D5F8CC2C012B01D10A60B2E70968B8
:103620009142ACDD18B9B4F8A220A4F8A420B4F8F3
:10363000A4209A42A6D80023338050F0C3FC022273
:103640000C2150F01BFC2046BDE8F840FFF75ABFA4
:103650000AD7233C24850020E02E654220850020E7
:1036600008B500F5804292F9903E6BB300F54053E7
:1036700093F9E030002B0EDA00F53A50134A062198
:10368000383052F09DFD50F09DFC0322BDE808400B
:103690000F2150F0F3BBB2F9963E8BB1D2F8F42C67
:1036A000642113FB01F39A420ADA00F53A50084A02
:1036B0000121383052F084FD50F084FC0222E5E70D
:1036C000BDE80840FFF71EBF08BD00BF00F70C08AB
:1036D00012F70C08F0B52DED028B00F540555C4E4D
:1036E000D5F8103193F8CB308DB0044643B195F93D
:1036F000E030002B04DB00F5005393F902332BB9C3
:10370000002333800DB0BDEC028BF0BD00F5804787
:1037100097F8E83E002BF3D101F084FB00287DD11F
:10372000D5F8EC0003689B6B98470028E8D004F5B7
:103730009940503052F0D2F82AF042FEF0EE087A6A
:10374000B4EEE70AF1EE10FAF0EE408AD8DA04F5AA
:10375000805303F59F6203F2FC43D3ED007A92EDB0
:10376000000A20EE270AAFF07FFEDFED3A7A20EE66
:10377000270AB2EE0E7AB4EEC70AF1EE10FABFD9FC
:10378000D7F81C3D93ED368A28EE278AF3EE0E7AA1
:10379000B4EEE78AF1EE10FAB2D904F595500023A1
:1037A00009A9103009930A930B930FF047FA0028E8
:1037B0003DD13388B4F9A42001339BB23380002A71
:1037C00040D0B4F8A420B3EB420F9BDB50F0FAFBDF
:1037D00001220C2150F052FB1F4B002218EE900AE0
:1037E000CDE90623F8F790FE1C4BCDE90401002239
:1037F00018EE100ACDE90223F8F786FE04F53A54D4
:103800003834CDE90001164A2046002152F0D8FC98
:1038100001220C211348FAF7E5FB73E7D5F8EC0019
:103820000368DB6C984700287FF47AAF68E709A843
:103830002AF0C6FDF2EE047AB4EEE70AF1EE10FAD1
:10384000B7DB5DE7B4F8A220A4F8A420B9E700BF75
:103850001C850020E02E65420000084000003E402C
:1038600028F70C08785A0020F0B52DED028B8BB0AC
:10387000002307930893099305AB0446019300F5D1
:10388000955007AB009302AA04AB03A910300FF0C8
:10389000EDF804F50056054686F8AC0E28B900256B
:1038A00028460BB0BDEC028BF0BD8BF09DFBD6F82B
:1038B000B03E9FED327AC31A07EE903AF8EE677A7F
:1038C000074667EE877A04F53A5006AA02A908303F
:1038D000CDED067A52F0AAF804F53A5006AA03A9EB
:1038E00014308DED020A52F0A1F804F53A5006AA00
:1038F00004A920308DED030A52F098F896EDC18AA4
:10390000C6F8B07EB5EEC08AF1EE10FAC7D9DDED8B
:10391000080A9DED070AAFF043FCDDED090AAFF0A0
:103920003FFCD6F8302EDDED037AB4EEC08AF1EE1E
:1039300010FA94BF012300231AB196F8342ED2074F
:1039400012D438EE087AB4EEE77AF1EE10FA0BD81A
:103950000233DBB2DDED027AB4EEE78AF1EE10FA63
:1039600009D8002B9BD09BE7B4EEE78AF1EE10FA62
:10397000F0D80133EDE7012B92D890E7BD378635BB
:1039800070B500F54055044695F8053143F0040341
:1039900085F8053150F016FB0122112150F06EFA26
:1039A000D5F8103193F8CB30002B43D0D5F8EC008C
:1039B00003681B68984709280AD1204608F01CFEB6
:1039C00030B104F5A9404030BDE8704008F0FCBDBE
:1039D000194BD3F8EC0003681B69984704F50053B2
:1039E00040B993F90133032B24D10621204608F076
:1039F000EFFD0DE093F901130229F6D195F8053199
:103A0000DB07F2D40622204602F01AF80028ECD098
:103A10000A4BD5F8EC0001225A7303681B6C9847D7
:103A2000034604F53A50064ABDE87040022138309A
:103A300052F0C6BB70BD00BF805C0020BD86002078
:103A40005CF70C0808B500F5405292F805315907AB
:103A500017D56FF3820382F805310A4B5A7B42B1C6
:103A6000002200F53A505A730221074A383052F0CA
:103A7000A7FB50F0A7FABDE808400022112150F042
:103A8000FDB908BDBD86002080F70C08F0B50546DD
:103A900085B005F595576846103715F0E5F9694684
:103AA00038460FF0BFF880B105F50053D3EDC17A69
:103AB000374CF5EEC07AF1EE10FA08D8354A0023FB
:103AC00028462380D373FFF7BDFF05B0F0BD28461D
:103AD000FFF7CAFE064628460CF07AFA10B92846C7
:103AE0000CF052FAA378002E18BF00200343DBB27B
:103AF000A370002BE9D06378A8BB83BB2378013384
:103B0000DBB2082B237003D14EB338460FF01AF8FE
:103B10002378092B02D138460FF00CF82378092BB3
:103B20001DD94FF48573238050F04CFA02221021E6
:103B300050F0A4F98BF064FA6368C01A47F230536E
:103B4000984209D905F53A50134A0221383052F00B
:103B500037FB8BF055FA60602846FFF711FF0D4BDD
:103B60006278DA73B1E72678002EF8D0013EF6B21B
:103B70002670002BF3D0002EF1D1667050F022FA9F
:103B80003246102150F07AF92846FFF75BFFE6E74E
:103B900028850020BD86002098F70C0800F54053CA
:103BA00093F805315B0701D5FFF7EABE70470000C7
:103BB00073B5044600F5955001A9103004F5005581
:103BC0000EF09EFDD5F8743E834206460CD004F5F7
:103BD0008043D3F81C0D7DF057FCC5F8746E50F08F
:103BE000F1F93E2150F02AF904F5805695F9781E36
:103BF00096F9C02596F8C03591421BD0FF2B19D0FD
:103C000004F58043D3F81C0D7DF03EFC96F8C035DA
:103C100085F8783E50F0D6F995F8782E182150F0B6
:103C20002DF904F53A5095F9783E034A04213830CD
:103C300052F0C6FA02B070BDA8F70C082DE9F043A7
:103C40008FB005468BF0DCF90023059306930793AC
:103C5000089309930A930B930C930D9305F59558CC
:103C600004AB019308F1100803AB009306460BABBD
:103C700008AA05A940460EF0D9FEDFED487A9DED71
:103C8000077AB4EEE77AF1EE10FA074632DB9DEDE3
:103C90000A7AB4EEE77AF1EE10FAACBF0124002400
:103CA00005F50059404699F8AC3E002B08BF0027A7
:103CB0000EF0CEFE8046FFB9444699F9343C012B04
:103CC0002BD174B105F54053D3F8102192F8CB40B5
:103CD0003CB1D3F8EC0003685B69984780F00100C1
:103CE000C4B299F87C3ECBBBCCB9C9F8806E0FB09A
:103CF000BDE8F0830024D3E7002CDDD005F53A5071
:103D0000143051F093FD90ED007AF7EE007AB4EEA6
:103D1000E77AF1EE10FAD0DCCEE70024E1E7D9F83B
:103D2000800E301AB0F57A7FE1D9C9F8843E0124BB
:103D300005F5804389F87C4ED3F8243D83F80C4484
:103D400050F040F922461D2150F098F8144A05F52C
:103D50003A500221383052F033FAC8E714B1C9F8AA
:103D6000846EC4E7D9F8840E43F69823361A9E422F
:103D7000BDD905F58043C9F8804E89F87C4ED3F84B
:103D8000243D83F80C44C9F8844E50F01BF92246B8
:103D90001D2150F073F8034AD9E700BF000000343A
:103DA000C0F70C08DAF70C080B4B10B501220446DB
:103DB0005A728BF025F904F58042D2F8D43EC31A2A
:103DC000142B07D9C2F8D40E04F59350BDE8104067
:103DD00044F0E2BF10BD00BFBD8600202DE9F743CF
:103DE000044604F5405600F50B5000233C300DF11D
:103DF00007018DF8073049F0F9FAD6F8100190F96B
:103E0000C030026883B3083BDBB2012B95692BD924
:103E10003221A84704F1100012F0E6FC204B04F513
:103E20003A581F684FF0000908F13808F86A03682B
:103E3000DB69984701281ED18BF0E2F841F2873305
:103E4000A0EB09029A42054605D9164A06214046CA
:103E500052F0B6F9A9462046FFF7A6FFB86A0368F4
:103E600003215B689847E1E704F500539269B3F8D2
:103E700010139047CEE70121D6F8100183F028F9FE
:103E8000D6F810010368DB6A98475BF0D3FFF86A45
:103E900003681B68012103B0BDE8F043184700BF69
:103EA000E0840020F8F70C0870B5044600F53A509D
:103EB0002DED028B184A194E9FED198A06213830D4
:103EC00052F07EF92046FFF789FF2046FFF76CFF8E
:103ED00020460BF0CFFD3368986A036803215B68C6
:103EE00098475CF0A9FB05465CF03CFB04F50053E9
:103EF000D3F8DC3CB3F9083000EE103A04F5405337
:103F0000B8EEC00AD3F8100120EE080A84F052FD82
:103F100028465CF02FFBD8E71CF80C08E084002052
:103F20006F12833A2DE9F047044600F53A502DED23
:103F3000028B2A4ADFF8AC900621383052F040F963
:103F40002046FFF74BFF5CF077FB04F54056054633
:103F50005CF008FBB7EE000AD6F8100184F02AFDE9
:103F600028465CF007FB8BF04BF841F2873A074696
:103F70008BF046F8C01B5045D9F8008017D99FED4B
:103F8000188A28465CF0EEFAB0EE480AD6F810011E
:103F900084F010FD28465CF0EDFA2046FFF704FFA0
:103FA000D8F82800036803215B689847E9E72846AA
:103FB0005CF0D8FAB7EE000AD6F8100184F0FAFCEB
:103FC00028465CF0D7FA2046FFF7EEFED8F8280026
:103FD000036803215B689847CAE700BF4CF80C08E8
:103FE00000000000E0840020F7B500F540530446CF
:103FF000D3F8103193F9C030032B2BD0364E652502
:1040000000F58047013D15F0FF050CD0D7F8D03EF4
:104010004BB93368986A036814215B689847204657
:104020000BF028FDEEE704F5375001213830F9F7A1
:10403000C1FD04F5005378B993F9FC3253B1092B53
:1040400008D08DF8070004F50B500DF107013C3046
:1040500049F0CCF903B0F0BD93F9FC22032A34D81F
:10406000DFE802F002252D30D3F8DC3CB3F908205C
:1040700040F2B5339A422ADD04F50B5001250DF1CB
:1040800007013C308DF8075049F0B0F904F53A507B
:10409000124A0221383052F093F8114B5D720E4BE8
:1040A0001C68A06A036805215B689847F9E7D3F8A4
:1040B000DC3CB3F9082040F2B5339A4207DD2046D4
:1040C000FFF7F2FE2046FFF72DFF092AC2D000239A
:1040D0008DF80730B7E700BFE084002070F80C08C7
:1040E000BD86002000F53A500B46024A04213830C4
:1040F00052F066B890F80C0810B504464FF062FF15
:10410000002205214FF0BAFE04F53A50034ABDE8FB
:1041100010400421383052F053B800BF9CF80C080E
:1041200013B50B464AB100F53A5000920421054AF6
:10413000383052F045F802B010BD02B0BDE8104072
:10414000FFF7D0BFB4F80C0808B500F53A50064A9E
:104150000421383052F034F84FF034FFBDE8084005
:10416000002208214FF08ABEC8F80C0838B5044672
:104170000D468AF045FF04F540533DB9D3F8FC20C5
:10418000C3F800010AB9C3F8FC0038BDD3F8002118
:10419000801A642884BF0022C3E93F22F5E70000AB
:1041A00037B5044600F59A4081F0D8FF04F5405237
:1041B000C0F3803592F8E230C3F34001A9421DD02C
:1041C00065F3410304F53A5482F8E23038346DB1B6
:1041D0004FF0F8FE02220B214FF050FE084A022158
:1041E000204603B0BDE8304051F0EABF4FF0EAFE90
:1041F0002A460B214FF042FE024AF0E703B030BDE1
:10420000E0F80C08FCF80C0838B50A460C46062104
:10421000054601F015FC28B1054A137843F0080360
:10422000137038BD21462846BDE8384008F0D0B9A3
:10423000DC86002038B50A460D461521044601F0FB
:10424000FFFB28B1094A137843F00803137038BD07
:1042500004F53A5004213830054A51F0B1FF29469F
:104260002046BDE8384008F0B3B900BFDC86002026
:104270000CF90C0838B50A460D461521044601F024
:10428000DFFB28B1094A137843F00803137038BDE7
:1042900004F53A5004213830054A51F091FF29467F
:1042A0002046BDE83840FFF7AFBF00BFDC860020E6
:1042B00034F90C0838B50A460D461B21044601F0B6
:1042C000BFFB28B1094A137843F00803137038BDC7
:1042D00004F53A5004213830054A51F071FF29465F
:1042E0002046BDE83840FFF78FBF00BFDC860020C6
:1042F0004AF90C0838B50A460D461121044601F06A
:104300009FFB28B1094A137843F00803137038BDA6
:1043100004F53A5004213830054A51F051FF29463E
:104320002046BDE8384008F053B900BFDC860020C5
:104330005CF90C0810B500F5405494F8E2309A0688
:1043400023D4D4F8EC0003681B689847032808D0EE
:1043500005D802280ED194F8E000C00914E01B280B
:10436000F9D194F8E00000F0A000A0F180035842D9
:10437000584109E0B4F8E00020F4FE4020F07F004E
:1043800080B2003818BF012010BD0120FCE70000FA
:1043900038B500F54055044695F80531184A43F004
:1043A000080300F53A5085F805310221383051F004
:1043B00007FF4FF007FE012217214FF05FFD204657
:1043C000FFF7B8FF40B104F537500122BDE838408F
:1043D00015213830F9F706BED5F8EC0003681B68E4
:1043E0009847062806D104F5AB405830BDE8384060
:1043F00009F0FABA20460B21BDE83840FFF704BFA8
:1044000070F90C0870B500F54055D5E93F239B1AAB
:1044100041F288329342064611D9D5F8EC00036880
:104420001B6D9847044695F80531C3F3C003A342BA
:1044300013D034B13046BDE87040FFF7A9BF002467
:10444000F1E74FF0BFFD224617214FF017FD95F819
:10445000053164F3C30385F8053170BD0B4610B513
:1044600011460446072B07D8DFE803F02A04131689
:10447000191C242708F0ACF804F50053D3F8383C95
:104480009B061DD504F585500830BDE8104067F047
:10449000A1B8FFF7B9FEEFE7FFF7ECFEECE7FFF797
:1044A000C9FEE9E700F53750012214213830F9F749
:1044B00099FDE1E7FFF7FEFEDEE7FFF71BFFDBE715
:1044C00010BD0000F8B5044604F500574FF07AFD22
:1044D000012205214FF0D2FC97F8E632072B98BF56
:1044E000304A204694BFD55C0125FFF723FF68B111
:1044F0002D4A2E492046FFF713FE04F537500122BE
:1045000010213830F9F76EFD002514E004F540560F
:10451000D6F8EC000368DB6C984798B196F8AD3696
:1045200083B196F9AC36012B0CDC214A2149204697
:10453000FFF7F6FD0125294620460322BDE8F84095
:10454000FFF78CBFD6F8EC000368DB6C984718B116
:10455000D7F8383C190715D4D6F8EC0003681B6867
:104560009847032803D1D7F8383CDA070DD4D6F89A
:10457000EC0003685B6A984768B90C492046FFF76E
:10458000B1FDD8E70A4A0949D1E70B4A0749204655
:10459000FFF7C6FDB8E7D7F8383C5B07EDD5074A0B
:1045A000F4E700BF50FA0C0890F90C0866CA0D0831
:1045B0009AF90C08ADF90C08BDF90C08CDF90C08F6
:1045C00038B5044615464FF0FDFC012206214FF098
:1045D00055FC2046FFF7AEFE98B104F53750012296
:1045E00007213830F9F7FEFC144A15492046FFF739
:1045F00097FD0025294620460422BDE83840FFF7F4
:104600002DBF04F54053EDB2D3F8EC000368DB6C2A
:10461000984768B104F50053D3F8383C1B0707D519
:1046200035B1084A06492046FFF77AFD0125E1E742
:1046300003492046FFF756FDDCE700BF90F90C0860
:10464000EAF90C089AF90C082DE9F041044604F542
:1046500000574FF0B7FC012208214FF00FFC5AF031
:104660008BF897F8D532072B98BF384A04F5405697
:1046700098BFD55CD6F8103193F8CB8088BF02255F
:10468000B8F1000F0BD132492046FFF72BFD002572
:10469000294620460522BDE8F041FFF7DFBE20464F
:1046A000FFF748FE60B104F537500122122138307F
:1046B000F9F798FC274A26492046FFF731FDE6E73F
:1046C000D6F8EC000368DB6C984768B196F8AD3615
:1046D00053B196F9AC36012B06DC1F4A1F49204620
:1046E000FFF71EFD0125D3E7D6F8EC000368DB6C6D
:1046F000984718B1D7F8383C190713D4D6F8EC000E
:1047000003681B689847032803D1D7F8383C9A07F9
:104710000BD4D7F8383CDB0609D40D492046FFF707
:10472000E1FCB5E70C4A0A49D9E70D4AC3E7D6F8D8
:10473000EC000368DB69984706460028EDD1094A7A
:1047400003492046FFF7ECFC3546A1E758FA0C0870
:1047500091E50C0890F90C089AF90C08E4F90C089A
:10476000F2F90C0807FA0C08F8B500F500550446F4
:1047700095F9D532B3B300F54056376F97B38AF049
:104780003FFC05F5496595ED000ADFED177A9FEDD1
:10479000171ADFED170AC71B20EE270A8D2025F018
:1047A000BBFFBCEEC00A10EE103A9F420CD296F846
:1047B00005319A0716D520460021F9F76DFD2046F0
:1047C000BDE8F840FFF7C0BC0CD996F805319B074F
:1047D00008D420460121F9F75FFD2046BDE8F840E6
:1047E000FFF732BFF8BD00BF00007A440000804FE1
:1047F000000000002DE9F341074600F59A4081F0E2
:10480000ADFC07F54054C0F3804801908AF0F8FBF6
:1048100094F808314345454606460DD007F53A5011
:1048200084F808813830002D41D03C4B3C4AC4F814
:104830000C61022151F0C4FC94F8083107F50058CE
:1048400043B394F809312BBBB8F9A63C9FED350A68
:104850009FED351ADFED350A07EE903AF8EEE77A6C
:1048600040F2571027EE800A25F056FFBCEEC00A32
:10487000D4F80C0110EE103A361A9E420AD90123E0
:1048800007F53A5084F80931294A244B022138307F
:1048900051F096FC98F9A53C002B94F805310DDCFD
:1048A0006FF3451384F8053102B0BDE8F0811B4B6E
:1048B000204AC4F80C8184F80981BAE7C3F3401296
:1048C000AA42F1D065F3451384F805319B06EBD578
:1048D000194BD3F8EC0003681B6998470028E3D014
:1048E0004FF070FB01221F214FF0C8FA3846FFF746
:1048F00021FD48B107F5375001222121383002B09F
:10490000BDE8F041F9F76EBB98F8A51C3222384695
:1049100002B0BDE8F041FFF7A1BD00BF20FA0C08CE
:104920002FFA0C0800007A440000804F00000000BD
:1049300045FA0C083AFA0C08805C002008B5044BD4
:1049400001221A708AF050FB024B186008BD00BFAC
:104950003185002034850020014B00221A707047F9
:10496000318500202DE9F04104468AF03DFB2A4BB9
:10497000B4F8BE201988294E914205460ED01A80FF
:10498000274B18603378A3B1002434704FF01AFB22
:1049900022461321BDE8F0414FF070BA3378214F21
:1049A000DBB93B782BB11E4B1F4A1B68C31A9342DD
:1049B00001D8BDE8F0810123337004F54053D3F8EA
:1049C000100190F8CB3013B103689B6A98474FF001
:1049D000F9FA012213214FF051FA3B78002BE8D06D
:1049E0003378002BE5D00E4A10491368EB1A8B423E
:1049F000DFD904F540541560D4F8100190F8CB309D
:104A0000002BD6D0002182F063FBD4F8100103689C
:104A1000BDE8F0415B6A18473285002030850020F0
:104A2000348500203185002080841E0040420F0024
:104A30002DE9F84300F5405500F500580446D5F837
:104A4000EC0098F88C710368DB6C9847014650B90C
:104A500095F9E030002BA5BFD5F8103193F8CB00C5
:104A6000012180F0010104F5055909F110094846BA
:104A700067F0B8FDD5F8103193F8CB300646002B1F
:104A80007BD0002865D03E4B93F9E030002B04DB4F
:104A900002463C49484667F07FF998F9567157B18C
:104AA00095F9E030002B0EDA04F5375001220F2182
:104AB0003830F9F797FA4FF085FA3246BDE8F843F7
:104AC00009214FF0DBB9D5F8EC0003685B69984722
:104AD00058B195F9E130002B07DA95F80531DA077E
:104AE00003D498F88C31DB07DED53146484667F0B1
:104AF000DFFDDFED257AB4EEE70AF1EE10FA05DD11
:104B00000A220921204600F09BFFD4E7023F032F31
:104B100011D801A353F827F0014B0108294B0108D4
:104B2000474B01084D4B01080A221521204600F091
:104B300087FF0028BFD10A220621204600F080FF0F
:104B40000028B8D1DCE70A221121F6E70A22152154
:104B5000F3E797B198F88C317BB9094B93F9E030C2
:104B6000002B06DB04F53A50084A0521383051F095
:104B700027FB4FF027FA0022A0E7BDE8F88300BF2B
:104B8000805C002060FA0C080000C84269FA0C083A
:104B900070B500F5005300F59A4586B093F87C1E79
:104BA0000446284681F088FA02A814F05DF904F55D
:104BB000955002A910300DF0E5FF04F58043049AEA
:104BC000C3F8F82C059AC3F8FC2C284681F0C6FAE5
:104BD00082061AD5284681F0CFFA04F59945FDEEF4
:104BE000C07A703504F5805417EE901A02222846D8
:104BF00017EE906A14F03EF994F82C35DB0706D4D2
:104C000001223146284614F035F906B070BD012165
:104C1000284614F0C1F90028F2D0F6E770B500F587
:104C2000804486B0B4F8043F8B420D46164603D14B
:104C3000D4F8003F934221D08AF0E2F9D4F8FC3E48
:104C4000C31A132B1AD9C4F8006FA4F8045FC4F870
:104C5000FC0E4FF0B7F904468AF0DAF9084B094A1E
:104C60001B68CDE90453084B0193084B0093CDE931
:104C70000201074B074920464EF030FF06B070BDD9
:104C80003885002080FA0C0898FA0C0810D00C081F
:104C90004CB30C0893FA0C0838B500F540540D4697
:104CA00094F8E130C3F380138B420BD021B14FF065
:104CB00089F911214FF0C2F894F8E13065F38613B9
:104CC00084F8E13038BD0000F0B52DED048B00F51F
:104CD00040568BB0D6F8103193F8CB30054600F52E
:104CE0008044002B67D096F9E030002B63DBD6F8C8
:104CF000EC0003685B699847002861D1D4F81C0D6B
:104D00009FED440A6C3028F05DFF0AAACDED080A39
:104D10008DED091A8DED070A12E9070004AB01AF0A
:104D200083E8070087E80700384628F097FCD4F8A6
:104D30001C3D05F599405030D3ED368AB0EE409ACF
:104D400050F0CCFD29F03CFBD4F8243DD6F8EC0023
:104D5000D3EDDB9A0368DB6CB0EE408A9847DFED59
:104D60002E7AB4EEE79AF1EE10FA02DC96F8E8300B
:104D70000BB100283AD0DFED297A68EEA78AF3EE6E
:104D80000E7AF4EEE78AF1EE10FA2FDCF0EE087AF4
:104D9000B4EEE78AF1EE10FA28DCF5EEC09AF1EEF7
:104DA00010FA23DAD4F81C0D03689B6F98470BB0F8
:104DB000BDEC048BF0BDD4F81C0D03689B6F0FE0B5
:104DC00005F50055D4F81C0DD5F8DC2C0368B2F9B4
:104DD0000820002A03DCD6F8E420022AEED1DB6F9B
:104DE0000BB0BDEC048BBDE8F0401847D4F81C5D57
:104DF000DFED0B0A2B68D3F88060D4F8243D40F235
:104E0000AB1093EDC90AB7EE001A25F085FC2846D1
:104E1000B047CCE79F0CB3450080BB44E02E654211
:104E20000000000000F5405090F8E80070470000D6
:104E30002DE9F04100F54055064695F8E030B1EB1C
:104E4000D31F0C4648D0254B00221A6000293FD0C2
:104E50004FF0B8F812214EF0F1FF95F8E03064F30E
:104E6000C71385F8E03084F0010872F0F1FE414686
:104E700072F0CAFE06F50057B8F1000F06D097F899
:104E80006A321BB98AF0BCF8C7F86C0287F86A82EC
:104E900014B3B7F8B8325B071ED5D5F8103193F8C4
:104EA000CB30CBB1D5F8EC0003685B69984798B973
:104EB000D5F8EC00036820219B69984760B106F59E
:104EC00037500122BDE8F0410D213830F9F78AB89A
:104ED0004FF078F81C21BEE7BDE8F081388500204E
:104EE0002DE9F04F2DED0A8B00F540558DB0D5F82A
:104EF000103193F8CB60044600F580471EB90121BC
:104F0000FFF796FF0BE095F9E020002A65DAD5F867
:104F1000EC0003689B6C98470646002841D04FF090
:104F2000000B95F9E020B14E002AC0F25381D6ED76
:104F3000007AB4F9A420B8EE677A1AB9B4F8A220BE
:104F4000A4F8A420B4F8A430DFEDA96A07EE903AE3
:104F5000F8EEE77A67EEA67AB4EEE77AF1EE10FAA9
:104F6000ACBF012100212046FFF796FE95F9E02015
:104F7000002A95F8E120B8BF4BF0010B530697F8D3
:104F8000E82E48BF4BF0020B0AB14BF0080B326819
:104F9000594620460DB0BDEC0A8BBDE8F04FFFF737
:104FA0003DBED5F81031204693ED0C8AF9F744FA4E
:104FB000B4EEC80AF1EE10FAB1D5D5F8103193F875
:104FC000A130032BABD14DF009FB4FF480114222ED
:104FD0004DF0BCFA3146204692E797F8E8AEBAF1B8
:104FE000000F03D0814A0023136098E7D7F81C0D07
:104FF00093F8079003685B6F984780460090D5F858
:10500000EC0003685B69984720B1D5F8E430022BC7
:1050100000F0E280B9F1000F0CBF4FF0000B4FF42D
:10502000007BB7EE00BAB8F1000F02D04BF4806BF2
:10503000009604F59D4808F1300840466AF0CCFC23
:105040000130D7F81C0D9FED6B0A9FED6BCADFEDA9
:105050006B8A0CBF012302236C3008EE103A28F053
:10506000B1FD0CABCDED0A0A8DED0B1A8DED090AE1
:1050700013E907000DF10C0E0DF1180C8CE8070078
:105080008EE80700704628F0E9FAD7F81C2DDFED0E
:105090005C7A92ED36AA2AEE27AAB4EECC0AF3EE99
:1050A0000EBAF1EE10FA04F59940B4EEEBAAC8BFBF
:1050B0004BF4807B5030F1EE10FAC8BF4BF4807B8C
:1050C000F0EE40AA50F00AFC29F07AF9B8EEC88A4E
:1050D00004F59A40B4EEC80AF1EE10FA98BF4BF00E
:1050E000800BF0EE409A81F053F868EE288AB0EE1B
:1050F000C09AB4EEE89AF1EE10FA204648BF4BF0A1
:10510000400B0AF0A1FD002846D14BF0200B019680
:1051100040466AF061FC01284FD14BF0100BB246BB
:105120003249B9F1000F53D0009B002B50D0F4EE60
:10513000CCAAF1EE10FA4BDCB4EEEBAAF1EE10FAC9
:1051400046DCF4EEC89AF1EE10FA41D8B4EEE89AD3
:10515000F1EE10FA3CD5019BD3B3BAF1000F37D072
:105160000A68B4F9A40007EE902AB8EE677A18B975
:10517000B4F8A200A4F8A400B4F8A43007EE903A62
:10518000F8EEE77A67EE8B7AB4EEE77AF1EE10FA92
:1051900019D501320A60C4E604F53350383050F0B6
:1051A00045FBDFED187A90ED007AB4EEE77AF1EE88
:1051B00010FAAAD400230193AAE740466AF00CFC37
:1051C0000130ADD1A9E701212046FFF731FEA8E665
:1051D0000022DFE70121C6E6B9F1000FB0EE08BA00
:1051E0000CBF4FF0000B4FF4007B1FE73885002009
:1051F000CDCC4C3E9F0CB3450080BB440000C84260
:10520000E02E65420000484310B500F5B052044658
:1052100007CA88B002AB83E807009FED1D7ADDED79
:10522000047A77EE877A9FED1B7ACDED047AD4ED80
:105230002B7AF0EEE77AF4EEC77A04F59940F1EEB6
:1052400010FA00F150000BD5B4F9A22007EE902A15
:10525000F8EEE77AF7EE006A86EEA77A84ED2B7A0D
:10526000D4F8AC200192194601AA50F005FC204662
:10527000FFF736FE2046FEF755F92046FEF72AFADC
:105280002046FDF7E7FF2046FEF79CF808B010BD6A
:105290000AE81C410000003410B504462DED028BD5
:1052A0001D205AF087FF60B304F54053D3F8EC009B
:1052B00000F0C4FA192108EE100A04F5546048F011
:1052C0005BFC02281AD00338012808D804F53350B3
:1052D000383050F0ABFA90ED008ABDEEC88AB8EED7
:1052E000C88A9FED090A28EE000ABDEC028B04F57E
:1052F0009D403030BDE810406AF0F4BB9FED038A5A
:10530000EDE7BDEC028B10BD0AD7233C0000000086
:10531000134A0260134A426002F17401816012492B
:10532000C16002F52A510161083941612439816166
:10533000A2F6FC71C1610D49016202F6646141622D
:1053400002F62821816202F62C21C16202F5236156
:1053500002F634224263064A01638263704700BF4B
:10536000480E0D082C4F0020A87900209C790020C1
:10537000982D0020172952D8DFE801F0100C1418DE
:10538000221F2A1C5126512E51513236393D41518E
:105390005144484D00F59E400C30704700F5AC403C
:1053A0006430704700F59E404C30704700F59F40D8
:1053B0000830704700F5A640F2E700F5AA40F7E78D
:1053C00000F5A8407C30704700F5A9404030704798
:1053D00000F5AB405830704700F5A74024307047C7
:1053E00000F5A7406030704700F5A240FAE700F5ED
:1053F000AA404430704700F5A6402030704700F5C1
:10540000AD40FAE700F5AD407030704700F5005050
:10541000D0F8900B704700F5A8403430704700205A
:105420007047000073B50B6805461B6C08460C46B8
:1054300016469847034605F53A500F4A0096042150
:10544000383050F0BDFE4EF0BDFD236805461B68A8
:10545000204698470A21024628464EF00FFD074B8A
:1054600093F8E1309B0641BF054A137843F00403EB
:10547000137002B070BD00BF9CFA0C08805C002065
:10548000DC86002038B50C4A182305460C464CF043
:10549000F3FE78B121462846FFF76CFF30B1014694
:1054A000064A2846FFF7BEFF002038BD28464CF0CC
:1054B0002BFEF9E70120F8E71CFB0C08BCFA0C08EE
:1054C00010B500F50053002283F88C2D094B0446DB
:1054D00093F8E01000F5804304F54054D3F81C0D18
:1054E000C9097AF07DFCD4F8EC000368BDE81040EF
:1054F000DB681847805C002070B5054608680368C3
:105500005B690C461646984790B1306803685B6942
:10551000984768B905F54053D3F8102192F8CB208D
:1055200032B193F9E030002B02DB2846F8F79AFFFE
:1055300004480BF055F920680368BDE870409B688B
:10554000184700BF1486002070B500F5405504468A
:10555000D5F8EC000B4E0368DB6998473074D5F83A
:10556000EC0003681B689847F070D5F8EC000368FE
:105570005B6C9847014604F59350BDE8704043F0DA
:1055800025BC00BFBD86002070B52DED028B244BDD
:1055900093F80531DB0782B006460D461446B0EE9F
:1055A000408AF0EE608A06D500232B60236002B0AB
:1055B000BDEC028B70BD59F0DFF9037F002BF3D0F7
:1055C000F36A9FED181A1B689FED170AB3F90830AC
:1055D00007EE103AB36A1B68B3F9083007EE903A49
:1055E000B8EEC77AF8EEE77A67EE000A68EE811A3D
:1055F00027EE800A28EE011A01A9684625F080FFEF
:10560000DFED0A6A9DED007ADDED017A27EE267A5C
:1056100067EEA67A85ED007AC4ED007AC7E700BF91
:10562000805C00200AD7233C530469390000C8423B
:1056300070B52DED028B88B0002302930393364B97
:1056400093F8053113F0010F0646B0EE408A06AD1F
:1056500002AC03D159F090F9037F5BB994E80300E1
:1056600085E803009DED060ADDED070A08B0BDECF4
:10567000028B70BDB36ADFED296A1B68B3F908308D
:1056800007EE903AF36A1B68B3F9083007EE103A58
:10569000B8EEC77AF8EEE77A27EE267A67EEA67AB2
:1056A000F1EE476ACDED026ADFED1D6ACDED037ABA
:1056B000B0EEC77AB4EEE67AF1EE10FA06D5F0EE67
:1056C000E77AF4EEE67AF1EE10FAC7D403AA21469F
:1056D0001448F8F7F7FEDDED027A9DED037AF0EE5F
:1056E000E77AB0EEC77AF4EE477AF1EE10FACCBF63
:1056F000B0EE670AB0EE470A204627F0FDFE04A888
:105700008DED040ACDED050A27F0A8FF204688EEAE
:10571000000A27F021FFA1E7805C002053046939CB
:1057200000000034802C0020094B93F9E020002A6F
:105730000CDAB5EEC00AF1EE10FA07D9D3F8103141
:1057400093F8A100C31E584258417047002070478B
:10575000805C0020436A1B6893F8CB3043B1054B53
:1057600093F8E00000F0A000203818BF0120704737
:1057700001207047805C002010B5436A0446186819
:10578000D1B1022181F0B4FC236A9FED0C1A186894
:105790000368F0EE410ADB6AB0EE410A9847236ADB
:1057A000074A1868D2EDAD0A03689FED040A5B6EE4
:1057B000BDE81040002118470121E3E70000000088
:1057C000804C002010B5436A04461868002930D088
:1057D000022181F08DFC236A18687AF0D1FA636A9D
:1057E0001B6893F8A130012B04D8236A01211868A3
:1057F0007BF060F8636918687EF06CF9636918687B
:105800007EF0C8F963699FED0C0A18687EF0EEFB24
:10581000636918687EF05CFC236A9FED071A1868BC
:105820000368BDE81040DB6AF0EE410AB0EE410AC1
:1058300018470121CDE700BF0000000013B5044662
:1058400001A90C480AF090FA10B1019802B010BDFD
:10585000636918687DF048F818B9074BD3F8F40C61
:10586000F4E7064801AA032113F03AFB0028F4D01C
:10587000EBE700BF802C0020806C002070790020B6
:1058800070B504462DED028B00296AD18368B3F907
:105890006E58642DB8BF6425FFF7D0FFA842626838
:1058A000A4BF324B93F8E150B2F93430ACBFC5F32A
:1058B00080150125002BDBBF63691B685B4293EDFC
:1058C000C48AC8BF07EE903AB2F93230C8BFB8EE0A
:1058D000E78A002BB8BF5B429BB25B4207EE903A6F
:1058E000A368F8EEE77AB3F96E68F4EEC87AF1EEE1
:1058F00010FAD8BFB0EE678A2046642EB8BF64267F
:10590000FFF79CFF6369A26B1B68D2ED001A93ED51
:10591000C61AD3ED0E0A311A00EE101AB8EEC00AFC
:1059200025F0DCF96368B3F93230002BB8BF5B4275
:105930009BB25B4201EE103A40F29720B8EEC11ADA
:10594000F0EE480A24F0E8FE6369294618687DF005
:105950006FF8BDEC028B6369BDE8704018687EF09B
:10596000B7BB9FED030A0025EEE700BF805C002077
:1059700000000000436A186803681B6918470000AC
:1059800038B52DED028B03680446D3F88030984774
:10599000236B2A481B68F0EE408AB3F908500AF0DE
:1059A000F5F84FF47A72041E4FF000012846D8BF74
:1059B0004FF4FA7424F0EEFE8442B6EE000A2ADDBB
:1059C00007EE900AB8EEE77A07EE904A27EE007AE3
:1059D000F8EEE77A87EE278A4FF46D7038EEC00A4A
:1059E000F5EE087AB1EE400A80EE270AB7EE001A0B
:1059F000FEEE000A24F090FEF7EE007A77EEC07A11
:105A000028EE000A20EE080A20EE080AA7EE880A0F
:105A1000BDEC028B38BD031B07EE103AC4F57A7457
:105A2000B8EEC77A07EE904A27EE007AF8EEE77AEA
:105A300087EE278A38EE008ACEE700BF802C002050
:105A40002DE9F04F2DED028B00F5804900F540580F
:105A500099F8084F89F8082F0546D8F8EC00036834
:105A600083B01B680F4616469847B84221D105F50A
:105A700000551A2E85F8686207D130B905F66C45D5
:105A8000D9F81C3D2A68C3F8FC208C4B93F8E13010
:105A9000980606D40124204603B0BDEC028BBDE875
:105AA000F08FB442F6D0864A137843F002031370A5
:105AB000F0E7022E0CD01B2F12D105F59F40314686
:105AC000083003B0BDEC028BBDE8F04F01F066B9C1
:105AD00039462846FFF7D6FC04460028EBD1DAE722
:105AE00039462846FFF746FC0446019018B9284677
:105AF0004CF00AFBCFE7D8F8103193F8CBB003682D
:105B00005B699847019A05F5A74324338BF0010A96
:105B10009A4208BF0120BBF1000F08D10198036829
:105B200051465B689847044648BB664A22E098F9AC
:105B3000E030002B80F2B380002800F0B080DFF866
:105B40007CB1DBF8EC0003685B69984704460028E9
:105B500040F0A5800198FFF713FFABF54050B0EE81
:105B6000408AF8F769FCB4EEC08AF1EE10FA40F30F
:105B70009680554A01992846FFF754FC8BE705F5B6
:105B8000435101AA2C31284605F50054FFF7B4FC17
:105B90000198C8F8EC0084F8686203681B689847AD
:105BA0003246014605F57F604DF01EFD05F53A5081
:105BB0000021383057F0F4FF94F9563123B105F540
:105BC0000550103066F098FDD8F8EC0003681B68AB
:105BD0009847C21E5042504104F63C4289F8AC0D31
:105BE000D9F81C3D1268C3F8F82004F66C42D9F8C5
:105BF0001C3D1268C3F8FC20012F01D00B2F06D1E9
:105C000004F65444D9F81C3D2268C3F8FC20284609
:105C1000FFF79AFC294B93F8E1309B063FF543AF21
:105C200038E705F5005393F85021002A3FF476AF8A
:105C3000B3F86C21D1077FF571AF93F88C21002A5E
:105C40003FF46CAFD8F8102192F8CB20002A3FF433
:105C500065AF93F868320A2B7FF460AF98F9E030B3
:105C6000002BFFF65BAF194A01992846FFF7DAFBD4
:105C7000002410E716480AF0EDF90028D1D1D8F831
:105C8000EC0003685B6998470028CAD00198036854
:105C90005B69984704460028C3D10E4A6AE7019819
:105CA00003681B6998470028E4D009480AF0C0F946
:105CB00004460028DED1084A5CE700BF805C002073
:105CC000DC86002042A20E08E4FA0C0808FB0C084F
:105CD000802C0020F6FA0C08B2550E080148FFF798
:105CE000AFBE00BF802C002013B504468DED010A25
:105CF00069F00AFE6369A26B1B6892ED001A93EDCE
:105D00000E0AD3EDC60A01A968F08CFC9DED010ACC
:105D100002B010BD436A186803685B6A1847000048
:105D200038B5436A1C6894F8CB10054661B9204623
:105D300081F0DEF96B6A1B6893F8A10018B10128A5
:105D400014BF0320022038BD164803783BBBFFF781
:105D5000EBFC20BB144A92F8E03003F0A003202BA8
:105D600017D0B5EEC00AF1EE10FA10D592F8E23075
:105D70005B070CD40121204681F0BAF96B6A1B68DD
:105D800093F8A130012B0CBF02200320DBE7022196
:105D9000F1E72046022181F0ABF90420D3E701208E
:105DA000D1E700BF14860020805C002010B52DEDE7
:105DB000028B134B93F80531DB07044604D59FEDA6
:105DC000110ABDEC028B10BD58F0D6FD037F002BED
:105DD000F5D0636B186858F0F9FEA368DFED0A7A16
:105DE00003F5156292ED008A03F65413D3ED000A11
:105DF00028EE278A25F03EFB28EE000AE1E700BFE7
:105E0000805C0020000000000000C8420148F8F754
:105E100083BB00BF802C00200148F9F717B800BFF2
:105E2000802C00200148FFF70BBE00BF802C002013
:105E300070B52DED028B7D4D95F8E1308CB00026CC
:105E4000044658060496059603D5636918687CF0E5
:105E5000BFFB95F80531D9075DD463689B899A0724
:105E60001BD573484FF0E2FCDFED727A90ED007ABB
:105E7000B4EEE77AF1EE10FA0FDD4EF0A3F83D2113
:105E80004DF0DCFF6C4809220521FFF7D9FD20B950
:105E9000092202212046FFF7C5FF636893F95430B9
:105EA000CBB365489FED658AF8F7D0FFE3689FEDB7
:105EB000647A1B68D3ED0A7AF4EEC87AF1EE10FA30
:105EC000B8BFF0EE477AB6EE000A27EE800A204609
:105ED000FFF7AEFB8DED040AB0EEC00AB4EEC80ABF
:105EE000F1EE10FACDED050A06D5F0EEE00AF4EE7B
:105EF000C80AF1EE10FA0ED495F8E2301B0704D46C
:105F00004EF060F849214DF099FF95F8E23043F0EA
:105F1000080385F8E23095F8E3306FF3820385F8E3
:105F2000E330606909960A9609AD2A4604A900681B
:105F300001237CF0B7FB636918687DF02BFE636971
:105F400018687CF003FFA3688DED060ACDED070A03
:105F50008DED081AD3ED007AF5EEC07AF1EE10FA65
:105F600052DD384B9FED388AB3F9A83200EE903AF3
:105F7000F8EEE00A2046CDED030AFFF75FFCA368C8
:105F8000DDED030AD3ED001A9FED2A0AB7EE002AD1
:105F900007EE900A31EE822AB8EEE71A22EE082ABE
:105FA00061EE881A24F0F8FADFED287A20EE270A4D
:105FB000DFED277A20EE270AADF0F2F9DFED257A42
:105FC00020EE270A06A820EE088A27F047FBB4EE49
:105FD000C08AF1EE10FA17D5C8EE006A63699DED2C
:105FE000067ADDED077A27EE267A67EEA67A8DED42
:105FF000067ACDED077A1B68D3F88823C3F894237B
:10600000D3F88C23C3F89823236A13491C682846C5
:10601000FCF7E8FA0B9B009395E80C0006A92046D4
:1060200079F060FF0CB0BDEC028B70BD805C00208D
:106030006479002000002F44802C002000000034F0
:1060400000007A43804C00200000C8420AD7233C5D
:1060500035FA8E3C0AE81C41EC84002013B5044656
:106060000191FFF7E5FE0199204602B0BDE810401E
:10607000FFF706BC0148FEF7DBBE00BF802C002006
:1060800000487047385B00200148F8F733BA00BF7A
:10609000802C002030B50F4D87B0002304466946A0
:1060A000D5F8240D0093019302937CF067FED5F898
:1060B000240D02A97CF0B6FE009B0393019B049380
:1060C0000222029B059303A9204613F0D9F920462A
:1060D00007B030BD806C0020014B01221A70704760
:1060E0003C8500200020704700207047002070474A
:1060F0000020704700207047002070470020704744
:106100000020704700207047002070479FED010A73
:10611000704700BF0000000000207047002070475B
:106120000020704701207047002070470020704712
:106130000120704700207047012070470120704700
:1061400000207047012070470120704700207047F1
:106150000048704734FB0C080048704734FB0C08BB
:10616000836893F86439DB0706D5002380F83C3058
:10617000024B0222C3F8E42001207047805C00201B
:1061800090F83C3043B9836893F86439DB0742BF29
:10619000034B0122C3F8E420002380F83C30704711
:1061A000805C0020012380F83C3070472DE9F043EB
:1061B0002DED0C8BF0EE409A20EE000A97B00025F2
:1061C000A0EEA00A04468946B0EE41CAF0EE60AAED
:1061D00090461F46019502950395049505950695F1
:1061E000ADF0F4FAF7EE00CAB4EEEC0AF1EE10FAF4
:1061F000C8BFCCEE807AA36803F5126203F62413BD
:1062000092ED009A9FEDC5DAD3ED000AC4BF69EEA6
:10621000A79A6AEEA7AAB0EE690A25F02BF9A3683F
:1062200029EE0D9A03F5126203F62413D2ED008ACB
:10623000D3ED000A29EE009AB0EE6A0A25F01AF9A9
:10624000A36868EE8D8A03F6381203F63C13D3ED8B
:10625000000A92ED008A68EE808AB0EE4C0A25F0C2
:1062600009F9636828EE0D8A93F9703028EE008AE8
:10627000002B00F0D980236A9FEDA90A18686C30C2
:1062800027F0A0FCB0EE60AACDED080A8DED091A4A
:106290008DED070A24F0EAF9BDEEC0BAA14940F637
:1062A000B8321BEE100A24F065FA434207EE903A2A
:1062B0006368F8EEE77A93ED1A7A67EE877AB0EEC4
:1062C0004A0ACDED017A24F0D1F9FDEEC0BA40F6CC
:1062D000B83294491BEE900A24F04CFA42426368AB
:1062E000039507EE902A93ED1B7A93F97030F8EE40
:1062F000E77A022B67EE877ACDED027A6ED18A4B70
:10630000B3F9A8320AEE103AB8EECBBAB8EECAAA80
:10631000236AB4EECABAF1EE10FA1A683DDDA3683A
:10632000DFED820AA16B92ED051AD1ED001A03F59B
:10633000126393ED007A27EE0D7A3AEE4B0AC7EE20
:10634000200A24F0CBFCDDED017A37EE800A8DEDDA
:10635000010AB8EEEB0A236AB4EECA0AF1EE10FAAB
:106360001A6834DDA368A16B92ED061AD1ED001A0C
:1063700003F51263D3ED000A20EE8DDADFED6B0A30
:106380003AEE400ACDEE200A24F0A8FCDDED027AB8
:1063900037EE800A8DED020A20E0B1EE4A0AB4EE33
:1063A000C0BAF1EE10FAD4D5A368A16BDFED5F0A95
:1063B000D1ED001A92ED051A03F5126393ED007A00
:1063C00027EE0D7A30EE4B0AC7EE200AB9E7B1EEA0
:1063D0004AAAB4EECA0AF1EE10FAC3D4236AD3F87B
:1063E00000C00CF184030FCB12AD85E80F000EAE98
:1063F0000AAD86E80F0085E80F0004AB01AA294624
:1064000060467AF00BFA636893F97030022B16D16C
:10641000DDED047A39EE279ADDED057A78EEA78A6C
:10642000DDED067A38EE278A89ED009AC8ED008AFC
:1064300087ED008A17B0BDEC0C8BBDE8F083F0EE61
:10644000E99AF0EEEAAAF4EEE9AAF1EE10FA48BFF2
:106450006D46CDED009ACDED0AAAD5ED007ADFEDBF
:10646000340AB0EECCCAF4EECC7AF1EE10FAD8BF12
:1064700035468DED0ECA95ED007ADFED2E7A87EE6A
:10648000270AAD20B7EE001A3CEEC00A24F044F90A
:10649000E369D3ED937A04A820EE270A27F092FB54
:1064A000F0EEC07A8DED061AB0EEC91A31EE671A19
:1064B0008DED040AB0EEC11A39EE000ACDED050AE1
:1064C000B520F1EE410A24F027F9B0EE409A9DED97
:1064D000050AB0EEE81AF0EEC07A31EE671A38EE2F
:1064E000800AB0EEC11AF1EE410ABA2024F014F984
:1064F000F0EE408A9DED060AB0EEC81AF0EEC07AC2
:1065000031EE671A38EE000AB0EEC11ABF20F1EE84
:10651000410A24F001F9B0EE408A85E70000C84244
:106520009F0CB34548F4FFFF804C002000007A44E4
:106530000000000000A08C4510B52DED028B836A91
:10654000044686B0186858F041FBE36A1868B0EE5C
:10655000408A58F03BFB636B8DED010A186858F0D8
:1065600035FB05ABB0EE401A03A92046DDED010A6C
:1065700004AAB0EE480AFFF719FE636A186890F89B
:10658000CB1000293AD180F0B3FD2046FFF7F8F98F
:10659000636A1B6893F8A1100129B0EE408A3DD0D0
:1065A000032944D051B9236A012118687BF038F8D7
:1065B000236A186879F0CEFB9FED208A236AA268CF
:1065C000186892F8642903689DED030ADDED040A5A
:1065D0009DED051A92074CBFDB6B9B6B9847236AB6
:1065E000174A1868D2EDAD0A036800215B6EB0EE61
:1065F000480A984706B0BDEC028B10BD114B93F9C9
:10660000E120002A06DBD3F8E430022B04D190F815
:10661000A1300BB90121B6E70221B4E7236A18685B
:106620007AF0FEFF236A186879F0AAFBC4E7D979EB
:106630000029C3D12046FFF71DFDBFE70000000081
:10664000804C0020805C0020836893ED140AB5EE36
:10665000C00AF1EE10FA01DCFFF78CB970470000B8
:1066600070470000002070470120704702207047EB
:1066700000207047002070470120704700207047BD
:1066800081F0010070470000012070470120704731
:1066900000487047CCFB0C0800487047D8FB0C083A
:1066A00038B54369044618687CF040FA18B9636944
:1066B00018687DF0BFFB636920461D68FFF7E4FCA6
:1066C0006368B3F93820B3F9363000EE903A4342AC
:1066D00001EE102A00EE103AB8EEC11AF8EEE00A08
:1066E000B8EEC00A28467CF00DF9636920461D68A3
:1066F000FFF7CAFC6368B3F93820B3F9363000EE0F
:10670000903A434201EE102A00EE103A2846B8EEC5
:10671000C11AF8EEE00AB8EEC00A7CF06DF901206B
:1067200038BD000030B52DED028B0446436985B0BD
:106730001D68FFF7A9FC6368B3F93820B3F9363058
:1067400000EE903A434201EE102A00EE103AB8EE05
:10675000C11AF8EEE00AB8EEC00A28465B4D7CF09C
:10676000D1F82046FFF758FBB5F9A83208EE103AE9
:10677000236A186803689B6E9847B8EEC88AF0EEE3
:10678000400A02AA01A9B0EE480A2046FEF7FCFE24
:106790002046FFF70BFB236B1B68B3F90830F0EEC4
:1067A000408A00EE103A2046B8EEC00AFFF72EFBF2
:1067B0002046B0EE408A8DED030AFFF765FC636862
:1067C000B3F9363001EE103A434200EE903AB8EE9B
:1067D000C11AF8EEE00A2B20B0EE480A23F09CFF25
:1067E00020468DED030AFFF79BFA042813D8DFE853
:1067F00000F0032F252A4B00236A186879F0AAFAC3
:10680000236A002118687AF055F863699FED300A11
:1068100018687DF0EBFB236ADDED020A18689DED38
:10682000010A0368B0EE681ADB6A98476369186862
:106830007DF04EFC05B0BDEC028B30BD236A01211A
:1068400018687AF037F8236A186879F099FADCE763
:10685000204D2B7863B963689FED1F1ADFED1C0A8A
:1068600093ED040A452023F057FF284609F0A0FFC6
:1068700020469DED030AFFF737FA16488DED030A0F
:1068800003A909F0CFFFC6E7636A0221186880F008
:106890002FFCB5F9A832114800EE103A02AA01A95E
:1068A000B8EEC00A67F0EEFB20469DED030AFFF745
:1068B0001BFA0B488DED030A09F072FA63699DED2E
:1068C000030A18687CF0A4F8A5E700BF804C0020FC
:1068D000000000001486002000007A44C07A0020E6
:1068E000005A00200020704790F8B931002B14BFE7
:1068F0001B200320704700000020704701207047D4
:1069000090F89001062804D0A0F10A03584258419B
:106910007047012070470000012070470120704738
:1069200090F8B901034A044B002814BF10461846DA
:10693000704700BF70FC0C08CE680E0890F8B901D3
:10694000034A044B002814BF10461846704700BF86
:106950007CFC0C08CE680E0890F890010B3818BF2C
:106960000120704790F8B9312BB9044BD3F8880C4B
:1069700000F0010070470020704700BF804C0020ED
:1069800090F8903123B9034B187880F001007047DC
:1069900000207047F885002038B590F89041012C10
:1069A000054601D0002038BDC368186803681B691C
:1069B00098470028F6D1EB681B68204683F8B84852
:1069C000F1E70000C3681B68002283F8B8280120A3
:1069D0007047000070B52DED028B002380F8B931AF
:1069E000B0F87030012B84B004460D4601D8002960
:1069F00046D0636A254E1B6893F8CB3073BB24489E
:106A0000072384F890310368022B02D10021FBF7A1
:106A1000F3FB9FED208AE368F0EE480A1868B0EEB9
:106A2000481AF0EE481AB0EE480A01257EF0D6FD6D
:106A300084ED738A84ED748A84ED758A84F8B85184
:106A400004F59A7027F0A6FD134805F0D9F896F8DA
:106A5000E2306FF3C30386F8E23011E096F9E030DC
:106A6000002BCCDA04F13C0029F086FE0546002814
:106A7000C5D12046FFF704FB084A02214FF0A0FBD6
:106A8000284604B0BDEC028B70BD00BF805C0020C6
:106A9000EC84002000000000FC80002084FC0C0836
:106AA00038B5094D95F8C83F012B044603D105F6CA
:106AB000C47027F0D7FD95F8351E04485AF0C6FD7E
:106AC000002384F8B93138BD806C00203C7A002066
:106AD00010B52DED028B094B0446D3F8280DB0EE0E
:106AE000408A7EF013F99FED060A28EE008A012005
:106AF00084ED748ABDEC028B10BD00BF806C002059
:106B00000AD7233C10B52DED028B094B0446D3F870
:106B1000280DB0EE408A7EF009F99FED060A28EEB6
:106B2000008A012084ED758ABDEC028B10BD00BF88
:106B3000806C00200AD7233C10B52DED028B094B49
:106B40000446D3F8280DB0EE408A7EF0FDF89FEDA4
:106B5000060A28EE008A012084ED738ABDEC028BC0
:106B600010BD00BF806C00200AD7233CC3681B689F
:106B700018697CF01DBA000038B5D0F8943104468D
:106B80000D461BB988F03CFAC4F8940188F038FA35
:106B9000D4F89431C01A4FF47A73B0FBF3F0B4F820
:106BA0009231984209D32046FFF76AFA2B88044AAB
:106BB00006214FF005FB012038BD0020FCE700BF97
:106BC000A0FC0C0890F89031052B05D1054BD3F8AB
:106BD000303DD8687CF064B9C36818680368DB6826
:106BE000184700BF806C002008B590F89031052B45
:106BF0000BD1094BD3F8303DD868243026F02EFD58
:106C0000BCEEC00A10EE100A08BDC368186803681D
:106C10009B689847F4E700BF806C002090F89031A3
:106C20008B4206D00B2B80F8901102D10148FCF763
:106C3000B5BF7047802C002073B501231E4E80F82D
:106C40007530D6F8EC30834205460A4614D101244B
:106C500085F8B941D6F8EC00019203681B689847A3
:106C6000019A014615484CF0BFFC96F8E1309A06AF
:106C70001BD4204602B070BD01910321FFF7D2F86A
:106C8000019A04460028E2D185F875004DF09AF982
:106C90001B220A214DF0F2F896F8E1309B06E8D568
:106CA000074A137843F0040303E0054A137843F0DE
:106CB00002031370DDE700BF805C0020703C002001
:106CC000DC86002030B585B004460D460146684696
:106CD000FFF7E0F9694604F13C002AF0FFFAC8B971
:106CE0004DF070F91B220A214DF0C8F80D4B93F8B6
:106CF000E1309B0604D50C4A137843F0040313706B
:106D00002046FFF7BDF9094A04214FF059FA002047
:106D100005B030BD2946204605B0BDE83040FFF73C
:106D20008BBF00BF805C0020DC860020B4FC0C0818
:106D300030B585B004460D4601466846FFF7AAF90E
:106D4000694604F13C002AF0EDFAC8B94DF03AF971
:106D50001B220A214DF092F80D4B93F8E1309B066F
:106D600004D50C4A137843F0040313702046FFF750
:106D700087F9094A04214FF023FA002005B030BDFD
:106D80002946204605B0BDE83040FFF755BF00BF9B
:106D9000805C0020DC860020F0FC0C087FB50546F6
:106DA0000E4605F13C0401466846FFF773F9694653
:106DB00020462AF0B7FAC0B9204669462AF08EFA72
:106DC000044690B94DF0FEF81B220A214DF056F80A
:106DD0000D4B93F8E1309B060FD42846FFF750F98E
:106DE0000A4A04214FF0ECF904E031462846FFF747
:106DF00023FF0446204604B070BD054A137843F0D3
:106E000004031370E9E700BF805C002028FD0C0834
:106E1000DC86002030B5044685B00F4809F008F93B
:106E20000546B0B1072384F8903100230193029303
:106E30000393E36801A918687DF002FFE36818680E
:106E4000036801A95B680022984704480021FBF70A
:106E5000D3F9284605B030BD802C0020EC840020FA
:106E6000F0B5424FD7F8FC2CD7F8F83C2DED028B4B
:106E70001343D7F8F42C134387B005460C460CD1C6
:106E80004BF0ACFB40F275124FF4801107B0BDEC33
:106E9000028BBDE8F0404BF059BB80697FF06CF984
:106EA0002046B0EE408A12F00FF803283AD1EB6882
:106EB00001A918687DF0A0FF064698B3DDED017AC0
:106EC0006368009338EE678A294BDFED2A7A93F9DD
:106ED000E0309FED290A2948002BA8BFB0EE670AD1
:106EE00038EE008A009BBDEEC88A002118EE102AF9
:106EF0009342ACBF00930092FBF77EF96B69186870
:106F00007CF098FFDDED007A1D48B8EEE70A3146C7
:106F100009F008FF00212846FFF780FE07B0BDEC0E
:106F2000028BF0BD94E80F0002AE86E80F00D7F8A0
:106F3000F83C04936A46D7F8FC3C0593022130469E
:106F400011F0CEFF78B94DF03DF8022215214CF03A
:106F500095FFDDED037AF8EEE77A77EE887AFDEEBD
:106F6000E77ACDED007A0026AEE700BF806C002006
:106F7000805C0020000000000000C842EC8400207B
:106F8000F885002030B52DED028BC36887B004462C
:106F900018680D467DF024FF00284BD194F890210D
:106FA00000230093019302936AB93148039303A924
:106FB0000493059309F0E8FE28B1039B0093049B1A
:106FC0000193059B029394ED730A9FED2A8AE3686F
:106FD000DDED000A9DED011ADDED021A1868B4EE30
:106FE000C80AF1EE10FAAABFDFED237A9FED230A5B
:106FF00020EE270A7EF0F2FAD4ED747AF4EEC87A25
:10700000F1EE10FA07DBE3689FED1B0A186827EE24
:10701000800A7DF07BFED4ED757AF4EEC87AF1EE4D
:1070200010FA07DBE3689FED140A186827EE800A60
:107030007DF07CFEE368294618687EF0F7F9054686
:1070400088B10F4B1B68022B09D0032B03D10D4BCA
:1070500093F9D9321BB10A480021FBF7EDF8012161
:107060002046FFF7DBFD284607B0BDEC028B30BDA4
:10707000F8850020000000340000C8420000000035
:10708000EC840020804C002010B52DED028BC368ED
:10709000DFED348A1B684269D3ED0A0A9FED328A1C
:1070A00093ED060AF4EEE80A0446F1EE10FA1068D1
:1070B000B8BFF0EE480A7BF00BFAE36862691B6820
:1070C0001068D3ED0A0A93ED060AF4EEE80AF1EE31
:1070D00010FAB8BFF0EE480A7BF072FA63691868DC
:1070E0007BF002FC18B9636918687CF03DFCE3682A
:1070F00062691B68106893ED080A93ED0C1AD3EDD2
:10710000070AB0EEC00A7BF0FDFBE36862691B680A
:10711000106893ED080A93ED0C1AD3ED070AB0EE50
:10712000C00A7BF069FC636918687BF0FFFC18B942
:10713000636918687CF07EFE00210C48FBF75CF860
:107140000B4868F067FD0B4AB2F8E23023F4816324
:10715000A2F8E230BDEC028B20460221BDE81040CF
:10716000FFF75CBD0000003400007A43EC8400208F
:10717000307B0020805C002010B50C4B0446D3F817
:10718000300D90ED0B0A90F8502000F11C017DF0BD
:107190009FFA07480368022B02D00821FBF72CF85E
:1071A00020460521BDE81040FFF738BD806C002067
:1071B000EC840020F0B52DED028B4A4DDFED4A8ABC
:1071C000B0EE408A8FB00446D5F8300D0E46174613
:1071D0007DF0F4F8F0EEC87AF4EEE87AF1EE10FA09
:1071E00007D49FED420AD5F8300D28EE000A7DF055
:1071F0004BF9D5F8300D90ED0B0AB0EEC00A0FB187
:10720000B1EE400A7DF030F90023D5F8300D079338
:1072100002AA07A9089309937DF052F9DFED347AA9
:107220009DED027AB4EEE77AF1EE10FA56DD022215
:1072300007A90AA812F024F971680191304611F0EB
:1072400043FE019902460AA811F014FEE3680AA958
:1072500018687EF0EBF810B92648FDF799F8A06998
:107260007EF088FF02684368D5F8300D049303A9C7
:107270001C30039226F024F905A88DED050ACDED0A
:10728000060A26F0EBF91C4B1B68022B1BD0D5F825
:10729000303D1948D3ED0A7AF4EEE87AF1EE10FAAF
:1072A000B8BFD3ED047AF4EEC07AF1EE10FA4FF0E5
:1072B000000110D5DFED117AB4EEE70AF1EE10FA15
:1072C00009DDFAF7B9FF04212046FFF7A7FC0FB04C
:1072D000BDEC028BF0BDFAF78FFFF4E72046FFF715
:1072E0004BFFF4E7806C0020000000340000C8422F
:1072F00000009643802C0020EC8400200000FA431C
:1073000070B52DED028B294BDFED298AD3F8284D7E
:10731000D3F8245DD4ED0A0A9FED268A94ED060A7F
:10732000F4EEE80AF1EE10FAB8BFF0EE480A0646AD
:1073300028467BF0CDF8D4ED0A0A94ED060AF4EE67
:10734000E80AF1EE10FAB8BFF0EE480A28467BF0E2
:1073500037F928467BF0C8FA10B928467CF004FBC0
:1073600094ED080A94ED0C1AD4ED070AB0EEC00AA9
:1073700028467BF0C7FA94ED080A94ED0C1AD4ED78
:10738000070A2846B0EEC00A7BF036FB28467BF0A1
:10739000CDFB10B928467CF04DFD07480021FAF7D7
:1073A0002BFFBDEC028B0123337070BD806C00207D
:1073B0000000003400007A43EC84002008B5074840
:1073C000D0F8883C9B0704D50121A0F50050F6F7C2
:1073D000FFFEBDE80840024809F004BB804C0020D5
:1073E000F885002030B589B00446FEF7B3F930B116
:1073F0000021204609B0BDE83040FEF7E3B9636ADA
:10740000022118687FF074FEE368186803685B69FE
:10741000984701461048FCF7A9FE636918687CF09C
:1074200057FE236A1D68636918687BF08FFC05AC02
:1074300020460A498DED020ACDED030A8DED041AAE
:10744000FBF7D0F8079B009394E80C0002A92846AC
:1074500078F048FD09B030BD802C0020EC8400207D
:1074600038B50446FEF776F9054628B120460021D6
:10747000BDE83840FEF7A6B9636A022118687FF0BC
:1074800037FE29462046BDE83840FEF7E7BD00003C
:107490000148002106F0C2BE5882002030B5174DC9
:1074A0009FED170A05F5804389B00446D3F8300DE7
:1074B0007DF06EF901462846FCF758FE63691868AE
:1074C0007CF006FE236A1D68636918687BF03EFC49
:1074D00005AC20460B498DED020ACDED030A8DED7A
:1074E000041AFBF77FF8079B009394E80C0002A9AD
:1074F000284678F0F7FC09B030BD00BF802C002092
:1075000000000000EC84002030B589B00446FEF78E
:1075100021F930B10021204609B0BDE83040FEF726
:1075200051B9636A022118687FF0E2FDE3681868C8
:1075300003685B69984701461048FCF717FE6369CA
:1075400018687CF0C5FD236A1D68636918687BF0C4
:10755000FDFB05AC20460A498DED020ACDED030A7C
:107560008DED041AFBF73EF8079B009394E80C009E
:1075700002A9284678F0B6FC09B030BD802C002066
:10758000EC84002030B52DED028B83B00446FEF76D
:10759000E1F820B9636A1B6893F8CC3043B9002145
:1075A000204603B0BDEC028BBDE83040FEF70AB9BF
:1075B00094F89831DA071DD4E3681D682B682846D3
:1075C0009B689847D5ED097A94F89831B4EEE70AAC
:1075D000F1EE10FA4CBF0122002262F3000384F89E
:1075E000983107D4204603B0BDEC028BBDE8304093
:1075F000FFF7F8BE94F898319B0734D4E368DFEDC9
:10760000458A1B686269D3ED0A0A9FED438A93EDB0
:10761000060A1068F4EEE80AF1EE10FAB8BFF0EED0
:10762000480A7AF055FFE36862691B681068D3ED79
:107630000A0A93ED060AF4EEE80AF1EE10FAB8BF72
:10764000F0EE480A7AF0BCFF636918687BF04CF9E9
:1076500018B9636918687CF087F994F8983143F099
:10766000020384F898312D4BD4F8A021D3F8F43CD0
:107670009B1A07EE903AB8EEE78AF1EE047AB0EE84
:10768000C87AB4EEE77AF1EE10FA38D594F898316A
:1076900043F0040384F89831204684ED678AFEF7AE
:1076A000C7FB6369A26B1B68D2ED001A93EDC61A83
:1076B000D3ED0E0AB1EE480A23F010FB63691B6894
:1076C00040F2AA4093EDC31AD3EDC40A23F024F884
:1076D0002046FEF709FB12488DED010A08F060FB19
:1076E00063699DED010A18687BF092F96369186877
:1076F00003B0BDEC028BBDE830407CF0E9BCD4EDBA
:10770000677A68EE277AF5EEC07AF1EE10FAC3D503
:10771000BCE700BF0000003400007A43806C00200A
:10772000005A002030B52DED028B83B00446FEF7E1
:1077300011F820B9636A1B6893F8CC3043B9002173
:10774000204603B0BDEC028BBDE83040FEF73AB8EE
:107750006369DFED347A1B6894ED710A93EDC31A07
:10776000D3EDC40A20EE270A40F2C44022F0D4FF31
:107770002046FEF7B9FA236A186803689B6EB0EEDC
:10778000408A9847284BB3F9A83207EE903AB4F8EC
:10779000BC316425F8EEE77A13FB05F3B4EEE70A93
:1077A00007EE103A94F9BE31F1EE10FAD8BFF0EEC0
:1077B000407A13FB05F39FED1D0AF8EEC76A07EE4A
:1077C000103AF4EE407AB8EEC77AF1EE10FA58BFEC
:1077D000B0EE670A6846CDED006A8DED017A25F0BE
:1077E0008FFF236ADDED010A1868B4F8C031026822
:1077F0009DED000A126B13FB05F301EE103A012117
:10780000B8EEC11A90476369B0EE480A18687BF079
:10781000FFF8636918687CF05BFC03B0BDEC028B79
:1078200030BD00BF0000C842804C002000007A44F8
:107830002DE9F0432DED028BB64F85B00446D7F805
:10784000EC00FDF787FF48B1D7F8EC00002105B048
:10785000BDEC028BBDE8F043FDF7B4BF07F58056E1
:10786000D7F8100102217FF043FCD6F81C3D93EDC0
:10787000378A87F0C5FBB7F8E03003F4814305464B
:107880007BB1D6F8240D7AF0A3FE2378022B08D121
:1078900055F06AFBA04BA14A06214EF091FC032350
:1078A000237063F0BDFE63F0A7FE48B163F0B8FE3D
:1078B00063F0ACFE20B12378012B10D9022B1DD030
:1078C0002378082B00F28581DFE813F021003900CE
:1078D00063000A013E0145015A015C012A0055F08E
:1078E00043FB8D4B8E4A06214EF06AFCD6F8243DB0
:1078F000D3F85433636108232370E1E755F034FB78
:10790000854B884A06214EF05BFC0323F4E7D6F84A
:10791000280D03681B69984710B12046FFF7F0FC5B
:107920002378082B00F27381DFE813F05C01640117
:1079300064017A017A017A017A0182018201A560EB
:10794000D6F8243D9FED787AD3F854336361774BB2
:1079500003F6C842D2ED007AF4EEC77AF1EE10FADF
:107960004EDB9FED737A67EE877AD6F8283D93ED6C
:10797000087AB0EEC77AF4EE477A4FF07E53F1EE14
:1079800010FA48BFB0EE677A2361022384ED067ACD
:107990002370D4ED016A9FED647AD6F8243DF0EEB1
:1079A000E67AF4EEC77AF1EE10FA0AD4D4ED057A4D
:1079B00093EDD56A77EEC67AF4EEE76AF1EE10FA47
:1079C00029D4DFED5C6AD4ED067A67EEA67AD3EDB2
:1079D000DB6AF4EEE76AF1EE10FA26DCA368D4ED78
:1079E000047AEB1AB3F5FA6F21D2B4EE678AF1EE9E
:1079F00010FAC8BFB0EE678A84ED048AE5608FE7AD
:107A0000B3F9DE32002BB8BF5B429BB207EE903A6F
:107A1000F8EEE77AA9E70623237055F0A5FA3E4B66
:107A2000454A04214EF0CCFB7AE7A56078E7DFF801
:107A3000FC8008F6BC43D3ED006A67EEA67AF4EE4C
:107A4000C87AF1EE10FAD9D408F54C69D9ED007A6C
:107A5000F4EEC77AF1EE10FA22DB98F8F03C33B975
:107A60000623237055F080FA2B4B344AD9E7A8F54A
:107A7000005008F0E9F898B198F9063D83B9B8F9D3
:107A8000F23CD9ED007ADFED2A6A07EE103A67EE94
:107A9000A67AB8EEC77AB4EEE77AF1EE10FAADDC6A
:107AA000E068281AB0F5FA7F7FF63AAF0323237017
:107AB00008F6BC4855F058FA98ED007AD4ED047AEF
:107AC00067EE277A054617EE900AF4F71DFD124B74
:107AD0001B4ACDE90001062128464EF071FB1FE745
:107AE000D6F8240D7CF022FA63F09AFD63F084FD51
:107AF00068B155F039FA084B124A06214EF060FB86
:107B000063F08EFD63F066FD0423237008E7052310
:107B1000FBE700BF805C002074FD0C0882FD0C08B0
:107B20008CFD0C08A3FD0C0800000034804C0020E4
:107B30000000C842333373BFB5FD0C08D0FD0C08FC
:107B400000FE0C0828FE0C0863F06AFD63F054FD8B
:107B5000C0BB05232370404BE068DFED407AD3EDD6
:107B6000006A9FED3F7A2D1AA6EEA77A07EE905A8B
:107B7000F8EE677AF4EEC77AF1EE10FA3FF5D0AE80
:107B800007232370D6F8243D9FED367AD3EDC37AD0
:107B9000D3EDC66A67EE877AB6EE007A67EEA77A0B
:107BA00067EE877A87EEA67AD4ED057A77EEC77A04
:107BB00093EDD57AF4EEC77AF1EE10FA3FF6B0AE57
:107BC0000823A2E763F02CFD63F020FD0028C0D15C
:107BD000A6E64AF003FD40F29C524FF480114AF0B1
:107BE000B5FC9DE6204805B0BDEC028BBDE8F04336
:107BF000FFF7F8BBD7F8EC00FEF71AF994ED060A88
:107C00000121B1EE400AD6F8240D7AF011FFD6F822
:107C1000240D05B0BDEC028BBDE8F0437CF058BAF2
:107C2000D7F8EC00FEF704F99FED100A0021EAE70F
:107C30009FED0E8AD7F8EC008DED038AFEF7F8F879
:107C4000D6F8240D0123B0EE480A03AA04F114016A
:107C50007BF0F4FCDBE700BF4459002000007A44CD
:107C60000000FA43CDCCCC3D087C00200000000091
:107C700030B590F8B83185B00446F3B1684611F0DC
:107C8000F3F8414869460AF0CDFF50B104F13C00D9
:107C900029F010FB002384F8B83104F59A7026F01F
:107CA00079FC94F890310B2B2DD8DFE803F0294BA9
:107CB0004F534B572C5B5F632C6700F59A7026F08F
:107CC00069FC04F13C0590B194F84030012B0ED1D1
:107CD00094F89031012B0AD1284629F059F950B176
:107CE0002046FEF7CDF9294A02214EF069FA2846CE
:107CF00029F07CF9D5E72046FEF7C2F9244AF3E7DC
:107D00002046FFF75BFB94F844303BB994F84630CB
:107D100023B994F840309A1E5342534194F8B92144
:107D200082B37BBB84F8B9311A4BD3F8EC000368FB
:107D30001B689847014618482D2205B0BDE8304021
:107D40004BF052BC2046FFF74DFBDCE72046FFF727
:107D500087FBD8E72046FFF79BFBD4E72046FFF7D9
:107D60009DFBD0E72046FFF7CFFBCCE72046FFF78F
:107D700009FCC8E70948FFF75BFDC4E72046FFF7A9
:107D8000D1FCC0E705B030BD303F002044FE0C08F8
:107D90006CFE0C08805C0020703C00203C850020BC
:107DA0002DE9F0412DED028B074684B008460E46C2
:107DB00011F08AF8032880466D4628D1FB681868C0
:107DC0007CF074FE012822D12148294607F0CCFF1F
:107DD0000446B0B17B69DDED007A1B68F8EEE77A06
:107DE00093EDF27A77EEC77A4246FDEEE77A17EE28
:107DF000901AC829CDED007AB8BFC821304611F0DD
:107E000039F8204604B0BDEC028BBDE8F081114B7F
:107E10000FCB85E80F00304611F056F80146284692
:107E200011F0BAF804460028EBD07B69DDED017A49
:107E30001B68B8EEE78AD3EDF27A284638EE678AF7
:107E400011F042F8BDEEC88A024618EE101AD5E7C6
:107E5000802C00207079002010B543699FED126AD4
:107E60001B68D3EDF06A93EDF17AD3EDF27A86B028
:107E700066EE866A27EE067A67EEC67A68460C4694
:107E8000CDED006A8DED017ACDED027A25F05EFE32
:107E900003A920468DED030ACDED040A8DED051AE8
:107EA00011F042FB06B010BD0AD7233C30B50832B2
:107EB00004461D460FCA84E80F00134301BFAB6898
:107EC000A360EB68E360636885B093B9204610F067
:107ED000FBFF03AA0146284611F002F860B103999E
:107EE0000191204610F0F0FF01990246204610F063
:107EF000C1FF204605B030BD696801912846F1E711
:107F000030B50B6985B004460BB94B6953B30023F8
:107F1000C4F8B43108310FC96D4685E80F00294611
:107F20002046FFF73DFF98B9124B0122D3F8F41C0D
:107F3000284610F09FFF4CF045F8022215214BF027
:107F40009DFF2046FEF79CF80B4A02214EF038F9BF
:107F500029462046FFF716F810B90848FCF718FA2A
:107F600005B030BD0123C0F8B43105B0BDE83040E4
:107F7000FFF78AB8806C0020A0FE0C08802C00203F
:107F800070B51A4B04460E460FCB88B06D4685E897
:107F90000F0020462946FFF75FFFE36818687CF072
:107FA0001FFF98B1E368186803681B69984768B1B8
:107FB000E368294618687CF085FD38B94AF00EFB65
:107FC00040F295624FF480114AF0C0FA214604A8AD
:107FD0002B463246FFF76AFF04A92046FEF7D2FF80
:107FE00010B90348FCF7D4F908B070BD70790020CF
:107FF000802C002070B5154B0C4606460FCB88B080
:108000006D4685E80F0029463046FFF725FF2B46D1
:108010002246314604A8FFF749FF6288A388122A46
:108020004FEA132305D1227ED20744BF03EB83031B
:108030005B00227A07EE903AC2F34002B8EE670A7C
:1080400004A93046FFF7B6F808B070BD707900207B
:1080500038B504460D46FFF793FF0023C4F894316A
:10806000AB88A4F8923138BD7FB50D460446FFF7C2
:1080700087FF05F108010FC96E4686E80F0013431C
:1080800006D1234BD3F8F82CD3F8FC3C029203938F
:1080900004F5D0720121304610F022FF94F8983197
:1080A00070B923F0050343F0050384F898312046A6
:1080B000FDF7E6FF174A06214EF082F804B070BDC6
:1080C00023F0070384F898310023C4F89C31E36857
:1080D00062691B68106893ED080A93ED0C1AD3EDE2
:1080E000070AB0EEC00A7AF00DFCE36862691B680B
:1080F000106893ED080A93ED0C1AD3ED070AB0EE61
:10810000C00A7AF079FC08212046FEF787FDD5E702
:10811000806C0020CCFE0C082DE9F0438DB06D463C
:1081200088461C46074613460A4601462846DDE9AE
:108130001469FFF7BBFE95E80F0084E80F0007A85D
:1081400010F092FEB8F80430F3B9B8F8001001311D
:1081500005AA89B207F13C0028F0C6FAA0B123466F
:1081600005AA39462846FFF7A1FE95E80F0086E8E4
:108170000F00BDF81630A3F152025342534189F863
:1081800000300DB0BDE8F08394E80F0086E80F00E2
:108190000023F4E770B58B8892B004460D4616466E
:1081A000002B47D10DA810F05FFE298801310BAAE2
:1081B00089B204F13C0028F097FA00283AD0BDF8C3
:1081C0002E1052291CD019D8112913D80F2913D9D0
:1081D00033462A46214603A8FFF768FE03AB214633
:1081E00007A80BAAFFF762FEE36807A918687DF0ED
:1081F0005DF901E01329EBD012B070BD5E29FAE7FA
:1082000007AD03A810F030FE284610F02DFE0DF14A
:108210000B03CDE90053324603AB0BA92046FFF711
:108220007BFFE0689DF80B3000682A4603A97DF0CB
:1082300013F9E1E70120DFE770B5214B04460E4654
:108240000FCB88B06D4685E80F0020462946FFF722
:1082500003FEE36818687CF0C3FD98B1E368186812
:1082600003681B69984768B1E368294618687CF081
:1082700029FC38B94AF0B2F940F216624FF4801185
:108280004AF064F9214604A82B463246FFF70EFE59
:1082900004A92046FEF776FE20B90A48FCF778F8D4
:1082A00008B070BD0023C4F89431B388A4F89231AB
:1082B00004AA31462046FFF76DFF0028F0D1ECE715
:1082C00070790020802C0020F0B5324B04460E4619
:1082D0000FCB91B004AD85E80F0020462946FFF78B
:1082E000BBFDE36818687CF07BFD98B1E368186813
:1082F00003681B69984768B1E368294618687CF0F1
:10830000E1FB38B94AF06AF94FF4DF624FF48011AB
:108310004AF01CF90CAF08A810F0A6FD384610F082
:10832000A3FD0DF10F03CDE900732A4608AB3146DA
:108330002046FFF7F1FEE0689DF80F3000683A46EE
:1083400008A97DF0CFFB20B91348FCF721F811B044
:10835000F0BD0023C4F89431B388A4F8923108AA80
:1083600031462046FFF716FF0028EDD00B4B1B6867
:10837000022B09D0032B03D1094B93F9D9321BB13E
:1083800006480021F9F758FF01212046FEF746FC78
:10839000DDE700BF70790020802C0020EC840020F5
:1083A000804C002037B504460D4686F029FEC4F8FF
:1083B000A801D5ED027AF5EEC07AF1EE10FA17DDDC
:1083C0009FED137A67EE877AFCEEE77AC4ED697A5F
:1083D0002046FDF755FED4F8A4214FF47A73B2FB82
:1083E000F3F30C4A062103B0BDE830404DF0E8BE7F
:1083F00063F006FC0023009395F90D2095F90E30EB
:1084000095F90C1063F098FBC4F8A401E0E700BFF5
:1084100000007A44E4FE0C0810B5B1F90A30A0F867
:10842000BC3191F90C3080F8BE31B1F90D30A0F8B3
:10843000C031B1F90F3007EE903AF8EEE77A044612
:10844000C0ED717A86F0DCFD0B21C4F8C80120462E
:10845000BDE81040FEF7E2BB38B504460D4686F095
:10846000CFFDC4F8B001D5ED027A9FED047A67EE36
:10847000877AFDEEE77AC4ED6B7A38BD00007A4466
:108480004A7C06480B46003A91F91010D3ED030AD6
:1084900093ED020A18BF0122F9F7D8BEEC84002040
:1084A00070B51B4E0446D6F8EC00036886B01B6816
:1084B0000D469847042806D16B88102B0FD0732BDC
:1084C00020D000201CE0D6F8EC0003681B68984719
:1084D0000328F6D194F89031062BF2D1ECE705F1A0
:1084E00008010FC902ACDFED0B0A84E80F0000237E
:1084F00009480093B0EE600A1A46214603F0C2F91B
:1085000006B070BD20462946FFF7BAFF0120F7E705
:10851000805C002000000000FC80002038B5D1F80D
:10852000093007EE903AF5EEC07AF1EE10FA054602
:108530000C4605DD0B7A022B03D01ED9032B0ED07F
:1085400038BD154B9FED150AD3F8280D27EE800A8C
:108550007CF0DCFBD4F80930C5F8D031F0E70E4BE5
:108560009FED0E0AD3F8280D27EE800A7CF0DEFB83
:10857000D4F80930C5F8D431E2E7074B9FED070A7C
:10858000D3F8280D27EE800A7CF0DEFBD4F8093002
:10859000C5F8CC31D4E700BF806C00200000C84291
:1085A00038B5114D0C4605F6BC5095F8351E59F0FE
:1085B0002FF858B195F8351E05F6BC5059F030F833
:1085C00020B994ED040A0948F9F7DEFE94ED041A87
:1085D000D4ED020A94ED030A95F8351E0448BDE86F
:1085E0003840002259F054B8806C0020EC84002000
:1085F0003C7A0020F0B50B69214F85B005460E4648
:108600000BB94B6953B300233B7006F108030FCB42
:108610006C4684E80F0021462846FFF7C1FB98B955
:10862000184B0122D3F8F41C204610F023FC4BF029
:10863000C9FC022215214BF021FC2846FDF720FD44
:10864000114A02214DF0BCFD21462846FEF79AFC56
:1086500038B90E48FBF79CFE05B0F0BD3846FEF772
:108660004FFEB38807EE903AF8EE677A0921284664
:10867000C7ED017A05B0BDE8F040FEF7CFBA00BF04
:108680003C850020806C0020F4FE0C08802C00202B
:1086900010B5044C237813B1034867F0B5FA20787D
:1086A00010BD00BFF8850020307B0020007807282F
:1086B00094BF00200120704713B5094B0191044677
:1086C000D3F8280D03681B69984730B101992046FB
:1086D00002B0BDE81040FEF74FBA02B010BD00BFB7
:1086E000806C002090F8983113F0010018BFC3F39C
:1086F00080007047094A034692F8150668B192F85F
:108700001426043A012A07D85B6A1B6893F8A10073
:10871000431E58425841704700207047807C00201B
:1087200010B5044686F06CFCD4F8B031C01AD4F809
:10873000AC3123EAE37398424FF0000084BFC4F8E1
:10874000AC01012010BD000010B503680446DB6DCC
:108750009847D4F8AC3123EAE37398424FF0000015
:108760003CBFC4F8AC01012010BD000008B50448AE
:108770000321F9F741FDBDE808400148F9F760BE63
:10878000EC84002070B51C4B0446D3F8280D036818
:108790001B690E469847054610B90025284670BD4E
:1087A000D4F894315BB986F02BFCB4F89231C4F85C
:1087B000940123B1114A537843F00103537086F0BA
:1087C0001FFCD4F89421B4F89231801A4FF47A72D5
:1087D000B0FBF2F09842E0D323B9084A537843F053
:1087E000010353702046FDF74BFC3388044A0621F1
:1087F0004DF0E6FCD2E700BF806C0020DC86002054
:10880000A0FC0C0810B590F89031042B0446164BD0
:108810000AD1D3F8280D03681B69984718B1204680
:10882000FEF7AAFC002010BD0A79D3F8303DDFED39
:108830000F6A93ED0E6A07EE902A0A7E920748BFF0
:108840009FED0B7AF8EE677A48BF67EE877A86EE7F
:10885000267AB0EEC77AB4EEE77AF1EE10FAACBF42
:1088600001200020DFE700BF806C0020DB0FC94043
:108870000000803B13B5094B01910446D3F8280D45
:1088800003681B69984730B10199204602B0BDE8E2
:108890001040FEF771B902B010BD00BF806C00201F
:1088A00010B5044686F0ACFBD4F8A831C01AD4F851
:1088B000A43198424FF0000084BFC4F8A401012005
:1088C00010BD000038B505460C4686F099FBD5F87A
:1088D000C831C01A23894FF47A725343984294BF27
:1088E0000020012038BD0000C368186808B190F866
:1088F000B808704710B5012104460A4805F00EF883
:1089000028B120460321BDE81040FEF787B949F0A1
:1089100065FEBDE8104040F26B124FF4801149F043
:1089200015BE00BF5882002090F89031022B04D071
:10893000032B04D1034804F0C1BF0120704700207D
:10894000704700BF5882002038B50C4BD3F8885CC4
:1089500090F89031032B044605F004050AD108482D
:1089600004F0C4FF94F8903135B110B9023B58427D
:10897000584138BD0020F5E70120FAE7804C00207F
:108980005882002010B50F4A137843F0800313700B
:108990000D4B93F9E020002A044609DBFEF73AFA72
:1089A00070B920460822BDE810400921FDF73ABA07
:1089B000BDE8104001220E21A3F50270F5F712BBAD
:1089C00010BD00BFDC860020805C0020F8B5D0F828
:1089D000B44105465CB1012C1AD049F0FFFD40F6C8
:1089E00043024FF4801149F0B1FD012407E0184B18
:1089F000D3F8280D03681B69984710B90024204656
:108A0000F8BD2846FEF740FB0123C5F8B431F6E770
:108A1000104F97F9E030002BF0DA436A1B6893F8A7
:108A2000A160012EEAD13C3027F0B4FE04460028B4
:108A3000E5D1D7F8103193F8CB3033B132460D2160
:108A4000A7F50270F5F7CEFAD9E73446D7E700BFAD
:108A5000806C0020805C002038B56E4BD3F8EC2091
:108A60006D4B9A4204460D4601D0002072E04B88BF
:108A70005E2B55D8512B0CD8103B9AB20F2A29D90E
:108A80002046FDF7FDFA6B88644A04214DF098FBFF
:108A900059E0523B0C2BF3D801A252F823F000BF4F
:108AA000F78B0108818A0108B98B0108CD8B010879
:108AB000818A0108818A0108818A0108818A010866
:108AC000818A0108818A0108818A0108FD8B0108D9
:108AD000D58B01080F2BD3D801A252F823F000BF89
:108AE000C78B01086B8A0108DD8B0108E38B010845
:108AF000F18B0108CD8B0108B98B0108818A01082F
:108B0000818A0108818A0108818A0108818A010815
:108B1000818A0108818A0108818A0108E98B01089C
:108B2000732B74D006D8702B6ED0722BA8D1FFF7A0
:108B30000BFE44E04AF2CF62934262D0A0D8B32B3E
:108B400009D8B12B9CD92046FDF79AFA298851F013
:108B500023FD012038BDBC3B9AB2132A90D8132BB9
:108B60008ED801A252F823F0478B0108478B0108E9
:108B7000818A0108818A0108818A0108818A0108A5
:108B8000818A0108478B0108818A0108478B010807
:108B9000818A0108818A0108818A0108478B0108BE
:108BA000818A0108818A0108818A0108478B0108AE
:108BB000818A0108478B01082046FFF769FD0028DC
:108BC0003FF453AFBFE7FFF7DDFDF8E72046FFF7BF
:108BD000FDFEF4E71248FFF769FDF0E7FFF712FE2C
:108BE000EDE7FFF769FDEAE7BDE83840FFF77ABD3A
:108BF000FFF780FDE3E7FFF73DFEE0E7FFF750FEFC
:108C0000DDE7FFF75FFEDAE7FFF78AFDD7E7FFF75B
:108C1000ADFDD4E7805C0020087C002028FF0C0814
:108C20003C85002090F89031032B0BD0062B06D00A
:108C3000012B0AD1C368186803681B6818470448E9
:108C400002F012BA034804F0C3BE0020704700BF10
:108C5000FC800020588200208B88012B05D00B69F6
:108C60003BB94B692BB9CB681BB904480021F9F714
:108C7000F7BE024800220831F9F714BF802C00200B
:108C800010B54B885E2B04460A464DD8512B05D8AB
:108C9000103B99B20F2921D900209DE0523B0C2BAB
:108CA000FAD801A151F823F0138E0108998C01081C
:108CB000CD8D0108E38D0108998C0108998C01087C
:108CC000998C0108998C0108998C0108998C0108EC
:108CD000998C01081B8E0108238E01080F2BDBD80D
:108CE00001A151F823F000BFDB8D0108ED8D0108D3
:108CF000F58D0108FD8D01080D8E0108E38D010839
:108D0000CD8D0108998C0108998C0108998C010876
:108D1000998C0108998C0108998C0108998C01089B
:108D2000998C0108058E0108B32B00F0848016D8B9
:108D3000732B7DD00ED8702B77D0722BACD1D1EDA8
:108D4000027A9FED447A67EE877AFDEEE77AC0ED0E
:108D50006B7A40E0B22B9FD1FFF7E0FB3BE0CD2BDD
:108D60002CD8BB2B98D9BC3B112B95D801A151F81D
:108D700023F000BFD78D0108D78D0108998C010819
:108D8000998C0108998C0108998C0108998C01082B
:108D90003D8E0108998C01083D8E0108998C0108CF
:108DA000998C0108998C01083D8E0108998C010865
:108DB000998C0108998C0108498E01084AF2CF620A
:108DC00093427FF469AFFFF727FB04E002F108014B
:108DD0002046FEF745F8012010BD1146FFF72CFA9A
:108DE000F9E711462046FFF78BF8F4E71146FFF745
:108DF000C7F8F0E71146FFF7FDF8ECE71146FFF77B
:108E000027F9E8E71146FFF72FF9E4E7FFF772FDCE
:108E1000E1E71146FFF758FADDE71146FFF7C2FA1E
:108E2000D9E71146FFF7E6FBD5E7FFF715FBD2E7D9
:108E3000FFF726FBCFE7FFF70FFFCCE7064802F16D
:108E40000801F9F7C1FAC6E711462046FFF7A8FB6B
:108E5000C1E700BF0000C842EC840020704700005A
:108E6000704700007047000090F8280080F0010073
:108E700070470000024B436040F6050303817047D2
:108E80000001020490F85501704700000F20704760
:108E90000020704700207047002070470020704776
:108EA00000487047D4FF0C0800487047E0FF0C08EA
:108EB00008B5094800F50053D3F8DC3CB3F9083095
:108EC00000EE103AB8EEC00AF5F726FBBDE8084000
:108ED0000248FCF709BF00BF802C0020E07D002085
:108EE00010B514482DED028B1C4600F5005300F51B
:108EF0008040B3F9A832D0F81C0D08EE103A036890
:108F000082B09B6ECDE900219847B8EEC88AF0EE9A
:108F1000400ADDE90021B0EE480A0748FCF734FBBF
:108F20000548FCF743FF84ED000A02B0BDEC028B5C
:108F300010BD00BF802C0020E07D0020F8B51C4D46
:108F400005F5005405F580462846D6F8247DF5F74A
:108F5000D1FAB4F9E43201EE103AB4F9E23200EE9B
:108F6000903A434200EE103AB8EEC11AF8EEE00A29
:108F7000B8EEC00A384679F0C5FC2846D6F8246D0C
:108F8000F5F7B8FAB4F9E43201EE103AB4F9E23286
:108F900000EE903A434200EE103A3046B8EEC11A65
:108FA000BDE8F840F8EEE00AB8EEC00A79F024BD5A
:108FB000802C002038B5144C04F5804504F57F64FE
:108FC000D5F81C0D03689B689847692100F194024D
:108FD000204649F0E1FFD5F81C0D0368DB6898478F
:108FE0006A2100F19402204649F0D6FFD5F81C0D05
:108FF00003681B6998476B2100F194022046BDE885
:10900000384049F0C9BF00BF802C0020014807F05C
:109010000FB800BF802C00203C3084F0ABBB0000B8
:1090200008B549F0DBFABDE8084072224FF4801120
:1090300049F08CBA08B549F0D1FABDE8084066227B
:109040004FF4801149F082BA08B549F0C7FABDE87B
:10905000084080224FF4801149F078BA73B51F4D53
:109060000646D5F8EC0003681B6B9847044680B3AE
:1090700095F9E130002B2FDBD5F8103193F8CB4078
:109080003CB395F8E03003F0A003202B24D1D5F8B1
:10909000EC0003681B689847052808D0D5F8EC0059
:1090A00003681B689847A0F110035C425C410C4ABE
:1090B00002F550630193A2F500532146D3F8F43D25
:1090C0000093D2F8243DD2F81C2D304684F000FBEA
:1090D0000446204602B070BD0024FAE7805C002000
:1090E000806C00203C30FFF7B9BF000038B5114D4F
:1090F00004461148F5F7AAFE95F9E030002B14DA82
:10910000236A93F8A120012A06D0D5F8EC000021AB
:10911000BDE83840FCF756BB0D21A5F50270F4F709
:1091200061FF95F9E030002BEFDB2046BDE83840C9
:1091300084F00ABE805C0020802C00203C30FFF7C9
:10914000D5BF000001207047012070470120704703
:1091500001207047112070470120704700207047A0
:1091600000207047002070470048704724010D0818
:10917000004870472C010D0838B5436904461D6846
:1091800080697CF0FDFF25F01BF9DFED1B0A284606
:1091900079F09EF96369A0691D687CF0F1FF25F004
:1091A0000FF9DFED150A284679F00AFA63691868A5
:1091B0007AF0DAFB6369DFED110A18689FED0E1A89
:1091C000B0EE600A79F09EFB6369DFED0C0A186867
:1091D0009FED091AB0EE600A79F00EFC6369186819
:1091E00079F0A4FC18B9636918687AF023FE0023AB
:1091F0002364012038BD00BF00803B4400007A4357
:1092000070B52DED028B88B00446FCF7A3FA70B15F
:1092100020460021FCF7D6FA63699FED310A1868F1
:1092200008B0BDEC028BBDE870407AF0DFBE636A27
:10923000022118687DF05CFF2A4B93F8E1305B0651
:1092400003D56369186879F0C3F99FED258A6069D1
:109250008DED018A8DED028A8DED038A8DED048AF4
:1092600003AA01A90068012379F01CFA6369186850
:109270007AF090FC236A1D682B68DE6C63691868BD
:1092800079F064FD0122CDED060A8DED071A05A9DE
:109290008DED050A2846B0EE480AB0476369B0EE86
:1092A000480A186879F0B4FB636918687AF010FF0F
:1092B000236C8BB185F0A4FEE36BC01A236C98423B
:1092C0000AD309480C220521FCF7BAFB20B906484D
:1092D0000C220221FCF7B4FB08B0BDEC028B70BD80
:1092E00000000000805C0020802C002038B504467F
:1092F0000D4685F085FEC4E90F0538BD072070478F
:1093000001207047002070470020704701207047FF
:1093100000487047C4010D0800487047CC010D0893
:1093200070B52DED028B0025C36880F83C501B689A
:10933000DFED488AD3ED0A0A42699FED478A93ED33
:10934000060AF4EEE80A0446F1EE10FA88B0106856
:10935000B8BFF0EE480A79F0BBF8E36862691B68B1
:109360001068D3ED0A0A93ED060AF4EEE80AF1EE6E
:1093700010FAB8BFF0EE480A79F022F96369204686
:109380001E68FCF781FE6368B3F93820B3F9363004
:1093900000EE903A434201EE102A00EE103AB8EE89
:1093A000C11AF8EEE00AB8EEC00A304679F0AAFA1F
:1093B000636920461E68FCF767FE6368274CB3F9B3
:1093C0003820B3F9363000EE903A434200EE103ABE
:1093D00001EE102A3046B8EEC11AF8EEE00AB8EEF7
:1093E000C00A79F009FBD4F8300D7BF08DF9D4F880
:1093F000306D338B1B0723D504A80FF035FD09F022
:109400002DFE9FED170A044606F11C0024F0DAFB3E
:1094100001AA04A920468DED010ACDED020A8DEDC9
:10942000031A09F0E9FD80B10322294604A80FF0D0
:1094300021FD0C4B186804AA90F8791058F044FAF2
:1094400009480821F8F7D8FE012008B0BDEC028BCE
:1094500070BD00BF0000003400007A43806C002023
:109460000AD7233C68900020EC84002030B52DED15
:10947000048BC3689FED898A1B684269D3ED0A7A21
:10948000DFED870A93ED060AF4EEC87AF1EE10FAE2
:109490000446A8BFF0EE670A106889B079F018F8A2
:1094A000636920461D68FCF7EFFD6368B3F9382057
:1094B000B3F9363000EE903A434200EE103A01EE36
:1094C000102A2846774DB8EEC11AF8EEE00AB8EE39
:1094D000C00A79F017FAD5F8300D7BF057FAA5F5E8
:1094E000805393F80531D90747D4D5F8303D1A8B0E
:1094F000D20742D593ED0A9AB4EEC89AF1EE10FA6B
:10950000B8BF93ED049AE36A186855F05FFBD5F88D
:10951000283DD3ED067AA36B20EE270AD3ED007A1F
:10952000F0EE498AE0EE278AB0EE490AF5EEC08AED
:10953000F1EE10FAD8BFDFED5C8AF0EE680A20F099
:10954000E7FF28B9D5F8300DB0EE680A7AF09CFF35
:10955000636893F95130272B0FD0A36A186855F030
:1095600035FBF0EEC07AF4EEC87AF1EE10FAB0EE08
:10957000407A20D5002384F83C30236B1B68B3F974
:10958000083000EE103A2046B8EEC00AFCF73EFC68
:109590002046FCF7A9FB2046B0EE408AFCF7DAF83B
:1095A000002848D00021204609B0BDEC048BBDE85E
:1095B0003040FCF707B9D5F8303D9FED3C0AD3EDBC
:1095C0000F7AD3ED0B6AA36B27EE800AF4EEC86A1C
:1095D000D3ED007AF1EE10FA67EE277A10DB9FEDFB
:1095E000341ADFED310A552037EE800A21F094F865
:1095F000012384F83C30D5F8300D7AF035FFBCE714
:109600009FED2C7AF4EEC76AF1EE10FA05D89FEDC3
:10961000261ADFED290A5920E6E7F0EEE66AF4EEB5
:10962000C86AF1EE10FAE3D594F83C30002B08BF7D
:10963000B0EE670ADCE7636A022118687DF058FD26
:109640001E4806F0ADFBB0EE480AD5F8300D7BF0B1
:109650009FF801461A48FAF789FD636918687AF09D
:1096600037FD236A1D686369186879F06FFB05ACE4
:10967000204614498DED020ACDED030A8DED041A42
:10968000F8F7B0FF079B009394E80C0002A9284666
:1096900076F028FC09B0BDEC048B30BD000000342E
:1096A00000007A43806C002000000000E02E65423C
:1096B0000000B442000000B40000B4C2005A002010
:1096C000802C0020EC84002008B5064BD3F8303DF8
:1096D000D868243023F0C2FFFCEEC07A17EE900A5F
:1096E00008BD00BF806C0020024BD3F8303DD86825
:1096F00079F0D6BB806C00200B20704701207047AA
:1097000000207047012070470020704700487047D4
:1097100064020D08004870476C020D080120704774
:1097200008B5DFED237AF4EEE70AF1EE10FA2DED3D
:10973000028BF0EE408AB0EE608A35DDDFED1D7AF7
:10974000F4EEE70AF1EE10FA2ED5F6EE007A70EE9E
:10975000E77ADFED196A9FED190ADFED190AF0EEDD
:10976000E77A87EEA67A8720B7EE001A30EE470A2E
:1097700020F0D2FFDFED137A9FED131ADFED130A0D
:1097800020EE270A8A2020EE280A20F0C5FF30EEBE
:10979000080ABDEC028BDFED0A0ABDE808408D2007
:1097A000B7EE001A20F0B8BF9FED050AEFE700BF43
:1097B000AC1C5A3ED578493F8FC2753E9A99993F65
:1097C00000000000FAEDEBBA9A99993E9A9999BE79
:1097D00030B52DED048B7D4BB3F9A83200EE903AF5
:1097E000F8EEE00A83B0044601AA6946B0EE600ACA
:1097F000FBF7CAFEA0697CF0C3FCE369D0ED008AE8
:10980000D3ED946AD3ED977A90ED016AA3689FED4A
:10981000701ADFED700A27EEE80A68EEA68A03F6F2
:109820003813E6EE278A05463B20DFED6B7AB0EE73
:10983000E87AB4EEE77AF1EE10FA58BFB0EE677A44
:10984000DFED667AC7EE275AF7EE007A77EEE57A13
:109850009DED007A67EE877A93ED007A67EE877A5E
:109860009FED5F7AA6EE260A87EE879A20F054FFD6
:109870003C209FED571ADFED570AB0EE408AB0EE5C
:10988000680A20F049FF626B564B1268DFED567A8A
:10989000B2F90820D3ED006A9FED541ADFED540AA7
:1098A00007EE102AB8EEC77AF0EE408A27EE277A44
:1098B000DFED507AA6EEA77A4520F4EE007AA7EE07
:1098C000678ABAEE000A28EE000A83ED007A8DED71
:1098D000000A20F021FFDDED017A9FED477A474B2A
:1098E0008DED000AF0EEE77AF4EEC77AF1EE10FAA9
:1098F00051D593ED007ADFED427A77EE277AB2EE1A
:10990000007AF4EEC77AF1EE10FA58BFF0EE477A1B
:10991000C3ED007A67EEA87ACDED017A636A186824
:1099200090F8CB10002939D17DF0E2FB636A1B6807
:1099300093F8A110012939D0032940D039B9236AFD
:10994000186876F0B7FF236A186876F003FA236A7E
:10995000DDED010A18689DED000A0368B0EE491AB2
:10996000DB6A9847204695ED028AFCF709F8204605
:10997000F0EE400AB0EE480AFFF7D2FE236A6268B2
:109980001868D2ED020A036801215B6E984703B0A4
:10999000BDEC048B30BD00221A60BFE7194B93F970
:1099A000E130002BB4BF01210221BDE7236A186812
:1099B00076F080FF236A186876F0E2F9C7E7D97974
:1099C0000029C4D12046FCF755FBC0E7804C00209D
:1099D00000000C4400000CC40000FA4400409C4508
:1099E00000003442588500200AD7233D00A08C4552
:1099F00000A08CC58FC2753F000000345C8500203C
:109A00008FC2F53C805C00200E207047002070471C
:109A100000207047002070470020704700207047EA
:109A20000048704704030D080048704704030D0800
:109A300070B52DED028B436A1B6893F8CB3004465A
:109A4000FBB9052384F848302046FBF799FF636A89
:109A500002211868B0EE408A7DF04AFB94F950303C
:109A6000E2696BB3D2F8F8515D4394F84820052AB7
:109A70004FD8DFE812F02B005F008400B100DF0058
:109A80001E01836A1B68B3F90830002BB8BF5B4224
:109A90009BB2B3F57A6FD4D2C36A1B68B3F90830AE
:109AA000002BB8BF5B429BB2B3F57A6FC9D285F089
:109AB000A7FAE36CC01A40F6C4139842C1D8C3E7B2
:109AC00094F95150D2F8FC215543CEE7226A94F91B
:109AD000511010689FED801A49F64042534351439C
:109AE00000EE103A00EE901A0268F8EEE00A926B6F
:109AF000B8EEC00A9047DFED797A41F293139D42A8
:109B000038EE278A05DD94F950308BB1012384F8B3
:109B10004830236A62681868D2ED020A0368B0EE22
:109B2000480ABDEC028B5B6EBDE87040002118470F
:109B30000223ECE7226A9FED681A106849F640425A
:109B4000534300EE103A0268B8EEC00A926BF0EE92
:109B5000410A9047DFED627A38EE678A05F50C55C9
:109B6000B5EEC08AF1EE10FA05F1270543F2BA43CB
:109B7000D8BF9FED598A9D42CBD80423C7E7236AFB
:109B80009FED551A186894F9513049F640425343F5
:109B900000EE903A0268F8EEE00A926BB0EE410AED
:109BA0009047DFED4F7AE36938EE678AD3F8F831F2
:109BB000B5EEC08AF1EE10FAD8BF9FED478A002BB0
:109BC000B8BF5B4242F228329342A2DD41F29413C5
:109BD0009D429EDD03239AE7236A9FED3F1A186892
:109BE00094F9513049F64042534300EE903A0268EE
:109BF000F8EEE00A926BB0EE410A9047DFED387A5A
:109C0000E36938EE678AD3F8F831B5EEC08A03F518
:109C10000C53F1EE10FA03F1270344F24E62D8BF61
:109C20009FED2D8A93423FF674AF2E4B9D42FFF677
:109C300070AFA2E7236A94ED111A1868D4ED100AE8
:109C4000036894ED0F0A1B6B00219847DFED237A20
:109C500094F95020E36938EE278A1AB393ED7E7A9F
:109C6000D4ED0F7AB8EEC77A77EEC77A9FED1E7AF9
:109C7000F0EEE77AF4EEC77AF1EE10FA3FF649AF6C
:109C80000D2294F849101948FBF7DAFE024618B97C
:109C900001461648FBF7D4FE4AF094F916214AF023
:109CA000CDF836E793ED7F7AD4ED107AB8EEC77A27
:109CB000DAE70D2294F849100C48FBF7C1FE024682
:109CC00018B901460948FBF7BBFE4AF07BF90222AE
:109CD0000D214AF0D3F81CE700000000CDCC4C3E2B
:109CE0008FC2753E6DEEFFFF0000FA43802C00200E
:109CF00073B5474D0446D5F8EC0003685B6B984795
:109D000018B90026304602B070BD95F9E130002B3D
:109D10005FDBA36A1B68B3F90830002BB8BF5B4256
:109D20009BB2B3F57A6FECD2636A1B6893F8CB6091
:109D3000002EE6D095F9E030002BE2DBD5F8EC0000
:109D400003681B689847002584F8490084F8485048
:109D500085F056F9E36AE064A4F850501B68B3F943
:109D60000830B3F5967F43DD012384F851304AF083
:109D700029F915214AF062F8264BB3F9A83201EE11
:109D8000103AE369B8EEC11A93ED7E0A8DED011A1F
:109D9000F1EE410A5320B8EEC00ACDED000A20F0E2
:109DA000BBFCE36984ED0F0A93ED7F0A9DED011A78
:109DB000DDED000AB8EEC00A542020F0ADFCE369E6
:109DC00084ED100AD3ED807AF8EEE77AC4ED117ACB
:109DD00098E7D5F8EC0003681B689847012890D0F5
:109DE000D5F8EC0003681B689847002891D188E7F4
:109DF00013F5967F01DAFF23B7E7A36A1B68B3F96F
:109E00000830002BACBF0123FF2384F85030AEE7AD
:109E1000805C0020804C0020162070470020704796
:109E200000207047012070470020704781F001003A
:109E30007047000001207047004870479C030D08E0
:109E4000004870476CE40C0803681BB1007900F00F
:109E50000100704718467047F0B5494D95F9356EC9
:109E600085B00446A5F50055002E00F085804548D4
:109E7000FFF7EAFF064600287ED0636920461F6888
:109E8000FCF702F96368B3F93820B3F9363000EE15
:109E9000903A434201EE102A00EE103AB8EEC11A91
:109EA000F8EEE00AB8EEC00A384678F02BFD636998
:109EB00020461F68FCF7E8F86368B3F93820B3F967
:109EC000363000EE903A434200EE103A01EE102A8E
:109ED0003846B8EEC11AF8EEE00AB8EEC00A78F0DB
:109EE0008BFD05F58043D3F8240D78F01FFE18B9DB
:109EF0006369186879F09EFFB5F9A43004F13C005D
:109F00001BB9B5F8A230A5F8A430B5F8A43007EE17
:109F1000903AF8EE677A04F1980203A90027CDED94
:109F2000037A4BF015FD04F15C00C4F8A0700190B9
:109F30006CF072FF002384F8A530B5F9A4300198C5
:109F40001BB9B5F8A230A5F8A430B5F8A43007EED7
:109F5000903AF8EEE77AB7EE000A80EE270A6CF046
:109F60007FFF09487CF008F9C4F8C870DFED077A74
:109F700020EE270A84ED310A304605B0F0BD00BF5F
:109F8000804C0020B05A0020807900200AD7233C62
:109F900010B50446FBF7BCF92046154B40F83C3B96
:109FA0004BF062FC134B2365134B9FED142A9FED7E
:109FB000141ADFED140A9FED140A6365F1EE041A1A
:109FC00004F15C006CF062FF002320460F49C4F8E6
:109FD000A830C4F8AC30C4F8B030C4F8B430C4F819
:109FE000B830C4F8BC3042F0BDFB204610BD00BF05
:109FF000A4040D08CDCCCC3D000040400AD7233B43
:10A0000000803B459A99993ECDCC4C3E3C040D08CE
:10A010002DE9F0432DED028B9BB0914604460D4691
:10A0200084F0EEFFB8499FEDB98A0646A1F1080019
:10A0300023F046FA94ED161ACDED110A7E20F1EECA
:10A04000410A8DED100A20F067FB94ED161A8DED94
:10A05000100AF1EE410A7F209DED110A20F05CFB11
:10A0600010A904F13C008DED110A4BF08FFCA848BB
:10A07000CDED130A8DED120A7CF07EF8D4ED327A24
:10A08000D4ED140A94ED151AE0EE087A892004F153
:10A090005C074FF00008B0EE670A20F03DFB12A805
:10A0A00023F05AFA9B4812A909F02AFA14A9384653
:10A0B0008DED140ACDED150A6CF08EFD3846CDF805
:10A0C0005880CDF85C806CF0CBFD8DED160ACDED9F
:10A0D000170AB9F1000F00F001810123C4F8D06024
:10A0E00084F8CC308C4E04F1A80116A823F010FAA5
:10A0F000B6F9A83200EE103A16A8B8EEC00A23F05E
:10A100002BFA16A9A6F5556009F0E6F918A9284614
:10A110008DED180ACDED190A23F0FAF9B6F9A83237
:10A1200095ED007A07EE903AF8EEE77AB0EEC77A4E
:10A13000B4EEE77AF1EE10FA00F3CE8095ED017AF5
:10A14000B0EEC77AF4EEC77AF1EE10FA4CBF0123F5
:10A15000002384F8A530B6F9A83295ED000A5A42DA
:10A1600007EE903A00EE902AB8EEE71AF8EEE00A11
:10A17000CA2020F0D1FA85ED000AB6F9A83295ED93
:10A18000010A5A4200EE902A07EE903AF8EEE00AF1
:10A19000B8EEE71ACB2020F0BFFA85ED010A94F85B
:10A1A000A4305A1C84F8A4201422B3FBF2F102FB61
:10A1B0001133DBB2002B34D149F004FF064684F0A2
:10A1C00027FF8046D4F8AC000F46F2F79DF9CDE9A1
:10A1D0000E01D4F8A800F2F797F9CDE90C01D4F8F4
:10A1E000A000F2F791F9CDE90A016868F2F78CF95D
:10A1F000CDE908012868F2F787F9CDE9060113983F
:10A20000F2F782F9CDE904011298F2F77DF9CDE970
:10A210000087CDE90201414B414A4249304649F0AD
:10A2200047FC1BB0BDEC028BBDE8F08312A823F005
:10A2300015FADFED3D7AB4EEE70AF1EE10FA57D4E5
:10A2400094F8CC3063B956E038466CF069FD94F868
:10A25000CC3084ED2A0AC4ED2B0A002B3FF442AF28
:10A26000DFED325ADFED324A9FED324ADFED323A0E
:10A2700012AA2B4605F10801B2EE0E5AB7EE003ACB
:10A28000B2EC016A94F99D00B0EEC67A67EE256AD9
:10A2900007EE900A76EE842AF8EEE77AB0EE647A5A
:10A2A000A7EE857AC3EEA27A27EE087A77EE837A54
:10A2B00027EE267AB5EEC06A67EE877AF1EE10FADD
:10A2C00048BFF1EE677AE3EC017A9942D8D1CDF834
:10A2D0005C80CDF8588005E701233AE794F8CC304C
:10A2E0004BB1D4F8D00040F6B833361A9E429DD90F
:10A2F000002384F8CC3094F8A530002BA4D1384644
:10A300006CF074FDA3E700BFDC5A00200AD7233CA1
:10A3100080790020303F0020804C002040CF0C0886
:10A32000A8030D086CE40C089A99993E0000C842F5
:10A330000000BE42000070420000FA432DE9F04FD9
:10A340002DED048B0446A5B0BD487BF015FFBD4B39
:10A35000DFEDBD7A1B68DB6A93F89C3060EE278ADC
:10A3600033B9F1EE687AC4ED327AC4ED318A47E050
:10A37000B64D05F54053D3F8103193F8A090B9F1DC
:10A38000020FEED184F03CFE05F58043D3F8343D56
:10A39000C01A40F2DB539842E3D99FEDAD8A95F89D
:10A3A000DB1B8DED218A18AB21AA05F6C8008DEDC7
:10A3B000228A8DED238A1EF0D7FC08B3A54821A977
:10A3C00021F080FAD4ED2C7A8DED210A37EE800A47
:10A3D000D4ED2D7ACDED220A77EEA00A9E4884EDC9
:10A3E0002C0AC4ED2D0A8DED231AFFF72DFD60B95F
